:020000040800F2
:10000000006000204529010895290108952901086B
:1000100000000000000000000000000000000000E0
:100020000000000000000000000000009529010809
:100030000000000000000000952901083DB60008FE
:100040009529010895290108952901089529010894
:10005000952901088DB600089DB60008ADB60008C8
:10006000ADCE0008952901089529010895290108B8
:100070009529010889AA0008A1AA0008A9AA0008D0
:10008000C1AA00080000000000000000D9AA000872
:1000900000000000F1AA000809AB000811E7000801
:1000A00079E700089529010895290108A5CB0008E2
:1000B000C5CB0008000000000000000000000000A8
:1000C000030001221040134205D1042B02D9186805
:1000D000000980B270470020FCE7C30711D4042850
:1000E0000FD90F2302681340032B0AD119400133A3
:1000F0005B1AC0215B07C9050B4002490A40134344
:1001000003607047FFFFFF9F03000122022013429C
:1001100005D11000042B02D918680F23184070472E
:1001200010B50400FFF7CCFF002809D0421E830061
:1001300004349000225C002A02D001309842F9D1A8
:1001400010BD0378002B03D05AB2002A01DB013026
:1001500070473F229343C03B59424B41C01803783C
:100160009343802BF4D10130F9E710B500240378D4
:10017000002B01D1200010BDFFF7E3FF0134F6E7AB
:10018000020000787F2809DDDF2808DCF8238001E1
:10019000DB00184053783F22134018437047EF2884
:1001A0000BDCFC21537809019B010007000C0B407C
:1001B000034390783F221040EFE7F72812DCFC2140
:1001C000537889021B030B40E02180044903084057
:1001D00003433F20D17801409078FC220B438001FB
:1001E0001201E8E701204042D8E710B57F2902DC80
:1001F0000170013010BD80231B0199420CDA4023AD
:100200008A115B42134303703F2280230A405B4202
:10021000134343700230EDE780235B02994210DA0A
:1002200020230A135B4213433F24802203708B1167
:10023000234052420C4013432243437082700330E8
:10024000D8E788235B029942D4DAF0230370603B3D
:100250004370113B8A11FF3B1A4382703F221140C9
:100260000B43C3700430C5E7064B1B6818680009D0
:1002700080B20238C343DB17184043000120184303
:100280007047C04670040020024A5368013353602F
:100290007047C04670040020024A1369013313619D
:1002A0007047C04670040020024AD3690133D3610D
:1002B0007047C04670040020024A936A013393627B
:1002C0007047C04670040020002802DD0B68DA0782
:1002D00004D41122074B1A70002070475B10013BB9
:1002E000032BF9D80C214B43034AD2180023536047
:1002F000F2E7C046A4040020700400200A4B002846
:1003000003DD01200A68024204D1112200203433A7
:100310001A7070470C215210013A4A439B185B68CF
:100320005B001843F5E7C0467004002010B5036871
:10033000984710BD012A02D1016000207047022AAF
:1003400005D0032AF9D0002AF7D10260F5E70B683F
:100350000360F2E770B50E000400FFF7B1FE050080
:100360003000FFF7ADFE0023854206D1231DAD000E
:1003700004365D19AB4202D30123180070BD197811
:1003800032780C001443F7D0013301369142F1D09A
:100390000023F2E7020010B5152813DC0B4B0C4CC0
:1003A0001B680C494000234208D11B02085E1B0A4F
:1003B000012B06D0042A04D1074802E009182C2397
:1003C000C85E10BD01204042FBE7C0460470FF1F1D
:1003D000F0FFFF0068420108110200000020704792
:1003E000002070470420704704207047002804DC78
:1003F0001C22054B1A70002070470B68DB07FAD4EB
:100400000D22014BF6E7C046A4040020012300287A
:1004100003DC1C22024B1A70002318007047C046F0
:10042000A4040020C3070BD4064B9A6B824207D862
:10043000DB6B834204D3031F1B68002B00D0180022
:100440007047C04670040020F7B501272E4C2F4A94
:10045000A16BE06B2E4E082513682B4225D1136843
:100460001B099BB202339B00D218B242F3D3002582
:10047000284E3068FFF7D6FF013501C6802DF8D130
:10048000254D2868FFF7CEFF2860206C002802D099
:10049000FFF7C8FF2064636C002501931F4B1E000B
:1004A0000093019B9D4218DBF7BD1B099BB29B008B
:1004B000D3189A42D3D01D68AC463D420BD1A94215
:1004C00009D2A84207D304256D42AC4465462D6885
:1004D000002D00D01D60043BEBE73378002B02D1E8
:1004E0000135F036DDE73C246C433369E4185F1EC8
:1004F000009BA400E418043C002FF1DBA069FFF787
:1005000091FF013FA061F6E770040020CC29002094
:10051000F8450020BC11002000000020BC13002082
:100520000123F0B59C4685B0184248D1254B9A6B03
:100530000092904243D3DB6B019398423FD8031F54
:100540001B68002B3BD1020003681B099BB2002BE8
:100550001ED09900029102995618614634680C42E7
:100560002AD1009D2100A54226D8019DA54223D372
:10057000251F2F680395002F1ED127683D0717D52B
:10058000151F37602B60236822601B099BB20DE0AA
:100590006146131F1960904211D011680B1F1B6830
:1005A0009C000C192568013B156022600A00CEE70B
:1005B0006146039C2160CEE71100013BF6E705B0E0
:1005C000F0BDC046700400203622024B00201A7095
:1005D0007047C046A40400200E2300280BDD0A68E3
:1005E000D10708D4042A06D9126801331A40013B06
:1005F000042A00D10D33024A002013707047C04610
:10060000A40400200120034B034A1B685B00134035
:10061000184370470470FF1FFEFFFF010020014BCD
:100620009864704770040020002802DD0B68DB0727
:1006300002D40D22014B1A7000207047A404002040
:10064000002802DD0B68042B02D90C22014B1A7022
:1006500000207047A4040020F8B5040011F010FB3E
:1006600001000020144A1379032B0ED113681D00DA
:100670005B6808359B00013BEB189D4202D21E7857
:10068000002E09D05B1A9D4208D901300832FF289C
:10069000E9D10138FF3807E0013BEEE71D7801336F
:1006A000002DF2D1A94200DCF8BD5F5D665DB74266
:1006B000EBD10135F6E7C046E81D002010B583797F
:1006C00004003C2B18D81F4A99008858421C00D0BF
:1006D00018000FF0EFFCE3793C2B20D8194A990061
:1006E0008858421C00D018000FF0E4FC01235B4244
:1006F000E3800023236010BD3F2219009143C029ED
:100700000AD1CE2B08D810491A40920089188A6D58
:100710000C4892001058D9E701204042D9E73F2207
:1007200019009143C0290AD1CE2B08D806491A4096
:10073000920089188A6D034892001058D1E7012071
:100740004042D1E7444A01086842010810B5002838
:1007500002DD0B68DA0704D41122074B1A7000205F
:1007600010BD5B10013B032BF9D80C225343034807
:10077000C018FFF7A3FFF2E7A404002074040020D0
:1007800070B5040080790EF09FFD431E9841C5B2FC
:10079000E0790EF099FD431E9841227AC0B2002AFA
:1007A0001AD02279D1B2AA4208D00121226885420A
:1007B00000D1023952182260257170BD62798242DF
:1007C000FBD02268814204D101215218226060715D
:1007D000F3E701214942F8E701212268854200D16F
:1007E000023952182260E8E710B50248FFF7C8FF47
:1007F00010BDC0467404002010B50248FFF7C0FFCA
:1008000010BDC0468004002010B50248FFF7B8FFB5
:1008100010BDC0468C04002010B50248FFF7B0FFA1
:1008200010BDC04698040020F0B5B7B0040011F028
:1008300027FA01284CD923785B2B49D1013823189A
:100840000193235C5D2B43D1671C3A21380013F0E0
:10085000C0FB051E3CD0C61B002E39DD3900002729
:10086000320004A813F0C3FB04AB9F55019B691C25
:100870005D1ABD422CDD2A001DA813F0B8FB6422CE
:1008800004AB9B181A4E5F550197306800280CD0B6
:1008900004A911F0EBF9071E07D1B568002D04D0AB
:1008A00073680293029BBB4206DC019B0C3601334A
:1008B0000193112BE9D10BE028681DA9039511F0D4
:1008C000D5F9083500280CD1039B5868002806D1BB
:1008D0002000FFF7C1FE431C05D0064B184337B07C
:1008E000F0BD0137DEE71B22034B1A70F7E7C04665
:1008F0001C1D002000FFFFFFA404002010B50AF01B
:10090000C9F9431E9841800010BD204B10B5DC6C26
:100910000AF054F9002C02D11D4B984233D9012121
:100920001C4BDA688A43DA609A680A439A6080222C
:100930009868D20010439860586A08435862186A51
:1009400088431549186299610221D8688843D860A4
:1009500098680143996099680A4310219A605A6A1D
:100960000A435A621A6A8A431A620C4A09399A611E
:100970001A688A4303390A431A60094B1A691143FA
:10098000196130BF30BF002010BDC0467004002088
:100990003F4B4C00007000400100010002000100CC
:1009A00000ED00E010B5064C9AB002000B0001A863
:1009B000210013F0D5FA01A80AF082F91AB010BD8F
:1009C00037610108F0B5B9B00400029104920593B3
:1009D000102805D91B220020164B1A7039B0F0BD23
:1009E0000C2200274243144B9B185A689D680392BF
:1009F000039B9F420BDB029BC82100930F4A2300FD
:100A000006A813F079FA06A80AF05AF9E2E728686E
:100A100000280BD0029911F029F9061E06D16B6847
:100A2000059904989847064B1E64D7E701370835A7
:100A3000DEE7C046A40400201C1D00203E61010822
:100A400070040020F7B5454E7268002A71DBD3B2FE
:100A5000434F3C2B00D970E0424BD2B29200D358A6
:100A60005A1C5BD0B2680192934257D13C6D002C66
:100A700054D00122200025693B49EB681030934394
:100A8000EB602B6A0B4208D12B6A9C466146374BC0
:100A9000194202D12B6893432B60230001224D336E
:100AA0001A700093022300990B702B6A2E490B4297
:100AB00006D1296A2D4B194202D12B6893432B6032
:100AC0000BF08AFA28000BF0CDFA08F001FF20693C
:100AD0000BF0F8FA08F0FCFE2300002558331D70D7
:100AE0000A3B1D705D709D70DD701D715D719D71A3
:100AF000DD711D725D72009B29001D7023004C3357
:100B000001981D700AF0F1FD012320005B42B360E3
:100B100011F090F8200012F049FB3D6570685437E1
:100B20003B5C002B05D000210EF034FB00227368E3
:100B3000FA5401235B427360F7BD3F201A008243E1
:100B4000C02AEBD1CE2BE9D8094A03409B00D2182A
:100B5000936D04499B005B5882E7C046000000206B
:100B600070040020444A01081111000044040000F0
:100B70006842010810B5034811F00DFF4300012041
:100B8000184310BD57610108F0B5614C85B0237C56
:100B9000002B3CD101225F4B196E0A431A660222D8
:100BA000196E1142FCD001201A6C02431A641A6CAF
:100BB00002400092009A8022D96B52051143D963FA
:100BC000D96B114001910199DD6B0021154207D1CC
:100BD000D96B1143D963D96B0A4001000392039A80
:100BE000DA6D4D4DD20514D48022D86D9200284084
:100BF0000243DA65012929D10020DA6B47490A400E
:100C0000DA63002822D003214548FFF7CBFE05B068
:100C1000F0BD8020DA6DDF6D160040023843D865E4
:100C2000D86D404F2E403840D865DE65D207DBD501
:100C3000022066693C4FDA6D0242D5D16269921B8F
:100C4000BA42F8D903200129D7D0DCE78022D96D38
:100C500012020A438021DA65DA6BC9000A43DA63BB
:100C6000DB6B22000B400293029B00233C3213708B
:100C70007F222262803262628022E361A362E362A9
:100C80002363A3632300294DD2053D336263A5612D
:100C90001A7802221A70EB68DB0634D4CA236B621E
:100CA000773B6B620EF036FD00280CD00320FF224C
:100CB000A3695A62002826D003211D48FFF772FE5F
:100CC00001232374A3E7AB691A4A1340AB61E269BD
:100CD000AB691343A26A1343226B1343AB61236ACC
:100CE000626A1B0413432B610EF040FD0028DDD126
:100CF000616BA36BAA690B43E16AD2000B43D20874
:100D00001343AB61D3E7230001223D331A70D7E7C9
:100D1000F004002000100240FFFCFFFFFFFFFFEF88
:100D20005B610108FFFFFEFF881300000028004000
:100D30007B610108BFFF8FFFF7B50E0002284ADD77
:100D4000264C237C002B01D1FFF71EFF23003C33F0
:100D50001A78012A3FD0B26835680192012277687B
:100D60001A70230092183D331A70A369C8325A6270
:100D7000773A5A620EF0CEFC032300281FD1A669F1
:100D80006810C0B2B36909F0B5FC05007810C0B2B4
:100D900009F0B0FC019B00022D0405435810C0B2BD
:100DA00009F0A8FC0E4B284318403060B3690D4A87
:100DB0001340B361B369B3610EF0D8FC0300FF21A7
:100DC000A2695162002B03D1230001223D331A7026
:100DD00000233C3423700020FEBDC046F0040020F8
:100DE0007F7F7F00FFFFFBFF0023F0B585B00F0082
:100DF0000290019302285BDD2F4D2B7C002B01D14B
:100E0000FFF7C2FEFA233E68DB0076109E4201DD4A
:100E10002A4BF618BB687C680393029B6410E4B20B
:100E2000032B03D0FB685B10DBB201932B003C3338
:100E30001A78012A3CD001221A702B0092183D33F7
:100E40001A7010231C4202D09C430A34E4B2CA2216
:100E5000AB695A62773A5A620EF05CFC03230028B1
:100E60001AD1039BAF695810C0B209F043FC019B33
:100E70005B030343F0B2019309F03CFC019B0604C1
:100E800020001E4309F036FC0D4B00023043184091
:100E900078600EF06BFC0300FF21AA695162002B01
:100EA00003D12B0001223D331A7000233C352B70F7
:100EB000002005B0F0BDC046F004002030F8FFFF70
:100EC0003FFFFF00F0B50D0085B016000090002731
:100ED00010F072FDEC0F64196410009AFB00D0183A
:100EE000BC4218DCEB0712D50023013DAD00042203
:100EF000711902A8039311F076FF029A039BE14354
:100F0000C9170C400099E40008190FF0F3F910F02C
:100F100049FD05B0F0BDF1184A78F35C12021A439E
:100F20008B7801371B041343CA7812061A430B79D6
:100F300001929C4662464B791B0213438A79120444
:100F40001A43CB791B061343019A0FF0D3F9C4E778
:100F500070B54E680A00B51C29000400FFF7B2FF07
:100F600001231D40AD190235AD00601970BDFA2393
:100F70009B004343044A1364044B1A78002A01D1AE
:100F8000FF321A707047C046F0040020A40400200D
:100F9000030001220220134205D11000042B02D9C4
:100FA00018680F2318407047214B224A1B6800B570
:100FB0001802000A134205D11F4B012800D11F4B14
:100FC000180000BD11280FD80B2803D81C4BF7E7D9
:100FD0001C4BF5E70C380528F8D811F001F8151767
:100FE00019F72703184BEBE7184A154B8218072A05
:100FF000E6D8174BC018174B0628E1D810F0F0FFC1
:10100000E80A0C0E10121400134BD9E7134BD7E764
:10101000134BD5E7134BD3E7134BD1E7134BCFE774
:10102000134BCDE7134BCBE7134BC9E7134BC7E784
:101030000470FF1FF0FFFF008E6101089661010838
:10104000FC680108C26101089F610108FFFFF3FF0E
:10105000FEFFF3FFBB610108A6610108AF61010853
:10106000B5610108CC610108D9610108E06101089E
:10107000E6610108EC610108F4610108FF61010803
:1010800070B5054E0400335C0D008B4202D00EF0AB
:1010900081F8355570BDC046C4040020F0B5694BD9
:1010A0008BB0022803DC1C2234331A709DE001252A
:1010B0000E682E4205D04C682C4202D08F682F4219
:1010C00002D111223433F0E773100593013B0493EE
:1010D00000230393032805D0CB68043B59424B41BE
:1010E000DBB20393049B032B00D9A7E00C23049AE3
:1010F0005548534364107F10E6B2C018FDB2FFF7A5
:10110000DDFA3C2E00D973E0504BE2B29200D35886
:101110000193013301D0E3B201933C2D00D97AE071
:101120004A4BFAB29200D3580293013301D0FBB27A
:101130000293019B013300D180E0039B002B03D07D
:10114000029B013300D179E0FF2000212040FFF70E
:1011500097FFFF2000213840FFF792FF059B3C4F8F
:10116000023B022B03D83B4A9B00D218576906ACBE
:101170000C220021200011F0DBFD002309939F4287
:1011800004D0354B06970993344B089306AC0222E2
:101190002100019810F058FC200010F01DFC039B6A
:1011A000002B15D00C220021200011F0C1FD0023DE
:1011B000E3609F4204D0284B0697E360274BA3606F
:1011C00002980222210010F03FFC200010F004FCE5
:1011D0000C2204991B4B4A439B1800225A601A7236
:1011E0005A72039A9E72DD721A7300200BB0F0BD22
:1011F0003F2332009A43C02A0AD1CE2E08D8184A7B
:1012000033409B00D218936D10499B005B587FE7D9
:1012100001235B4280E73F232A009A43C02A0AD178
:10122000CE2D08D80E4A2B409B00D218936D07494B
:101230009B005B5878E701235B4279E73522094B35
:1012400033E7C0467004002074040020444A0108BB
:10125000E9070008E84201082D03000835030008EB
:1012600068420108A4040020F0B5514F89B001285C
:1012700005DC1C2234373A70002009B0F0BD012390
:101280000C681C4202D04D681D4202D11122343735
:10129000F1E76410621E039200220192022807D037
:1012A0008A681100194001911A4201D0531001932C
:1012B000631E032B77D86D10EBB202930C23621ED2
:1012C0005343381DC018FFF7F9F9EBB23C2B38D85F
:1012D000384BEAB29200D358013364D0EDB200210A
:1012E0002800023CFFF7CCFE334E022C03D8334BD0
:1012F000A4001B191E6A019B04AC012B33D10C22E4
:101300000021200011F014FD0023E3609E4204D070
:101310002B4B0496E3602B4BA36003222100280093
:1013200010F092FB200010F057FB0C23039A029957
:101330005343FB1800229972FF215A60D9721A7325
:101340009AE73F23EAB29A43C02A2CD1EAB2CE2AC6
:1013500029D8E8B21C4A03409B00D218936D154966
:101360009B005B58B8E7019B0C2200212000022B58
:101370000CD111F0DDFC0023E3609E4204D0104B41
:101380000496E3600F4BA3600222C7E711F0D0FC84
:101390000023E3609E4204D0094B0496E360094BAE
:1013A000A3600422BAE73B00352234331A7063E7A6
:1013B00070040020444A010889020008E84201083C
:1013C0002D03000835030008684201080C4B0D4A44
:1013D0001B6810B5134206D010241B021B0AA3423F
:1013E00002D0002010BD1B2420000321FFF748FE7F
:1013F00020000DF069FF0128F3D10330F2E7C04669
:101400000470FF1FF0FFFF0002001C281ED8114BC4
:1014100011481B68114903420AD11B021B0A012B08
:1014200004D12C31885CFF2810D070474931F9E78E
:101430006631885C153A012AF5D8094A1A40102A03
:10144000F1D01B021B0A123B012BECD901204042B8
:10145000EBE7C0460470FF1FF0FFFF00E842010801
:10146000FEFFFF000122F8B50368134202D0446872
:10147000144203D10D221B4B1A70F8BD5D10772B5F
:10148000FBD82800FEF786FF061EF6DB2800FFF7D4
:10149000BBFF154B154F1B5C012B02D030000AF02F
:1014A000CCF92800FFF7B0FF54373B5C012B07D085
:1014B00001210DF06FFE2800FFF7A6FF01233B542A
:1014C00080236210DB009A4208DB094A3000094998
:1014D0000FF06EFE0122084B5A55CEE7D343DB17BF
:1014E0001A40F3E7A4040020C40400207004002084
:1014F000FF030000EEB600003405002010B5080020
:10150000FFF7B0FF002010BD70B50D003B2816D8C6
:10151000152815D8144B1B5C002B11D0FEF73AFF91
:101520006B425D4104000AF088F9FA210F4B6A42D0
:101530001A400F4B2000D21889000FF039FE70BD01
:10154000FFF762FF0400431CF9D00A4E335C012B05
:1015500004D001210DF01EFE012333552900200087
:101560000DF076FEEBE7C0463405002001FCFFFFDE
:10157000FF030000C4040020036810B5DA0703D499
:101580000D22054B1A7010BD4168581004394A42AB
:101590005141FFF7B9FFF6E7A404002010B5080099
:1015A000FFF7EAFF002010BDF0B50C001021774BCB
:1015B00089B001931B1805005956002C5DDC0029E9
:1015C00059DB03234B43724AD31860331978002345
:1015D000C90051184B70D1184978012947D00833F8
:1015E000602BF8D1012002246A4A1369D96881432B
:1015F000D960D968A143D960D9682419A143D960B9
:10160000D9680434A143D960D9680834A143D960AA
:101610001C6A61490C4206D11C6A60490C4202D125
:10162000196881431960100001214D30017018685C
:101630008843186013004E33197013004F3319702C
:1016400013005033197013005133197013005233C3
:1016500019701300533319701300543319701300A9
:101660005533197013005732563319701170019B9E
:101670005D19FF232B7409B0F0BD002907DB03239C
:101680004B4347482100C01808F0FBF8F3E7FFF789
:10169000BBFE030000900133EDD000263C4B404FD1
:1016A00002933A780299D300CB185B780393002B0E
:1016B00067D1019B5D192E740B2ADCD8012100989B
:1016C0000DF068FD03227243029B02986033D15CE7
:1016D0009B18039A009D5A709A708823C90045543C
:1016E0009B009C420BDAB42C00DDB424E820C0003F
:1016F0006043B42110F06AFB88239B00C4183800B3
:10170000210008F0BEF80023214FFA185278012A70
:101710002DD00833602BF8D11E4C200009F014F9AD
:10172000204910F0C9FA256901382900A862200073
:1017300009F0C8F8002220001B4909F019F900231C
:1017400005931A4B04AD0493194B29000793194BC9
:101750002000069309F09EF8280010F03DF9802142
:101760002269200013688B43136009F001F80323FA
:101770003A00734360329B5C0122DB00FB185A7015
:1017800079E7013603370C2E8BD174E70000002077
:1017900070050020A40F0020111100004404000077
:1017A000D005002040420F00204E0000A9A90008EB
:1017B0002D03000835030008012270B518C9180070
:1017C000104013421BD020001040144217D00020BC
:1017D0005D10392B13D80A4B14419C4200DD1C00CC
:1017E000084E735D012B05D0012128000DF0D2FCBD
:1017F0000123735528002100FFF7D6FE042070BD99
:1018000088130000C4040020F0B518C90122180094
:1018100087B01040134218D0210011400800144234
:1018200013D05810392B1DD94D4B1A684D4B1A4205
:1018300017D04D4813021B0A83422FD007D8102B14
:101840000DD00720112B0DD0042007B0F0BD474864
:10185000834225D0464B1A40464B9A42F4D103208E
:1018600000E01520FFF7D0FD0500431CECD0424EF0
:10187000424F335C012B04D001210DF08BFC01237E
:101880007355641022003E4B103A9A420AD9FFF772
:10189000D9F8002128000DF0DBFCD5E70720E1E7AF
:1018A0000800DFE7374E73689D4201D0FFF7CAF8A2
:1018B00075602D2C02DCFFF7C5F8C5E7EBB23C2BB9
:1018C0003BD8314BAD00ED583B6D002B08D1B42017
:1018D00011F062FC2D4901900FF0A1FB019B3B65CB
:1018E0006B1CB1D0B3685A1C01D09D42ACD180238F
:1018F0005B029C42A8D2012328005B420121F360D5
:10190000B56009F0F2FE3D6D02222800610009F089
:101910002FF8002303931E4B02AC02931D4B2100B2
:1019200005931D4B2800049308F0B4FF200010F02D
:1019300053F8386D08F01CFF86E73F201A008243F9
:10194000C02A0AD1CE2B08D8144A03409B00D218D3
:10195000936D0D499B005D58B6E701256D42B3E7D5
:101960000470FF1FF0FFFF000100070003000C00E0
:10197000FBFFFF0001000C00C404002070040020E5
:101980009086010000000020444A01080020004029
:1019900015EB00082D030008350300086842010814
:1019A00070B501250A682B00A84200DD4B682A4269
:1019B00011D02B420FD0012A0DDD5810FFF724FD66
:1019C00004003B2807D8054E335C012B03D00121CE
:1019D0000DF0E0FB3555002070BDC046C40400206A
:1019E000414B10B51B68414C1B021B0A112B2BD11C
:1019F0001320FFF709FD60601620FFF705FDA060CA
:101A00000B20FFF701FDE0601520FFF7FDFC2061D2
:101A10001720FFF7F9FC60610820FFF7F5FCA061D3
:101A20000920FFF7F1FCE0610620FFF7EDFC2062E2
:101A30000520FFF7E9FC60620420FFF7E5FC0123C5
:101A4000A0622C34237010BD294A934225D107206F
:101A5000FFF7DAFC60600520FFF7D6FCA0600020ED
:101A6000FFF7D2FCE0600820FFF7CEFC20610620E3
:101A7000FFF7CAFC60610920FFF7C6FCA0611320D4
:101A8000FFF7C2FCE0611220FFF7BEFC20620420D9
:101A9000FFF7BAFC60620320CFE71620FFF7B4FC23
:101AA00060601720FFF7B0FCA0601820FFF7ACFCC7
:101AB000E0601B20FFF7A8FC20611C20FFF7A4FCBE
:101AC00060610420FFF7A0FCA0610720FFF79CFCE9
:101AD000E0610320FFF798FC20620620FFF794FCEA
:101AE00060620A20A9E7C0460470FF1FF0050020CD
:101AF00004000C00114B124A1B6870B51A40012AF1
:101B000004D0104A1B021B0A934215D10E4B0F4DF5
:101B10001B78002B01D1FFF763FF00242B1DE05839
:101B20000021FFF7ADFA2B001833E05801210434EF
:101B3000FFF7A6FA142CF1D170BDC0460470FF1F48
:101B4000EFFFFF0004000C001C060020F005002041
:101B5000114B124A1B6870B51A40012A04D0104A72
:101B60001B021B0A934215D10E4B0F4D1B78002B05
:101B700001D1FFF735FF00242B001833E058002176
:101B8000FFF77EFA2B1DE05800210434FFF778FAA6
:101B9000142CF1D170BDC0460470FF1FEFFFFF0091
:101BA00004000C001C060020F005002010B50028E1
:101BB0000BDD0A68074C131F591E8B412363042A4F
:101BC00005D0FFF7C5FF00236363002010BDFFF7BA
:101BD00091FFFAE7F0050020002070470023012262
:101BE00010B50A48990001334250802BFAD1084CB5
:101BF000084B00211A602000074A11F099F8074BA2
:101C0000074A6360074B1A6010BDC046BC11002034
:101C1000C829002000000020301C0000A070000037
:101C2000CC2900207004002003000B48DA0704D4FC
:101C3000042B03D8094800D1094870470F211A68BE
:101C4000181D0A40042AF8D00648092AF5D006488B
:101C5000032AF2D00548F0E7076201081162010883
:101C600033620108176201081E6201082A62010836
:101C7000012310B504001C40184202D0441020007B
:101C800010BD042810D90F2203681340042B07D17C
:101C9000FFF7CAFF21000A2211F022F80400EEE744
:101CA000032B01D10430F5E70D22014B1A70E6E752
:101CB000A4040020012310B504001C40184202D0E7
:101CC0004410200010BD042810D90F2203681340CF
:101CD000042B07D1FFF7A8FF21000A2211F000F81A
:101CE0000400EEE7032B01D10430F5E70D22014B90
:101CF0001A70E6E7A4040020F7B50C00042804DC01
:101D00001C22144B00201A70FEBD0868FFF7D2FF9A
:101D100001906068FFF7CEFF0600A068FFF7CAFFDA
:101D20000500E068FFF7C6FF07002069FFF7C2FF64
:101D3000AE4202D11F22074BE4E7019BC01B9B1B55
:101D40005843A91B10F042F8C31901205B00184347
:101D5000DAE7C046A404002070B50868FFF7AAFFC0
:101D60001C4910F019F90C1E01DA1A4BCC181A4B49
:101D700001269C4204DD194B9C4220DC184B1C1BA5
:101D80006421200010F022F864210500200010F0EA
:101D900003F90A0013496B005B5E002A0AD0013583
:101DA0006D00685E642150438A1A5A43801810F00F
:101DB0000DF80300012073435B00184370BD0A4B0C
:101DC0009C4204DC094BE41801267642D8E7014B1B
:101DD0001C1BF9E7A08C0000272300004F460000E1
:101DE000504600008E47010877690000B0B9FFFF38
:101DF00070B50868FFF75EFFC317C4185C40012C7C
:101E000003DC01206400204370BD66103100200017
:101E10000FF0DCFF85196D10AE420DDC731C1A004B
:101E200031005A437143121B641AA24200DB330093
:101E300001205B001843E7E7290020000FF0C6FFF0
:101E40004019C30F1B182E005D10E5E7002310B5E5
:101E50000C000B70C30705D50D494210200012F08D
:101E60007FF808E00B49002802D0042804D10A4971
:101E7000200012F0A1F810BD0428FCD90F2203683D
:101E80001340042BF7D1FFF7CFFE04490200E5E72A
:101E90003B610108386201083A6201083C620108AE
:101EA000012310B5040008001840194210D104297C
:101EB0000DD90F220B681340042B08D10800FFF73F
:101EC000B3FE010020000FF0D1FE4342584110BD87
:101ED0000020FCE7F7B50F00012804DC1C22384B7A
:101EE0001A700020FEBD4D68EB0706D4042D04D9FE
:101EF0000F222B681A40092A02D00B22304BEFE741
:101F00006C681B099BB26410A34200D85C1E0123BD
:101F10003E683340019301231E4212D070109E424E
:101F200047DD844245DB8300EB180433844243DC05
:101F30000123621C013C9C409200535123436B607F
:101F4000CFE731001F48FFF7ABFF002809D0019B06
:101F50009C42C6DB0122019B013301939B00EA50A6
:101F6000F5E731001848FFF79BFF00280AD0002C46
:101F7000B7D00122631C013C94409B0014435A518A
:101F80006C60AEE7042E0FD90F2233681340042B88
:101F90000AD13000FFF78EFE002808D10B483968BF
:101FA000FFF77EFF002804D11122054B98E7002897
:101FB000B7DC1222024B93E75A6801301A60B4E78B
:101FC000A404002045620108496201083862010842
:101FD000F0B51C2385B0012844DD4B680193012333
:101FE0001C00022806D08A681A4203D054109A4274
:101FF00000DC1C000127019B3B4200D073E0042B56
:1020000000D870E00F221B680D681A40042A38D1EE
:102010003D4226D1042D24D92B680B321340042BCA
:102020001FD10198FEF77CF8A0425CDB2800FFF787
:10203000FBFD03780500002B55D00198FFF7F4FD58
:10204000013C29000600001911F0E5FF051E4AD0E9
:102050003378002B01D0AE420DD37C000120204309
:1020600003E00E2300204E4A137005B0F0BD0F238D
:10207000F8E72823F6E73000FEF763F8013706009B
:10208000E6E7092A3FD1019B5E687610B4422ADC5C
:102090003D422DD1042D2BD92B6806321340042B41
:1020A00026D12800FFF7C0FD0390019A0294013465
:1020B000A300D058854203D1029B58003843D4E78F
:1020C00038420ED104280CD90F2203681340042B88
:1020D00007D1FFF7A9FD010003980FF0C7FD002805
:1020E000EAD0B442E1DD01204042BEE7B442FADC6E
:1020F000230001990134A2008A58AA42F6D1012096
:102100005B001843B1E7032AEDD11E09B6B25B0F9D
:10211000B6001340F61AB442E5DC3D4228D1042D46
:10212000A5D92B680C321A40032A15D1180980B2A0
:102130005B0F800013402F1DC01A019B361A013C13
:1021400038180433B442CEDC3A00191982421ED347
:1021500001348242F6D118E00F23042A00D081E72F
:102160002800FFF761FD07002800FDF7D9FFE4E72D
:102170006D10FF2D00D97CE7019B013C0433B44274
:10218000B1DC1A5D0134AA42F9D1640066E70D782A
:10219000AC461578AC45DBD101310132D6E7C046FB
:1021A000A40400201C2370B501281BDD01230A684C
:1021B0001A4216D04868184218D1042816D9016866
:1021C0000E331940013B04290CD15410012A06DDBD
:1021D000FFF72AFD0500FDF7C8FFA0420CDA122325
:1021E00000E011230020084A137070BD0E23F9E7A8
:1021F000FDF7A7FF0500013C2800012CF8D1FDF7F1
:10220000BFFF40002043F0E7A4040020F0B585B0F4
:10221000039301902F4B0291002A01D002211970E3
:1022200000272D499F548A63019B9F4201DB05B023
:10223000F0BD029ABB00D558274B264E9C6BFA2363
:102240009B00A6191C1B01231D4206D0234A6B10BC
:102250002100300011F050FE09E0214A002D02D08B
:10226000042D19D11F4A2100300011F045FE194CF0
:1022700020000FF005FD184A039B9063002B09D046
:10228000019B013BBB4205DD431C9363202222548A
:102290000022E2540137C7E72800FDF735FF0300AD
:1022A000042805D12800FFF7BFFC0F4A0300CFE741
:1022B000092803D16B680D4A5B10C9E70C4A032853
:1022C000C6D129680A0992B2490F92000B40D31A6D
:1022D000084ABDE7E0250020F00500203B61010829
:1022E0001162010833620108116401084E6201089D
:1022F000686201085D620108002310B51A00FFF74B
:1023000085FF034B986B0DF057FE002010BDC046B3
:10231000F0050020F8B501230D00060014000800A8
:102320001D40194227D1042941D90A680F210A40CA
:10233000042A3CD11C4215D1042C38D923680B4007
:10234000042B34D1FFF770FC05002000FFF76CFC74
:10235000010028000FF08AFC002830DA04237017EF
:102360001840F8BDFFF760FC29000A2210F0B8FC05
:102370000500601012E017001F401A4215D1042A10
:1023800015D913680F221340042B10D120004D10D3
:10239000FFF74AFC0A22390010F0A2FC8542DDDB7F
:1023A00008DD002E09DC0020DBE74D10E1E70F22FD
:1023B000044B1A700136022EF5D80420D1E700280C
:1023C000EFD1F7E7A4040020012310B504001C405E
:1023D000184202D04410200010BD042810D90F224A
:1023E00003681340042B07D1FFF71EFC21000A22CB
:1023F00010F076FC0400EEE7032B01D10430F5E782
:102400000D22014B1A70E6E7A404002010B50868FD
:10241000FFF7DAFF002010BD086810B5C30703D529
:10242000FFF7D2FF014B9864002010BD700400201C
:1024300070B508680D00FFF7C7FF04006868013C2D
:10244000FFF7C2FF042C0BD80138042808D8052256
:10245000012342431219934002498A6C13438B644F
:10246000002070BD7004002070B508680D00FFF7F3
:10247000ABFF04006868013CFFF7A6FF042C0BD8F3
:102480000138042808D805224243131901229A4032
:1024900002498B6C93438B64002070BD7004002054
:1024A000114B13B51B6804001B021B0A012B0BD038
:1024B00001210F200CF06EFE21680F2004394B42E1
:1024C00059410CF0C5FE13BD07230093043B019353
:1024D000036869460220042B02D1FFF7A9FFF2E747
:1024E000FFF7C2FFEFE7C0460470FF1F10B50800FA
:1024F000FFF7D6FF002010BD70B50C680123250042
:102500001D401C4217D1042C15D90F2223681340FB
:10251000092B10D166687610B54204DB0120FEF766
:1025200026FD002070BD2300AA0008339858FFF74D
:102530004BFF0135F0E72000FFF746FFEEE70868A4
:10254000F8B5C3071ED5FFF73FFF0300203B5E2B06
:102550001AD805220121534342430020104E9B3AD2
:1025600005241025F75C3D4200D04018013C49008D
:102570006D10002CF7D101339342F1D143000120BB
:10258000184302E0042801D80120F8BD0F23026897
:102590001340042BF8D1034B1A42F5D00079D4E74D
:1025A000D8430108F0FF0F00F0B5060087B00868B7
:1025B0000D00FFF709FF012303901C00022E07DD29
:1025C0006868FFF701FF0400A868FFF7FDFE03003D
:1025D0005A1D0492214A1800916C01220027019291
:1025E000461E059605264643B44605267642651ED8
:1025F000221DB444059E042E0DD8042D0BD866462A
:1026000077190126BE40019F0296039E374221D0D2
:10261000029E31430127019E013576000196AA42B0
:10262000E8D1049D0130A842DAD1002F01D00B4837
:102630008164042A0BD8012B09D108481D34816C10
:102640001D0095400532A9439442F9D181640020D0
:1026500007B0F0BD029EB143DCE7C0467004002025
:10266000F0B50C0097B0022805DC1C22D84B1A707C
:10267000002017B0F0BD0868FFF7A6FE0190606863
:10268000FFF7A2FE0500A068FFF79EFE04002800E9
:10269000FEF7BAFE06003B28EAD8CE4D2B5C012B94
:1026A00004D001210CF076FD0123AB550021300050
:1026B0000CF0CEFD2100C8480FF088FB0138050062
:1026C0006A1E9541C54C451BA368FA2114936368A3
:1026D00089000133180068431F000FF0EDFA002253
:1026E000149B1593A36814931599149B994200D3D6
:1026F00046E11599149BFB1A5B18D218149B15938D
:102700009042EFD80121019B300019400CF0A0FD50
:10271000A368FA21129363688900013318006843A3
:102720001F000FF0C9FA0022129B1393A3681293A3
:102730001399129B994200D326E11399129BFB1A1D
:102740005B18D218129B13939042EFD8019B300074
:102750009907C90F0CF07CFDA368FA2110936368F8
:1027600089000133180068431F000FF0A5FA00220A
:10277000109B1193A36810931199109B994200D359
:1027800006E11199109BFB1A5B18D218109B11934C
:102790009042EFD8019B30005907C90F0CF058FD4B
:1027A000A368FA210E936368890001331800684317
:1027B0001F000FF081FA00220E9B0F93A3680E9367
:1027C0000F990E9B994200D3E6E00F990E9BFB1ADE
:1027D0005B18D2180E9B0F939042EFD8019B3000EC
:1027E0001907C90F0CF034FDA368FA210C93636834
:1027F00089000133180068431F000FF05DFA0022C2
:102800000C9B0D93A3680C930D990C9B994200D3DC
:10281000C6E00D990C9BFB1A5B18D2180C9B0D930C
:102820009042EFD8019B3000D906C90F0CF010FD83
:10283000A368FA210A93636889000133180068438A
:102840001F000FF039FA00220A9B0B93A3680A932A
:102850000B990A9B994200D3A6E00B990A9BFB1A9D
:102860005B18D2180A9B0B939042EFD8019B300063
:102870009906C90F0CF0ECFCA368FA210893636871
:1028800089000133180068431F000FF015FA002279
:10289000089B0993A36808930999089B994200D360
:1028A00086E00999089BFB1A5B18D218089B0993CC
:1028B0009042EFD8019B30005906C90F0CF0C8FCBC
:1028C000A368FA21069363688900013318006843FE
:1028D0001F000FF0F1F90022069B0793A3680693EF
:1028E0000799069B994267D20799069BFB1A5B18CA
:1028F000D218069B07939042F0D8019B300019062E
:10290000C90F0CF0A5FCA368FA210493676889003D
:102910000137380068430FF0CFF90022049B05937C
:10292000A36804930599049B994249D20599049B95
:10293000FB1A5B18D218049B05939042F0D8300024
:1029400001210CF085FC2800FA21A368890002937C
:102950006668013670430FF0AFF90022029B0393C3
:10296000A36802930399029B99422DD20399029B7B
:10297000F31A5B18D218029B03939042F0D877E6C3
:10298000159B14995B1AB8E6139B12995B1AD8E64B
:10299000119B10995B1AF8E60F9B0E995B1A18E7CA
:1029A0000D9B0C995B1A38E70B9B0A995B1A58E749
:1029B000099B08995B1A78E7079B06995B1A97E7CA
:1029C000059B04995B1AB5E7039B02995B1AD1E753
:1029D000A4040020C404002040420F0010E000E0E6
:1029E00070B50400FEF7D4FA012805D1043C634217
:1029F0005C416500280070BD00250428FAD1200044
:102A0000FFF712F90400084821000FF02FF9A8423F
:102A100007D0210005480FF029F9A842EAD1032583
:102A2000E8E70225E6E7C0467B6801087A6201080C
:102A3000F8B50C68E30704D40D221E4B1A70012070
:102A4000F8BD00256410012803DD4868FFF7C8FFC2
:102A50000500172CF3D8184B18481A68184B61005A
:102A60005B18024222D1120204269E5F120A012A3A
:102A700004D1E31E012BE2D90C2CE0D0002EDEDBCA
:102A80002000FEF7C1FC0F4F3B5CAB4206D0290093
:102A90000CF080FB2000FEF7B7FC3D540A2130000B
:102AA00008F002FF430001201843C9E734269E5F67
:102AB000E4E7C046A40400200470FF1FF0FFFF00FD
:102AC00068430108C404002013B50020104C114BCA
:102AD000E0631B68104A13420ED11B0209221B0A35
:102AE000012B00D00E3201205200024301A90192B5
:102AF000FFF79EFF401003E0084A1340102B04D05C
:102B0000430060630120184316BD1122EBE7C04665
:102B1000F00500200470FF1FF0FFFF00FEFFFF0024
:102B2000F8B5060001200B680D00034203D10D2209
:102B3000104B1A70F8BD5810FEF766FC04003B28D5
:102B400001D90020F6E70027012E03DD6868FFF7B2
:102B500047FF0700084D2B5DBB4204D03900200021
:102B60000CF018FB2F5520000CF0AEFB0128E8D12B
:102B70000330DFE7A4040020C4040020086810B577
:102B8000C30706D4042804D90F2203681340042B7A
:102B900004D00E2200200D4B1A7010BDFFF744F830
:102BA0000378233B5A425341C0180378302B05D198
:102BB000202243789343582B00D102301022002169
:102BC00010F08EF8430001201843E6E7A40400202B
:102BD000086870B5012405002540204206D104286C
:102BE00004D90F2203681340042B04D00E220020C6
:102BF000054B1A7070BDFFF717F80222290010F07C
:102C00006FF840002043F5E7A4040020030010B54E
:102C1000C2070BD40A48042B07D90F211A680A40AF
:102C2000042A02D11800FEF7FFFF10BD431005482B
:102C30000F210400044A11F05FF92000F5E7C046B7
:102C400062630108300600203B6101081C2370B557
:102C5000012833DD0868012304001C4018422CD1F0
:102C600004282AD90F2602683240042A25D14D684B
:102C70001D4206D1042D20D92A680D333240042A82
:102C80001CD1FEF7D1FF06002800FFF7BFFF0100AF
:102C9000300006F0A8FD00281DD006F093FC037854
:102CA0007B2B0FD101300022110006F06FFD0028B0
:102CB00011D006F08EFC0134F5E70E230020084AFF
:102CC000137070BD5B2B06D1013006F043FD002868
:102CD00001D00134F9E7012064002043F1E7C04648
:102CE000A404002010B5002809DD0868C30706D435
:102CF000042804D90F2304681C40042C04D00E229D
:102D0000054B1A70002010BDFEF78EFFFDF7A4FCE6
:102D10000130F7D02000F6E7A4040020F8B5334BCB
:102D2000334A1B681A40012A04D0324A1B021B0A8C
:102D3000934214D1304C256B002D10D123002C333D
:102D40001B78002B01D1FEF74BFE2C4B226D9B6CA8
:102D50001900114304D1E36B002B00D0E163F8BDEF
:102D600021005431097800290DD1E06B002800D0F2
:102D7000E1632365002A04D0002B02D1FEF7E8FEB0
:102D8000EDE7FEF7B7FE230054331A780423002A38
:102D900000D0531E9B00E31800215868FEF770F91D
:102DA0002700052254373E78236D72435219134190
:102DB000012199432300AA001833D05801350CF0A3
:102DC00047FA052DECD1B600A61970680121FEF76F
:102DD00057F93E780121B300E41860680CF038FA26
:102DE0002900701C0FF0D8F83970B8E70470FF1F85
:102DF000EFFFFF0004000C00F0050020700400202D
:102E0000F0B5A1B005920A00574F0490386801321E
:102E1000036801911B099BB202929A4200DA89E091
:102E200006F055FBFFF77AFF07F0C8FE0024039079
:102E30004E4AA300D0580134FDF772FB802CF7D125
:102E40004B4B1868FDF76CFB386C002801D0FDF780
:102E500067FB0026474D7B6C9E4257DB4649474D3A
:102E60000A001368141F1B0926689BB2981C002EC9
:102E70005DD08B1A5E1EB3415B420B402360830022
:102E8000C91880001218AA42EBD3FDF7DDFA3A4CBC
:102E900026000F2233681D09ADB213420BD06F1C00
:102EA000A64204D031002000BA0010F0F9FC002343
:102EB000BF00E41908C40235AD0076192F4DAE42AB
:102EC000E7D32D1BAD10013D274E2B01236034604D
:102ED00007F074FE039AABB2821A023B284907A896
:102EE00011F03EF807A807F0EBFE06F0F0FAFFF746
:102EF00015FF3068029A03681B099BB29A4219DBDE
:102F00000A2300203436337021B0F0BD2B78002B1B
:102F100002D10136F0359EE72C69013C002CF8DB2C
:102F20002B00A20018339858FDF7FAFAF5E71B01B9
:102F30001360A6E7019A0C4D941CA2001B1B81187C
:102F40001B010B6029600021031F1960019B083AD7
:102F50001901049B1943030002C39A189A42D3D95A
:102F6000059902C3FAE7C04670040020BC11002096
:102F700000000020BC130020CC290020F8450020D0
:102F80007F62010870B5002204000D00411C092079
:102F9000FFF736FF002808D0012362001343010029
:102FA000436000230831A34200DB70BD9A00AE5895
:102FB00001338E50F7E7F7B50F000190012804DCCC
:102FC0001C221F4B1A700020FEBD0868FEF772FE1F
:102FD00005007868FEF76EFE019B06000124022BB7
:102FE00007D0B868FEF766FE041E02DC2922144BE7
:102FF000E8E7B5421CDC701B21000EF0E7FE461C22
:1030000000220920711CFFF7FBFE0028DBD0012203
:10301000730013434360944095400300B600361894
:1030200011002943996004332D19B342F8D1CBE73D
:103030002100A81B0EF0CAFE6442461CE0E7C04611
:10304000A4040020F7B54C680191E30706D4042CD2
:1030500004D90F2223681A40092A04D00B22304BCE
:103060001A700020FEBD1B0965689EB2731E6D10AC
:10307000AB4244D803200B2D08DD972361305B0061
:103080009D4203DC032128000EF0A0FE254FBB6B00
:103090009C4234D3FB6B9C4231D28319190001222C
:1030A000092000933C64FFF7ABFE00233C6C060054
:1030B0003B64984223D02268009B120992B20430EC
:1030C0009A4200DD1A009200211D0FF08CFE164A74
:1030D00016490020131F186013681B099BB20233A6
:1030E0009B00D2188A42F4D3271F3E60FDF7ACF94B
:1030F00000233B6023680E4A13402360340023689A
:103100001B099BB2013B9D42ABD2019B1A68AB1CD1
:103110009B001A51012301356D002B436360A0E72A
:10312000A404002070040020CC290020F8450020D1
:10313000F0FF0F0070B5002805DC1C22164B0024A0
:103140001A70200070BD01220D68154202D10D22B7
:10315000114BF4E701281DD04B681342F7D05B10E8
:10316000FF2B02D913220C4BE9E718020200C0180A
:103170001A43000402436D10EB43DB171D40E91CAA
:1031800003208910FFF73CFE041EDAD02900FCF76B
:10319000A4FFD6E70022EEE7A4040020F7B50F0055
:1031A000002805DC1C22324B1A7000242000FEBDD2
:1031B0000C68012625003540344211D06510FF2DE2
:1031C00002D913222A4BEFE7002231000320FFF738
:1031D00017FE041EEAD03100FCF77FFF2571E5E7FA
:1031E000042CEED90F2223681340042B19D12000A0
:1031F000FCF796FFC11C2A00060089100320FFF788
:10320000FFFD051E0BD03100FCF767FF2000FEF725
:103210000BFD2B1D0100320018000FF0E4FD2C0007
:10322000C4E7092B20D1032063682A005B100193B7
:103230000333D9170140C9188910FFF7E1FD041EB7
:10324000B3D03F680199FCF748FF0837221D019B66
:103250009D42ABDAAB00FB58334203D05B10FF2B2F
:10326000AFD853550135F2E7032BAAD19EE7C046EC
:10327000A404002010B5094C00222064022109207A
:10328000FFF7BEFD236C002803D10A2334342370DA
:1032900010BD032283604260FAE7C046700400203C
:1032A00070B50400C30708D54410FF2C07D91322BA
:1032B0000A4B00251A70280070BD631E9C41002235
:1032C00001210320FFF79CFD051E02D10A22034BBA
:1032D000EFE70121FCF701FF2C71ECE7A4040020CB
:1032E0000323043010B5C117194009180022042027
:1032F0008910FFF785FD10BDF7B50E00009001287D
:1033000005DC1C225D4B1A7000242000FEBD4B68BA
:1033100001221C001440134202D10D22574BF2E748
:103320000099022902D0B1681142F6D00122376813
:10333000174200D09EE0042F00D89BE05D1093421E
:1033400000DC15000F213B681940092927D17B6853
:1033500000995B101A00022901D0B2685210009245
:103360009A4200DD0093009B01225F1B0137FB4363
:10337000DB171F400920791CFFF742FD041EC3D054
:1033800001237F003B433268436003000833009908
:10339000A942BADB0135A900515802C3F7E7042955
:1033A0003CD13800FEF740FC0190FCF7DEFE009AAD
:1033B0000300022A01D0B3685B100093834200DD52
:1033C0000090009BAB4223DA0020FFF789FF040046
:1033D0009BE7FCF7B6FE070001343800A542F8D1A0
:1033E000009BA34216DAC51B2800FFF779FF041ED5
:1033F00000D18AE7FEF718FC00903068FEF714FC55
:103400002A00019BFF1AC11900980FF0ECFC7CE721
:10341000019FE2E7FCF795FE0134E1E7032929D19A
:103420001A0992B25B0F0B4092000099D21A130056
:10343000022901D0B3685B10934200DD1300AB4258
:1034400005DA002203201100FFF7DAFCBFE75E1B5C
:10345000B110002203200131FFF7D2FC041E00D17D
:1034600053E7013631000335FCF737FE3200201DEB
:103470007919CAE72122014B45E7C046A404002080
:10348000F0B593B005000191012806DC1C22984B91
:103490001A700025280013B0F0BD019B01261B689F
:1034A0001C003440334200D0ACE0042B00D8E7E0ED
:1034B0000F271B6802943B40092B45D1029B019AC0
:1034C0009B00D3581A0032400392334205D1042B9B
:1034D00003D918683840092804D02222844BD7E742
:1034E0000293EBE75B685B10E418029B01339D429B
:1034F000F6D10122611CFFF783FC051EC9D06400D0
:10350000344344600400039A083401999300C95875
:1035100008684B68000980B25B10984200D8431ECF
:103520000020083183420ADCD943C9170B400299B5
:103530009B00E418531C9142ACDD1A00E5E78600BD
:103540008F590130A751EDE7032B5ED1029B019A01
:103550009B00D0583042C0D10428BED90268110067
:10356000394003293FD113099BB2520F9B000A40F7
:103570009B1A1C19029B01339D4232D10320E31C8C
:10358000D9170140C91800228910FFF739FC051E20
:1035900000D17EE72100FCF7A0FD00262F1D019A37
:1035A000B300D45801231C4224D1042C22D90F2269
:1035B00023681A40032A1DD1180980B25B0F8000CE
:1035C0001340C01A00230434834217DBC343029A1A
:1035D000DB1718403F18731CB24200DC5AE71E008C
:1035E000DDE70293B2E7042900D076E7FCF798FD07
:1035F0002418BFE72000FCF793FDE3E7E25CFA54F0
:103600000133E1E700231C00029301260F27029BF0
:10361000019A9B00D058304236D1042834D9026830
:1036200011003940042936D1FCF77AFD2418029B99
:1036300001339D4226D12000FFF752FE051E00D126
:1036400027E70023041D0393039B019A9B00D65890
:1036500001231E422AD1042E28D90F2233681A4092
:10366000042A3AD13000FCF75BFD07003000FEF77A
:10367000DBFA010020003A000FF0B5FBE41923E06B
:103680000294C2E70293C2E705A9FEF7DFFB05A893
:103690000EF0F6FACAE7032900D01EE713099BB221
:1036A000520F9B000A409B1A1C19C0E7300005A965
:1036B000FEF7CCFB05A80EF0E3FA05A90600020010
:1036C00020000FF090FBA419039B029A0399013389
:1036D0008A42B8D100232370DCE6032AF4D11F0903
:1036E000BFB25B0FBF001340FF1A311DC2E7C046D7
:1036F000A4040020F0B50E0097B0002806DC1C22C0
:10370000604B1A700025280017B0F0BD0C6801232B
:1037100022001A4000921C4206D1042C04D90F2228
:1037200021681140092902D00B22564BE9E7616854
:103730004D100495012904DC0098FFF7D1FD050028
:10374000E1E75149019101280BD07068184208D176
:10375000042806D903681340042B02D1FEF764FA4B
:10376000019001980EF08CFA05000F27049B02903F
:10377000013B5D430593049B9B00E31803930123E6
:10378000A06818426CD104286AD902681100394037
:10379000042903D1FCF7C4FC451908E0032966D1CC
:1037A00013099BB2520F9B000A409B1A5D19039BA1
:1037B0000434A342E3D12800FFF792FD051EA1D0F7
:1037C00033680793029B002B03D07068FEF72CFA36
:1037D00001902800FEF728FA0600009B9A00079B3C
:1037E00008339F5801233B40069301231F4241D1D8
:1037F000042F3FD93800FEF717FA039003980EF014
:103800003FFA069B0400002B0ED1042F0CD90F2287
:103810003B681A40032A07D11C09A4B25B0F391D6B
:10382000A40013400391E41A3000220003990FF022
:10383000DAFA029B3619002B0AD0059B009A9342B4
:1038400006DD3000029A01990FF0CDFA029BF618BE
:10385000009B01330093009A049B9342BDD152E731
:1038600009A9FEF7F3FA09A80EF00AFA94E7FEF7A1
:10387000DBF9F9E7380009A9FEF7E8FA09AB039389
:10388000BCE7C046A40400206263010870B50500CF
:1038900008000C00FFF724FD002809D00023021DBA
:1038A000A34206DBE343DB171C400023121913700D
:1038B00070BDE95CD1540133F2E7F0B58DB00C0076
:1038C0000190012805DC1C22654B1A7000200DB008
:1038D000F0BD01230868184206D1042804D90F213D
:1038E00002680A40042A02D00E225D4BEDE76668AA
:1038F00035001D401E42F7D1042EF5D933680B4028
:10390000042BF1D1FEF790F907003000FEF78CF997
:1039100002900EF0B5F9019B03900495022B04D0A0
:10392000A368043B5A425A410492039B002B1FD1C7
:103930003800FCF71AFC0190019B01220920591C58
:10394000FFF75EFA474E30640028BFD00122019B8A
:103950005B0013434360039B002B2ED13800FCF720
:10396000F0FB019B0400AB4216D13E4B186CAEE756
:103970003800029910F04FFBC01B4342434138000E
:103980000193019B029901330193039BC01810F02E
:1039900042FB0028F5D1CFE73800E11BFFF776FFA7
:1039A000002800D192E7336CAA009B189860200091
:1039B000FCF7C7FB27000135D3E7019B012B02D1A0
:1039C00023688360D1E73800029910F024FB041EBD
:1039D000CBD038000EF054F901263B180593019B1B
:1039E0009E42C2DC049BE11B002B23D0A74221D2C4
:1039F0003A783B002D2A02D17B1C9C421AD99C426A
:103A000013D10D00132900DD13252A00390007A862
:103A100010F0EDFA002107AB18000A2259550FF0FB
:103A20005FF90123400018430AE01A780133303A65
:103A3000092AE4D93800FFF729FF002800D145E71B
:103A4000084B01361B6CB200D050039B0299E7185B
:103A5000380010F0E0FA041EC1D1059CBFE7C04653
:103A6000A404002070040020F0B50E0085B00028EA
:103A700004DC1C22314B1A70002419E00D6801246B
:103A80002F002740254206D1042D20D90F222B6874
:103A90001340042B0FD12800FEF70CF902AC0100F3
:103AA0002000FCF7A2FB011B2000FFF7EFFE040043
:103AB000200005B0F0BD092B09D16B685B100193A4
:103AC000019B9C4206DD1D4B1B78002B1DD02A223A
:103AD0001A4BD0E70134A300E858FEF7EBF80123B6
:103AE0007F2810DD8022DB18120190420BDB802240
:103AF00001335202904206DB8822023B520290427E
:103B000000DB00239B00FF18DAE73800FFF7E8FB33
:103B1000041EB1D0FEF788F8376805000126019B26
:103B20009E42C5DC0136B300F858FEF7C3F8010029
:103B30002800FCF75AFB0500F1E7C046A40400206A
:103B4000F0B50E008BB0012806DC1C22AA4B1A70BF
:103B5000002420000BB0F0BD0C682000FCF7D4FA64
:103B600005007068FEF760F8A44907000EF07EF8C3
:103B70000126002800D0023E3800A1490EF076F858
:103B8000002800D1022638009E490EF06FF8002868
:103B900000D1042638009C490EF068F8002800D1B6
:103BA0000926380099490EF061F8002800D1B6E1E5
:103BB000731C02D13022904BC9E7681E0828C8D870
:103BC0000EF070F80900240056014200C7FFC7FF3D
:103BD000C7FFC7FFB000B01E0728BAD80EF000FA22
:103BE000043009B9B9B9B911042C00D095E1013CF0
:103BF000AFE78748042C00D186480121FFF746FE35
:103C000002E02000FFF736FB0400A2E7701E082840
:103C10009FD80EF0E5F9059E150A9E9E9E9EF60021
:103C2000641000D194E7042493E77B49621002A852
:103C300010F096F902A80EF023F8010002A8DDE7C3
:103C40002000FFF72DFBDFE7701E082800D980E772
:103C50000EF028F80900120047007FFF7FFF7FFF6A
:103C60007FFF7FFF19002000FDF7DEFF68490DF0A0
:103C7000FDFF0028D7D16BE72000FEF71BF80124D9
:103C80004000044365E72000FDF7CEFFFCF76DFA26
:103C9000624D411C0600002209202C64FFF7B0F899
:103CA000041E02D10A22544B51E701227300134330
:103CB000286C6360FDF7B8FF00270500BE4200D105
:103CC00047E72800FCF75CFA012122004000BB0016
:103CD00008430832D0502800FCF733FA01370500BA
:103CE000ECE72000FDF7A0FF0DF0CAFF4B4EC11C12
:103CF00005000022032089103464FFF781F8041EB8
:103D0000D0D0366C2900FCF7E8F93000FDF78CFFC5
:103D10000023221D9D4200DC1BE7C15CD15401330E
:103D2000F8E703266568701E6D10032800D910E7B8
:103D30000DF0AEFF020E763A012D06D1A4682000E8
:103D4000FCF7E2F9012800D103E72D222A4BFEE619
:103D5000012D03D1A4682C4200D0FAE62C22264B78
:103D6000F5E60136B300E058FDF7A4FF01237F28F4
:103D700010DD8022DB18120190420BDB8022013320
:103D80005202904206DB8822023B5202904200DB44
:103D900000239B00FF18B542E3DA174B1F4E1A7839
:103DA000002A04D02A22D2E601260027F3E73800B1
:103DB0003464FFF795FA336C041E019300D1C7E613
:103DC000FDF732FF0127BD4200DAC2E6019A013752
:103DD000BB00D1580123194202D12722064BB6E677
:103DE000882349105B03994203D33123343633705F
:103DF000AEE6FCF7FAF9E6E7A40400209F620108AA
:103E0000A7620108AE620108B5620108BA62010842
:103E1000386201083A6201083B6101087004002021
:103E20000320EB1CD9170140444EC9180022891009
:103E30003464FEF7E5FF041E00D133E7376C290038
:103E4000FCF74BF93900002301270831201D9D4262
:103E500000DC7EE69A008A583A42BED05210FF2A11
:103E600002D913233436C2E7C2540133EFE72E00E0
:103E70002368701E1D09ADB25B00AD009B0FED1AEB
:103E8000082800D965E60DF00DFF0900120064FE58
:103E9000190064FE64FE64FE64FE2B00012D00D058
:103EA00053E723790424002B00D052E650E6012D7D
:103EB00000D053E7247964002C434AE61F4E2800C3
:103EC0003464FFF70DFA0423041E316C00D1E9E6D7
:103ED0001A1F954200DC3CE6CA5CE2540133F7E766
:103EE000164E691C002209203464FEF789FF316CEC
:103EF000041E00D1D6E601206B0003432600636058
:103F00000023083604319D4200DC22E6CA5C9F0093
:103F100052000243F2510133F5E7012419E6681E0D
:103F2000082800D915E60DF0BDFE8BFE8BFEA2FF22
:103F3000DCFE14FE14FE14FE14FEFCFE70040020D1
:103F400010B588B0002806DC1C220024194B1A701A
:103F5000200008B010BD0C682000FCF7D5F801382F
:103F6000082823D80EF03CF8050E19F4222222224C
:103F700019001148042C00D110480121FFF786FCDC
:103F80000400E5E70E49621068460FF0E9FF684655
:103F90000DF076FE01006846F0E72000FDF744FED4
:103FA00004000DF06DFE01002000E7E70020FFF7A0
:103FB00097F9E5E7A4040020386201083A62010895
:103FC0003B61010810B50C4C86B020000DF058FE86
:103FD00001002000032906D00849122201A80EF092
:103FE00002FF112101A8FFF751FC002802D10A228B
:103FF000034B1A7006B010BD45060020C5620108CB
:10400000A404002070B50C009AB0022845DD0122FE
:104010000868104246D1042844D90F2103680B4098
:10402000042B3FD16568154206D1042D3AD92A6880
:104030000A330A40042A31D1A368DB0734D5FDF7DF
:10404000F3FD06002800FEF7E1FD00236A460100AB
:104050003000A468137105F0C6FB64100500002C45
:1040600008DC01A80DF00CFE010001A8FFF70EFC12
:104070001AB070BD05F0F6FA0228F2D16422681C6D
:1040800001A905F083FB012CEBD005F063FB642252
:1040900001A905F07BFB013CF5E71C23034A002046
:1040A0001370E5E70E23F9E70D23F7E7A4040020DA
:1040B00010B5204CA544041E02D1FFF711F90BE006
:1040C00005F0D0FA0138062830D80DF0E1FD0909D5
:1040D000192004312C0004208023DB009D4410BDF6
:1040E000200005F076FA844204D3011B2000FFF77C
:1040F000CDFBF1E70378013B1F2BF6D80138F2E73F
:10410000200005F0D9FA430001201843E4E780229B
:1041100069462000D20005F0E6FA68460DF0B0FDD1
:1041200001006846E3E704210348E0E70020C4E714
:104130000020D1E700FCFFFFD7620108F8B50500B9
:104140000C001C23012833DD0122086810422ED107
:1041500004282CD90F2103680B40042B27D1676852
:10416000174206D1042F22D93A680A330A40042A9A
:104170001ED1FDF759FD06003800FEF747FD01008E
:10418000022D19D0A568EB0716D56D10300005F08B
:104190002AFB040005F066FA012816D1002D02DD85
:1041A0000134012D0BD12000FFF782FF03E00E2325
:1041B00000200E4A1370F8BD01256D42E6E720008D
:1041C00005F0C8FA013D0400EBE70228EBD1002D11
:1041D000E9DD0134012DE6D000222000110005F0B8
:1041E000D5FA05F0B7FA013D0400F3E7A404002076
:1041F00070B51C230C00022842DD01220868104221
:104200003DD104283BD90F2103680B40042B36D144
:104210006568154206D1042D31D92A680A330A404F
:10422000042A2DD1A368DB072ED5FDF7FDFC06007F
:104230002800FEF7EBFC01003000A46805F0D3FA7B
:10424000050000206410844225DD280005F00AFAEC
:104250000300681C012B1CD00020022B1BD1013550
:1042600002000100280005F091FA012C13D005F09E
:1042700071FA0022110005F089FA013CF5E70E23DE
:104280000020064A137070BD0D23F9E705F062FAAD
:10429000013C012CFAD1FFF70BFFF4E7A404002046
:1042A00070B50C68E30718D52000FDF703FD040086
:1042B000203C5E2C13D8002202210320FEF7A0FD33
:1042C000051E02D00521FBF708FF052254430B49C8
:1042D000281D61180EF087FD02E0042C02D801258C
:1042E000280070BD0F2223681340042BF7D1200053
:1042F000FBF7E6FE0028F2D02479D9E7B3450108A0
:10430000F0B5364C87B0237C002B01D1FCF73CFC88
:104310000A270F26A26932499368136913680B4074
:10432000D9B21C0C180A9B029B0F7B4334401B190B
:10433000C0B2039303097B4330401818C3B2029301
:104340000B097B4331405B1801935368254A1340A6
:104350001C04640F00940124D9B2180C1A0A1B0D16
:104360007B4330401B18D2B2DBB20D097D4305936D
:10437000130923405B42324031403B409B186D188B
:104380000022082109200493FEF73AFD002803D1FA
:10439000154B1F7007B0F0BDFA22D2009446059B62
:1043A0006D0063445B0023438360049B25435B00F3
:1043B0002343C360009B46605B0023434361039B30
:1043C00005615B0023438361029B5B002343C36160
:1043D000019B5B001C430462DCE7C046F004002044
:1043E0007F7F7F003FFFFF00A4040020F7B5070098
:1043F0000E000DF0E1FA1D4B1D4D1A78012A2FD049
:1044000001221A7000232B660BF0D6F9002824D164
:10441000F8231B06FB18DC176405640DE418E4128E
:10442000F61B2700F1174905490D8919CB12019395
:10443000019B104EE3189F420BD273690E4A134042
:10444000FA0013430D4A134373610BF0B5F90028CA
:1044500009D0022273699343736100235C352B708A
:104460000DF0A0FAF7BD0137E2E7C0464C06002088
:10447000F00500200020024007FEFFFF02000100BF
:1044800010B5002804D104480449FFF7AFFF10BD60
:1044900002480349F9E7C0460080010800C001084E
:1044A00000000208431E9841054B8003C0180368B2
:1044B00000201A0E532A01D11B02180A7047C04669
:1044C0000080010813B5431E98410A4B8403E41889
:1044D000A6230902090ADB050B430093002301937D
:1044E0000DF06AFA009A019B20000BF003FF0DF01B
:1044F00059FA13BD00800108154B01005B6F10B520
:10450000002B0BD1134C144B00290AD19A680800D8
:10451000120E522A01D10833180010BD0F4C0D4B5A
:10452000F2E700208C42F8D90B681B0E522BF4D115
:104530004B689A1C92008818DB0700D5043084422F
:1045400003D903681B0E522BE7D00020E5E7C046D5
:10455000F005002000C001080080010800000208EA
:10456000F8B50020FFF7C8FFFF26DA27050036045C
:104570003F04002801D12800F8BD0468FFF7BCFF04
:104580003440BC42F5D10500F3E7FF2270B51A4C68
:104590000021D20020000EF0CBFBFF25FFF7E0FF4B
:1045A000002600280CD1154B1A78002A03D05A781F
:1045B000D200A2589A600130F0330A28F4D170BDBD
:1045C00003681A142A400C2A0AD11A122A40FF2A18
:1045D00003D0D200A1180B71A050FFF78DFFE0E7C8
:1045E000132AFAD11B122B40FF2BF6D0DB00E21866
:1045F0001671E650F1E7C046E81D0020BC1300200C
:104600008022F0B5564BA1B004935B6900215200A3
:10461000544805930EF08CFB802200215200524832
:104620000EF086FB514B5B6F1A00039353425341CC
:1046300018000293FFF724FF029B9D034C4BED18DB
:10464000FFF78EFF061E2BD10398FFF72BFF411CAF
:104650000298FFF737FF029A444B64245A679D671C
:10466000FFF793FF039B80205A425341414A9B032B
:104670009B18EB1A5C43049AC00152690190E01741
:104680008004800C059900198013521A00903A4951
:1046900007A80FF065FC07A806F012FB21B0F0BDDB
:1046A00004F015FFFF22346823142712134017402B
:1046B0001A000C3A072A25D82A4BDC5D002C1BD1A6
:1046C0003000FF2103681A120A40974206D11B14DA
:1046D0000B400C2B14D0132B00D10024FFF70CFF40
:1046E0000028EED1002C04D028002100FCF730FC7B
:1046F00005001C4B0122DA553000FFF7FDFEA1E753
:104700000400EBE7153B082BF6D8174BDB5D002BBD
:10471000F2D1FF231B041C40184B3000E418634205
:104720005C4164423440FF2103681A140A40152A90
:104730000FD01D2A00D10024FFF7DEFE0028F2D1A1
:10474000002C04D028002100FCF702FC0500064BD9
:10475000D0E7FF221B1213409F42EDD10400EBE78C
:10476000F0040020A00E0020A00D0020F005002085
:104770000880010800800108DC6201080000EBFFEE
:1047800070B5104D2C686E68B4420CDD8022280094
:104790000D49D200121B6118083004F0F3FA001919
:1047A0008005840D2C60A6420ADD28000649321BD4
:1047B0006118083004F0E6FA00198005800D2860C1
:1047C00070BDC04670060020C4060020044A05499A
:1047D0005368C85401339B059B0D53607047C04616
:1047E00070060020C4060020064A53681268DB43A6
:1047F0009B189B0501229B0D834200DC00221000C8
:104800007047C04670060020F8B505000C00160081
:104810001F1E0ED10320FFF7E7FF002808D0FA2063
:10482000FFF7D4FFE8B2FFF7D1FFE0B2FFF7CEFF0A
:10483000F8BD501DFFF7D8FF0028F9D0FB20FFF787
:10484000C5FFE8B2FFF7C2FFE0B2FFF7BFFFF0B26B
:10485000FFF7BCFF3012C0B2FFF7B8FF0024B4422C
:10486000E6DA385DFFF7B2FF0134F8E7F0B587B05C
:10487000039203220333284FDC171440E4187B6FA4
:10488000A4105A1E9341BD6F244AA61D9B03B60077
:104890009B18AA1901900291934218D2FFF7B0FE1B
:1048A0007B6FBD6F5A1E934180225B42D201134041
:1048B0001A4AAE199B18B34209D2002319201A00D4
:1048C0001900FFF7A1FF0025280007B0F0BD019BEC
:1048D000039A1B041343029A2E0012021343A422CC
:1048E000D2051343049305940DF066F8049A059BD2
:1048F00028000BF0FFFC08360DF054F8002C07D010
:10490000210030000C9AFCF7DDFA012301349C43AE
:10491000A4003619BE67D7E7F005002000C00108E3
:1049200007B500210B000A001D200091FFF79EFF34
:1049300007BDF7B505000022204B5B6C0193204BAF
:104940000199914211DC0024F0231A006243009285
:1049500000991B4A575C5618002F0FD001340A2CBF
:10496000F3D1184806F0ACF927E05978A94202D1F2
:104970001978002921D10132F033E1E7F022390022
:1049800030000EF0D5F902230D4A0099757053548A
:104990000D4BEA00D358B570B3600423F360019B5C
:1049A00037617761A34202DC044B01345C6400236D
:1049B00029001A001020FFF727FFF7BD7004002020
:1049C000BC1300201E630108E81D0020F7B50C0091
:1049D0000190FEF75BFF0026194B1A4F18603B79D8
:1049E000062B01D0032B19D17F223868438913404D
:1049F000052B13D1C3891340292B0FD10C22835EC1
:104A00005B000C33C018FDF70FF903780500002B8D
:104A100011D00DF035F90023A0420AD00136083735
:104A2000FF2EDCD1F7BD019AE95CD25C9142F5D151
:104A300001339C42F7DCF0B2FFF77BFFEEE7C046A4
:104A400000000020E81D002070B506000024064D7F
:104A50002B79B34202D1E0B2FFF76BFF0134083586
:104A6000FF2CF5D170BDC046E81D0020F7B506F05B
:104A7000A5F8594CA369834201D90023A361574A81
:104A8000C31A93420BD90023554AA0611179073903
:104A9000022900D872E001330832FF2BF6D1F7BDAE
:104AA000226A002A00D083E02562002B62D0671DB5
:104AB000FB7F0126002B18D10920FFF7C5FF494BCA
:104AC000FE77DE77266A002E07D0A71DFB7F002B1E
:104AD00003D1B54213D22E002562E769002F17D10A
:104AE000002E38D1002FDAD01BE00720FFF7ACFFF3
:104AF0003C4BDE77E6E70820FFF7A6FF6AE0AB1B3A
:104B0000312BEAD90720FFF79FFF0123FB77E4E76A
:104B1000354BDB7F002BE3D1BD4211D2E561002E86
:104B200018D1009B002BBAD1631DDB7F002B02D173
:104B30000820FFF789FF0023E3610534E377AEE740
:104B4000ED1B312DCCD90820FFF77EFF0123264A2B
:104B5000D377C5E72F00019B002BC3D1A31DDB7FBB
:104B6000002B02D10720FFF76FFF0023A21D236255
:104B7000D377B7E7009B002B1FD1A3E71B4B5D69E1
:104B8000002D00D1013503211C20FCF779FA1C20EF
:104B90000AF09AFB013843425841830000200193F8
:104BA000FCF714FC019AE3690090002A00D077E733
:104BB000009A002A86D0002B84D1236AE561002B5D
:104BC00080D0A71DFB7F0126002B94D10920FFF781
:104BD0003BFFFE77044B8CE7700600200F27000098
:104BE000E81D00207606002075060020F004002055
:104BF000104B70B50500002418005A78AA4204D062
:104C00000134F0330A2CF8D170BDF0221300634355
:104C10000021C0180EF08CF8074A536C013BA342E8
:104C200000D15464002329001A001120FFF7ECFD85
:104C3000EAE7C046BC13002070040020F8B50F4D11
:104C400000262F000E4C636CB3420ADC962238001B
:104C5000002112010EF06CF800233434236123701C
:104C6000F8BD2B78002B05D0002311201A0069789D
:104C7000FFF7CAFD0136F035E4E7C046BC1300205B
:104C800070040020F0B5002485B00190FFF7D6FF36
:104C900003A80394FDF704FC274E3378002B17D0AC
:104CA0002000FBF777FB002801DB06F0C6FD2000A3
:104CB000FCF7AAFB0500431C08D0204F3B5C002BEF
:104CC00004D000210AF066FA00237B5500233370DC
:104CD00001340136162CE0D10024200000210134DB
:104CE000FCF762FC1D2CF8D10024FBF7ABFE134D42
:104CF0002B78032B0CD05A1E012A0FD8012B07D179
:104D00002000FCF781FB431C02D000210AF0A0FA2E
:104D1000002120000AF03EFA00232B7001340135F7
:104D20003C2CE5D1019B002B04D0FCF757FF044835
:104D300005F0C6FF05B0F0BD34050020C404002016
:104D40003363010870B50024FFF778FF0120FFF7F7
:104D500099FF084B084D5A69084B9A622B79043B1E
:104D6000012B02D8E0B2FFF7E4FD01340835FF2C37
:104D7000F4D170BDF0040020E81D00207006002072
:104D800010B50400064A53681268DB439B189B0564
:104D90009B0DA34200DB10BDFFF7F2FCF2E7C0461B
:104DA0007006002010B505F075FF002808D005201A
:104DB000FFF7E6FF002318201A001900FFF724FD73
:104DC000002010BDF0B51500764C0122A5442C0042
:104DD000019002911440154211D005AB1A706A106F
:104DE0005A70120E1A710522691299706D14029987
:104DF000DD70FFF709FDCF239B009D44F0BD042D1E
:104E000029D90F2029680840042831D1022305AE92
:104E100028003370FCF708FF05000CF031FFC822B2
:104E200001009200904200DD11006B1E651CA14242
:104E30000DD1904206D95C4804AB03225B49C018EF
:104E40000DF0D1FF33002A0002990198D1E72C0020
:104E50005D5D3555EAE7042D01D0002DCBD103224D
:104E600005AB043D1A706A42554102225D70EBE7C2
:104E700009287AD1042205AB1A706A6851105212BF
:104E800059709A700391202901DD20220392002796
:104E9000039A06ACDA70039BBB4202DC05ABE21A54
:104EA000D2E72B00BA0008339E583000FBF72CF9EC
:104EB0000138082855D80CF0EBFE3405471254543D
:104EC00054543C00012323707310637072121B0E44
:104ED0007614A270E670237105340137DBE70223F4
:104EE00030002370FCF7A0FE06000CF0C9FE0300A2
:104EF000A01C142B09D800226370934201D1C4185E
:104F0000EBE7B15C81540132F7E71423112263709F
:104F100031000DF068FF2E23E3742375637516349A
:104F2000DBE70323043E237073425E416670023464
:104F3000D3E70423237073685A1062705B12A37066
:104F40000023E3700434C8E705230321326823708B
:104F500013099BB2520F9B000A409B1A63701B12ED
:104F6000EDE7002323700134B7E7032800D042E7C0
:104F7000052205AB1A700A0992B2490F014092004E
:104F8000521A11125A709970642A00DD64220421A9
:104F9000DA70081F904201DB043255E7685C585410
:104FA0000131F6E7C4FCFFFF220300004162010863
:104FB000C368F0B587685B00FF180300BBB0183307
:104FC00001930269019B92009C18436901999B001F
:104FD000CB180293D04B00901B78002B0CD10021F2
:104FE0007B5E7F2192101D1202610B40CB4A9B0019
:104FF0009B5802379F461400C74B00261878C84DAF
:10500000FF283CD11E70C74B1D6CB54207DD012344
:10501000009A137005F0D2FD009B2D185D60009B77
:10502000009A9B68FB1A5B10D360019BE41AA410E2
:10503000029B1461019A9B1A009A9B10536121E014
:1050400014000700D8E714000700D5E71400D3E7E1
:105050001400D1E71400CFE73400CDE7039CCBE781
:105060001400C9E73400C7E73400C5E73400C3E7DC
:1050700014000700C0E7039FBEE7049FBCE7FE28BB
:1050800002D11E703BB0F0BD009B9A689B78BA1AA3
:10509000521012021A43009B597808AB1870101274
:1050A0005A7098701014120ED8701A7113200522BD
:1050B000FFF7AAFBF021009B9B4A1E706B6C013B23
:1050C00059438A5C002A00D16B64934B1E70A6E79B
:1050D000009B1120597800231A00FFF795FB00234D
:1050E000F021009A8E481370436C8F4A013B59435C
:1050F0008A5C002A00D092E7436490E7E8E7864B99
:10510000AD001B78641B002B00D075E70022BB5E4E
:10511000019A0099A21A92100A617F217F4A1D12FA
:105120000B409B009B58023764E7019B221DD11A5C
:105130007B4BD82903DD1A2234331A705CE73433F1
:105140001B782560002B00D055E700203B5E0098BF
:10515000891001617F2071491D1203409B001400DA
:105160005B58023746E7019B221DD11AD82903DD7F
:105170001A22694B1A703FE70026BB5FEDB21B0293
:105180001D43654BB81C1B782560002B00D057E7EA
:1051900002203B5E0098891001617F205F491D124B
:1051A00003409B0014005B58043723E7019B221D3A
:1051B000D11AD82903DD1A22574B1A701CE7002593
:1051C0007B5FB81C5B00FB182360534B1B78002BE4
:1051D00000D038E702203B5E0098891001617F20F3
:1051E0004E491D1203409B0014005B58043701E731
:1051F000019B221DD11AD82903DD1A22464B1A70B1
:10520000FAE64A4BAD00EB582360434B1B78002B6A
:1052100000D01BE700203B5E0098891001617F20D1
:105220003E491D1203409B0014005B580237E1E623
:10523000043C3E4B2268AD00EA50374B1B78002BF4
:1052400000D0D9E60022BB5E019A0099A21A921002
:105250000A617F21314A1D120B409B009B58023787
:10526000C8E6324EAD00A859FCF702FD2A4B049067
:1052700003931B78002B00D0BEE6043C2068FCF7AB
:10528000F7FC049BC018012340000343AB51039B70
:105290001B78002B00D0AFE60022BB5E019A00997C
:1052A000A21A92100A617F211C4A1D120B409B001A
:1052B0009B5802379EE6019B221DD11A184BD82914
:1052C00003DD1A2234331A7096E6019D029E0120F6
:1052D000B54202D230000C38006834331B782060AD
:1052E000002B00D0B4E600203B5E009889100161DD
:1052F0007F200A491D1203409B0014005B580237AF
:1053000078E6019B221DD11A054BD82910DD1A22FF
:1053100034331A7070E6C046A404002044480108E3
:1053200070040020F0040020BC130020BC110020F9
:105330000198029EB04210D230000C380068DB4E5B
:105340004010AD192D1A0298AD00343328581B783F
:105350002060002B08D014004EE618213433197059
:1053600000232360140047E600203B5E009889106C
:1053700001617F20CE491D1203409B0014005B5841
:10538000023737E6019A0299CA4B8A421ED20C397B
:105390000968C6484910043C2D1834336D1A226838
:1053A00002991B78AD006A50002B00D024E6002241
:1053B000BB5E019A0099A21A92100A617F21BC4A31
:1053C0001D120B409B009B58023713E61822343302
:1053D0001A7011E6019B029A93422ED21600B34B2B
:1053E0000C3EED183368043C5B10EB1A9B00985898
:1053F000FCF73EFC03902068FCF73AFC3368029A05
:105400005B10ED1A039BAD001E1801237600334399
:10541000AB50A94B1B78002B00D0EDE50022BB5E02
:10542000019A0099A21A92100A617F21A04A1D12C6
:105430000B409B009B580237DCE518229E4B1A70EC
:10544000DAE5019B221DD11A9A4BD82903DD1A22D5
:1054500034331A70D0E50298AD00343328581B78E5
:105460002060002B00D0F5E500203B5E00988910FD
:1054700001617F208E491D1203409B0014005B5880
:105480000237B7E5043C2368029AAD00AB508A4B63
:105490001B78002B00D0AFE50022BB5E019A00997B
:1054A000A21A92100A617F21814A1D120B409B00B3
:1054B0009B5802379EE5029BAD00043C5D192068B5
:1054C0002E68FCF7D5FB012376103618760033439F
:1054D0002B60794B1B78002B00D08DE50022BB5E42
:1054E000019A0099A21A92100A617F21704A1D1236
:1054F0000B409B009B5802377CE5019BAD00641B71
:10550000A34213D86C4B1B78002B00D074E500220B
:10551000BB5E019A0099A21A92100A617F21644A27
:105520001D120B409B009B58023763E5634A644998
:1055300008A80EF015FD08A805F0C2FB05F0F8FB61
:10554000FCE7002D02D10023FD5E02376B00FF183F
:10555000002D00DA63E5584B1B78002B00D04BE59B
:105560000022BB5E019A0099A21A92100A617F2163
:105570004F4A1D120B409B009B5802373AE5002D05
:1055800002D10023FD5E02377F226D007F19BB1E12
:105590001B881340132B14D10C3C474B1B78002B5A
:1055A00000D029E50022BB5E019A0099A21A921050
:1055B0000A617F213E4A1D120B409B009B58023717
:1055C00018E51A2BE9D1043CE7E7002D02D10023AE
:1055D000FD5E0237043C2368042B04D16B00FF18E6
:1055E000002D00DA1BE5344B1B78002B00D003E5BF
:1055F0000022BB5E019A0099A21A92100A617F21D3
:105600002B4A1D120B409B009B580237F2E4002DE1
:1056100002D10023FD5E0237043C2368042B04D032
:105620006B00FF18002D00DAF9E4234B1B78002BE8
:1056300000D0E1E40022BB5E019A0099A21A921008
:105640000A617F211A4A1D120B409B009B580237AA
:10565000D0E4002D02D10023FD5E0237261F306802
:10566000C3070AD540100138002809DB0123400098
:105670006D0003437F193360D1E4FCF7F9FAF2E7D8
:105680000D4B34001B78002B00D0B5E40022BB5E2C
:10569000019A0099B21A92100A617F21044A1D12E0
:1056A0000B409B009B580237A4E4C046FDFFFF3F20
:1056B0004448010870040020A4040020426301084B
:1056C000526301080022BB5E02371A1203926A4637
:1056D000127BDB4DD2009446AA181179D94A0329CE
:1056E00003D002233432137086E4260001990C366D
:1056F000701AD82803DD1A23343213707CE4FF219A
:105700005B0049000B40FE39FF390B432360009BCF
:1057100034329B681278FB1A0B41009F1B02BF7842
:105720003B438B400B436360019F029BDB1B9B1041
:105730008B401943A160009B0399997063460099BF
:105740005B598B60002A04D008331F003400029696
:1057500052E47F211F0008229B5E009A80101D12D8
:1057600010610B40B84A9B0034009B580A370296E0
:1057700040E4231F1D68029A019B934234D10A2002
:10578000EB0713D4042D18D90F222B68F7301340E0
:10579000FF30042B0AD12800FCF746FA0CF070FA0F
:1057A000C8239B00984200D9180006306430FFF7E8
:1057B0001BF800280DD1023F31E40720042DF5D05D
:1057C00068426841A14B4042184080239B00C018AA
:1057D000ECE7009B2A0059781220FFF7F3FA002328
:1057E000009A1370FFF71BFC029B994C0C3B1B6843
:1057F00000995B10E41A029BA4001C1920C4083B0A
:105800001B685A108A708E49D2B2D2005B0057587A
:105810009B0A009A5B009760FF18029B019A043B69
:105820001B685B109B00D31802938A4B1B78002BDC
:1058300001D0FFF7E1FB0022BB5E019A0099A21A9A
:1058400092100A617F21804A1D120B409B009B58D9
:105850000237FFF7CFFB231F1868FCF709FAAD00EA
:105860000600641B1E2835DC7A4B1D78002813DCEB
:10587000002D01D0FFF7C0FB0022BB5E019A00990A
:10588000A21A92100A617F216F4A1D120B409B00E1
:105890009B580237FFF7AEFB05F090F9033E361830
:1058A00005F08CF96C4B801B9842F9D8002D01D083
:1058B000FFF7A2FB0022BB5E019A0099A21A921088
:1058C0000A617F21604A1D120B409B009B580237E2
:1058D000FFF790FB0123009A073E137005F06EF965
:1058E000009B36185E60FFF79AFB231F1868FCF7D1
:1058F000BFF9AD000600641B002815DC554B1B7872
:10590000002B01D0FFF778FB0022BB5E019A0099C3
:10591000A21A92100A617F214B4A1D120B409B0074
:105920009B580237FFF766FB4C4B984204DD1D2263
:10593000484B1A70FFF760FB0123009A137005F0C3
:105940003DF9FA239B007343009A073B1B185360F1
:10595000FFF765FBAB00E41A002328001A002100C2
:10596000FCF754FC3E4D3F4EA96B3000FDF78EFF17
:105970003D4BA96B18603000FFF728F8A86B0AF0C0
:105980001BFB344B1B78002B01D0FFF735FB0022AB
:10599000BB5E019A0099A21A92100A617F212A4ADD
:1059A0001D120B409B009B580237FFF723FB294B2E
:1059B000AD001B78641B002B01D0FFF71DFB0022FC
:1059C000BB5E019A0099A21A92100A617F211E4AB9
:1059D0001D120B409B009B580237FFF70BFB002664
:1059E000224D009B0136AB421AD1164B5E64F03556
:1059F0000A2EF6D1174B1B78002B01D0FFF7FCFACB
:105A00000022BB5E019A0099A21A92100A617F21BE
:105A10000D4A1D120B409B009B580237FFF7EAFA14
:105A20002B78002BE3D0002369781A001120FEF7B1
:105A3000EBFEF022002128000DF07AF9D7E7C046EE
:105A4000E81D0020700400204448010807FEFFFF05
:105A5000FDFFFF3FA40400207F96980080EE3600F3
:105A6000F0050020E025002000000020BC130020ED
:105A7000231F1868002855D1083B1868C30733D581
:105A80004010220001234100083A0B431360002814
:105A900000DC92E0012342001A43211F0A60220029
:105AA000083A1668043A1E41361A106818423CD06B
:105AB000F6189E401E43029BAD00EE50C54B1B786E
:105AC000002B01D0FFF798FA0022BB5E019A0099E3
:105AD000A21A92100A617F21BF4A1D120B409B003F
:105AE0009B580237FFF786FA042816D90F2203685D
:105AF0001A40092A01D14068C2E7042A04D1FCF700
:105B000093F8FAF732FBBCE7032A06D1180980B2F2
:105B10005B0F80001340C01AB3E71922AD4B1A7017
:105B2000FFF76AFA40100138B1E7042840D90F2185
:105B300002680A40092A06D10236B6003358AD0081
:105B4000029AAB50BAE7042A2AD1029BAD005B1936
:105B50000493FCF769F805000136012E10DC2800DB
:105B6000FAF7EFFA431B18000393FDF7B9FB061E83
:105B70000ED0FCF759F82900039A0DF034F907E02C
:105B80002A78013E002A06D112211600914B197085
:105B9000049B1E6092E72800FAF7D3FA0500DCE7C1
:105BA000032A05D180190279AD0052001343C7E7DB
:105BB0001922884B1A70FFF71FFA04377EE7019A03
:105BC000AB00E3189B1AD82B18DC0123002D1ADC3C
:105BD000804B1B78002B01D0FFF70EFA0022BB5E32
:105BE000019A0099A21A92100A617F217A4A1D1225
:105BF0000B409B009B580237FFF7FCF91A22754BAC
:105C00001A70FFF7F9F908C4013DDFE7019A231D77
:105C1000724E9B1AD82B04DD1A2334363370FFF7EB
:105C2000EBF9019B029A934232D2231F1868FCF7CA
:105C30001FF8002828DD029B0C3B1B685B10834289
:105C400022DBC01A664BC018029B8000C258AB0012
:105C5000E31A1A6001235B1B9B00E4185D4B1B7861
:105C6000002B01D0FFF7C8F90022BB5E019A009912
:105C7000A21A92100A617F21574A1D120B409B0005
:105C80009B580237FFF7B6F9202334363370E1E72B
:105C900018233436FAE7534AAB001268E31A1A6045
:105CA00001235B1B9B00E4184A4B1B78002B01D09F
:105CB000FFF7A2F90022BB5E019A0099A21A921086
:105CC0000A617F21444A1D120B409B009B580237FA
:105CD000FFF790F9002D02D10023FD5E0237231F4C
:105CE0001A68042A17D16D007F193A4B1B78002BD4
:105CF00001D0FFF781F90022BB5E019A0099A21A38
:105D000092100A617F21344A1D120B409B009B5860
:105D10000237FFF76FF91C00E7E7002D02D10023DF
:105D2000FD5E0237231F1A68042A19D000226D0075
:105D30001A607F19274B1B78002B01D0FFF75CF905
:105D40000022BB5E019A0099A21A92100A617F217B
:105D5000214A1D120B409B009B580237FFF74AF95E
:105D60001C00E7E7AA00A21A002D25DD100001267D
:105D700013685B100168314220D10D2315490B7067
:105D80000023136001235B1B9B00E418114B1B785D
:105D9000002B01D0FFF730F90022BB5E019A009979
:105DA000A21A92100A617F210B4A1D120B409B0020
:105DB0009B580237FFF71EF91C23DFE749108B427F
:105DC00000DD0B0004308442D4D101215B000B4381
:105DD000D7E7C046A404002044480108700400200E
:105DE000FCFFFF3F00000020AA00A21A002D25DDC5
:105DF0001000012613685B100168314220D10D2389
:105E0000D4490B700023136001235B1B9B00E41833
:105E1000D04B1B78002B01D0FFF7EEF80022BB5EC1
:105E2000019A0099A21A92100A617F21CA4A1D1292
:105E30000B409B009B580237FFF7DCF81C23DFE781
:105E400049108B4200DA0B0004308442D4D1012186
:105E50005B000B43D7E72300083B1968231F1A6830
:105E60000123AE00194223D01A4221D019411A4110
:105E70000023914200DA0433A61B336001235B1B2D
:105E80009B00E418B34B1B78002B01D0FFF7B4F84C
:105E90000022BB5E019A0099A21A92100A617F212A
:105EA000AD4A1D120B409B009B580237FFF7A2F82A
:105EB00002204042FCF72EFAA61B3060DEE72300EA
:105EC0000122083B1968231F1B68AE00114226D02F
:105ED000134224D05A1094464810CA0F6146DB176B
:105EE00081425A41A61B9200326001235B1B9B003A
:105EF000E418984B1B78002B01D0FFF77DF80022A7
:105F0000BB5E019A0099A21A92100A617F21924AFF
:105F10001D120B409B009B580237FFF76BF80120C6
:105F20001A004042FCF7F6F9A61B3060DDE72300BB
:105F3000083B1868231F1968AB00E31A0393042376
:105F40009C46814219D000239C46042815D901267D
:105F5000304212D10F2203681340042B0DD131427D
:105F60000BD1042909D90B681340042B05D1FAF78A
:105F7000F1F9431E984183009C466246039B1A60D8
:105F800001235B1B9B00E418724B1B78002B01D094
:105F9000FFF732F80022BB5E019A0099A21A921014
:105FA0000A617F216C4A1D120B409B009B580237EF
:105FB000FFF720F82300083B1868231F1968AB007F
:105FC000E31A039300239C46814219D004339C4674
:105FD000984215D90126304212D10F22036813408E
:105FE00063450DD131420BD1614509D90B6813408E
:105FF000634505D1FAF7AEF94342584183009C4608
:106000006246039B1A6001235B1B9B00E418514B03
:106010001B78002B01D0FEF7EFFF0022BB5E019A38
:106020000099A21A92100A617F214B4A1D120B405F
:106030009B009B580237FEF7DDFF23000122083B3F
:106040001968231F1B68AE00114226D0134224D0CA
:106050004A109446CA1761465810DB0F81425A41D4
:10606000A61B9200326001235B1B9B00E418394B96
:106070001B78002B01D0FEF7BFFF0022BB5E019A08
:106080000099A21A92100A617F21334A1D120B4017
:106090009B009B580237FEF7ADFF1A000120FCF76A
:1060A00039F9A61B3060DEE72300083B1968231F7F
:1060B0001A680123AE00194223D01A4221D0194197
:1060C0001A410023914200DD0433A61B33600123F3
:1060D0005B1B9B00E4181F4B1B78002B01D0FEF7C5
:1060E0008BFF0022BB5E019A0099A21A92100A61EE
:1060F0007F21194A1D120B409B009B580237FEF767
:1061000079FF0220FCF706F9A61B3060DFE7231FAA
:106110001B68043B5A1E9341AA009B00A21A1360FD
:1061200001235B1B9B00E4180A4B1B78002B01D05A
:10613000FEF762FF0022BB5E019A0099A21A92103C
:106140000A617F21044A1D120B409B009B580237B5
:10615000FEF750FFA4040020444801082300083B38
:106160001868FBF785FD231F06001868FBF780FD04
:106170000123361876001E435B1B9B00AA00A21A5F
:10618000E418F34B16601B78002B01D0FEF734FFA8
:106190000022BB5E019A0099A21A92100A617F2127
:1061A000EC4A1D120B409B009B580237FEF722FF62
:1061B0002300083B1868FBF75BFD231F06001868E7
:1061C000FBF756FD0123361A76001E435B1B9B002E
:1061D000AA00A21AE418DE4B16601B78002B01D02F
:1061E000FEF70AFF0022BB5E019A0099A21A9210E4
:1061F0000A617F21D74A1D120B409B009B58023732
:10620000FEF7F8FE2300083B1868FBF731FD231F5B
:1062100006001868FBF72CFD01227043AB0040001C
:10622000E31A10431860CA4B521B1B789200A41843
:10623000002B01D0FEF7E0FE0022BB5E019A009920
:10624000A21A92100A617F21C24A1D120B409B00C4
:106250009B580237FEF7CEFE231F1868FBF708FD98
:10626000BD4B061E039320D11F2234331A70AB009E
:10627000E31A1E6001235B1B9B00E418039B34336D
:106280001B78002B01D0FEF7B7FE0022BB5E019AFF
:106290000099A21A92100A617F21AE4A1D120B408A
:1062A0009B009B580237FEF7A5FE2300083B1868A9
:1062B000FBF7DEFC31000BF089FD012640000643B0
:1062C000D5E7AE00A61B3068FBF7D2FC04907068DF
:1062D000FBF7CEFC00281DD11F229D4B1A70012315
:1062E0005B1B9B00E4189A4B30601B78002B01D09D
:1062F000FEF782FE0022BB5E019A0099A21A92105C
:106300000A617F21934A1D120B409B009B58023764
:10631000FEF770FEC317C2185A401100049803928A
:106320000BF03AFE002901DA039BC918012049004D
:106330000843D4E7231F1868FBF79AFCC21780189C
:1063400050400122AB004000E31A10431860804B1C
:10635000521B1B789200A418002B01D0FEF74CFEB4
:106360000022BB5E019A0099A21A92100A617F2155
:10637000784A1D120B409B009B580237FEF73AFEED
:10638000AB00E31A04950393012D07D11868FBF7BE
:106390006FFC061E0EDA01256D420BE0022D35D191
:1063A000039B1868FBF764FC039B05005868FBF728
:1063B0005FFC0600B54202DC33002E001D000135F3
:1063C000AD1B0CF01DFB29000BF0E6FD0123891924
:1063D000039A490019431160049A9B1A9B00E41820
:1063E0005B4B1B78002B01D0FEF706FE0022BB5E44
:1063F000019A0099A21A92100A617F21554A1D1232
:106400000B409B009B580237FEF7F4FD64250126E4
:10641000D5E7AE00A61B31002800FCF7AFFB012337
:106420005B1B9B00E4184A4B30601B78002B01D0AB
:10643000FEF7E2FD0022BB5E019A0099A21A9210BB
:106440000A617F21434A1D120B409B009B58023773
:10645000FEF7D0FD2300083B1868FBF709FC231F5B
:1064600006001868FBF704FC01223040AB00400036
:10647000E31A10431860364B521B1B789200A41885
:10648000002B01D0FEF7B8FD0022BB5E019A0099F7
:10649000A21A92100A617F212E4A1D120B409B0006
:1064A0009B580237FEF7A6FD2300083B1868FBF750
:1064B000DFFB231F06001868FBF7DAFB0123064306
:1064C00076001E435B1B9B00AA00A21AE418204B17
:1064D00016601B78002B01D0FEF78EFD0022BB5EFC
:1064E000019A0099A21A92100A617F21194A1D127D
:1064F0000B409B009B580237FEF77CFD2300083BB6
:106500001868FBF7B5FB231F06001868FBF7B0FB04
:106510000123464076001E435B1B9B00AA00A21A83
:10652000E4180B4B16601B78002B01D0FEF764FDBE
:106530000022BB5E019A0099A21A92100A617F2183
:10654000044A1D120B409B009B580237FEF752FD78
:10655000A40400204448010870040020231F186888
:10656000FBF786FBC0430122AB004000E31A104357
:106570001860D54B521B1B789200A418002B01D039
:10658000FEF73AFD0022BB5E019A0099A21A921012
:106590000A617F21CD4A1D120B409B009B58023798
:1065A000FEF728FD2300083B1868FBF761FB231F5B
:1065B00006001868FBF75CFB8640012376001E434B
:1065C0005B1B9B00AA00A21AE418BF4B16601B7845
:1065D000002B01D0FEF710FD0022BB5E019A00994E
:1065E000A21A92100A617F21B84A1D120B409B002B
:1065F0009B580237FEF7FEFC2300083B1868FBF7A8
:1066000037FB231F06001868FBF732FB0641012306
:1066100076001E435B1B9B00AA00A21AE418AA4B3B
:1066200016601B78002B01D0FEF7E6FC0022BB5E53
:10663000019A0099A21A92100A617F21A34A1D12A1
:106640000B409B009B580237FEF7D4FCAB00E31ACB
:106650009C4600231900012D4FD163461A68130090
:106660002B402A4248D1042A47D90F2610683040CF
:10667000092842D1110056681A000831039176109A
:10668000964203DC01225B00134319E0039891005A
:1066900041580120014203D0014112185B18EFE775
:1066A00027230AE052109B1801318D42EADD66462D
:1066B0008A00B2580242F5D10D23834A1370002399
:1066C0006246136001235B1B9B00E4187E4B1B7822
:1066D000002B01D0FEF790FC0022BB5E019A0099CE
:1066E000A21A92100A617F21784A1D120B409B006A
:1066F0009B580237FEF77EFC0B000120D5E72300F4
:106700000C3B1868FBF7B4FA2300083B0600186836
:10671000FBF7AEFAF1170200C31730000DF092FC40
:10672000231F039018680491FBF7A2FA0499020052
:1067300003980BF069FC0123400018435B1B9B008E
:10674000AE00A61BE418604B30601B78002B01D014
:10675000FEF752FC0022BB5E019A0099A21A921029
:106760000A617F21594A1D120B409B009B5802373A
:10677000FEF740FC01210026AB00E31A0A00039358
:10678000B5420DDD0E001B681E40194203D05E109D
:10679000F343DB171E402A00012D01D0039B5A68EA
:1067A0000920711CFCF72CFB002803D00123760084
:1067B00033434360039B186001235B1B9B00E41879
:1067C000414B1B78002B01D0FEF716FC0022BB5E6C
:1067D000019A0099A21A92100A617F213B4A1D1268
:1067E0000B409B009B580237FEF704FCAB00E31AFA
:1067F0005E680693320001231A400792002203923A
:106800001E4216D1042E14D933680F321A40092AB9
:1068100009D172681B0952109BB20392934208D8A7
:10682000013B039305E0042A32D13000F9F778FCEC
:106830000390069B1B680593DB0734D5059B5B1013
:106840000493059B012B03DD049B039A934264DDB3
:10685000122200261C4B1A70069B1E6001235B1B34
:106860009B00E418184B1B78002B01D0FEF7C4FBEB
:106870000022BB5E019A0099A21A92100A617F2140
:10688000124A1D120B409B009B580237FEF7B2FBC9
:10689000032ACED1190989B25B0F89001340CB1AA4
:1068A000BFE70B22D5E70A480599FBF7F9FA00285C
:1068B00010D0039B002BCBD00CF0A2F803990BF067
:1068C0006BFB4B1C049328E0A404002044480108FF
:1068D00063630108C5480599FBF7E2FA00282BD14C
:1068E000059B042B10D90F221B681340042B0BD1DE
:1068F0000598FBF7DFF90490002807D1BC480599FB
:10690000FBF7CEFA0028A3D11122A2E7049B002BAB
:106910009EDD039B049A93429ADB079B002BC0D118
:10692000042EBED90F2233681340092B06D1049BD5
:1069300001339B009E598FE7039BC3E7042B24D1AF
:106940003000FBF771F9049E0390012E12DC0398CE
:10695000F9F7F7FB039BC31A18000493FCF7C0FC7C
:10696000061E00D178E7FBF75FF9049A03990CF053
:106970003AFA71E7039B013E1B78002B00D167E7D1
:106980000398F9F7DEFB0390DFE70B22032B00D01F
:106990005FE7049BF618F37801265B001E435BE774
:1069A000AD00641B666801223100A36811400493A6
:1069B000164201D000F0EFFE042E01D800F0EBFEED
:1069C0000F2033681840059009282CD172681B09E4
:1069D00052109BB203920691934201D8013B03935C
:1069E000256884482900FBF75BFA002844D0059B02
:1069F000092B35D1039B98422DDD7F4B1B78002B53
:106A000001D0FEF7F9FA0022BB5E019A0099A21AA2
:106A100092100A617F21794A1D120B409B009B58FE
:106A20000237FEF7E7FA0599032901D000F0B3FE1B
:106A30000499114201D100F0B1FE4A100692FF2ADA
:106A400001D900F0ABFE1A09059992B25B0F9200D2
:106A50000B40D31AC3E7049A01308300F250C9E710
:106A600003225242331D921B0398D1188142C4DC89
:106A7000069919700133F7E7EB0707D56810012D68
:106A800020DC12235C4A1370FEF7B6FA290057483F
:106A9000FBF706FA002822D1042D0FD90F222B680C
:106AA0001340042B0AD12800FBF704F9002807D172
:106AB00029004F48FBF7F4F90028E2D11123E1E760
:106AC0000028DEDD039B8342DBDB0F2233681340AB
:106AD000092B06D1049B0130800083518DE7039878
:106AE000F3E7032B89D1069B3618F37085E701265F
:106AF000AB00E31A18680393304207D1042805D984
:106B00000F210268114009291CD14668039B1E60B1
:106B100001235B1B9B00E418374B1B78002B01D033
:106B2000FEF76AFA0022BB5E019A0099A21A92103F
:106B30000A617F21314A1D120B409B009B5802378E
:106B4000FEF758FA032908D113099BB2520F9B0094
:106B50000A409B1A5B001E43D8E70429D6D1FBF7F5
:106B600063F8F9F702FB40000643CFE7231F1868DC
:106B7000FBF75AF82300083B06001868F9F7C4FA37
:106B80000138082810D80BF083F805292F2B0F0F98
:106B90000F0F2D001A4930000BF068F8434258419E
:106BA000AB008000E31A186001235B1B9B00E41814
:106BB000114B1B78002B01D0FEF71EFA0022BB5EA2
:106BC000019A0099A21A92100A617F210B4A1D12A4
:106BD0000B409B009B580237FEF70CFA0949DAE795
:106BE0000949D8E70949D6E70949D4E749620108C4
:106BF0003862010845620108A404002044480108E5
:106C00009F620108A7620108AE620108B56201082F
:106C1000BA620108019B261DF31AE64D0393D82B97
:106C200004DD1A2334352B70FEF7E6F9EB6C3435AE
:106C3000049303F0C3FFFA220023049992000BF09F
:106C4000F1F9DD4B400018400123034323602B780A
:106C5000002B01D0FEF700FA0022BB5E039A0099D8
:106C600092100A617F21D54A1D120B409B0034000F
:106C70009B580237FEF7BEF9019A231D03939E1A13
:106C8000D82E04DD1A22CE4B1A70FEF7B5F903F0A8
:106C900095FFC94B40001840012303432360C84BB4
:106CA0001B78002B01D0FEF7D9F97F210022BB5EB3
:106CB000009AB6101D1216610B40C04A9B009B58EB
:106CC000039C0237FEF796F9019B221DD11AD829A1
:106CD00004DD1A22BA4B1A70FEF78EF9B948BA4B86
:106CE000856A5B69581B9D4202D9B8481B18581B1E
:106CF0000123400003432360B14B1B78002B01D0DC
:106D0000FEF7AEF900203B5E0098891001617F20FC
:106D1000AA491D1203409B0014005B580237FEF77E
:106D200069F9A94BAD005A69A64B641B9A62A44B42
:106D30001B78002B01D0FEF75FF90022BB5E019AA1
:106D40000099A21A92100A617F219C4A1D120B40E1
:106D50009B009B580237FEF74DF903F09BFFAE00F6
:106D6000A61B002816D1964B1B78002B01D0FEF7EE
:106D700079F90022BB5E019A0099B21A92100A6159
:106D80007F218E4A1D120B409B0034009B58023716
:106D9000FEF730F9012328001A003100FBF736FA1C
:106DA0008B4B9D6B28006430FDF71EFD002801D140
:106DB000FEF701FD009A874B51782A001420FDF759
:106DC00023FD0123009A0635137003F0F7FE824B72
:106DD00034001B6B5D43009B2D185D60FEF71FF9AF
:106DE00003F058FFAE00A61B002816D1744B1B7889
:106DF000002B01D0FEF738F90022BB5E019A009902
:106E0000B21A92100A617F216C4A1D120B409B003E
:106E100034009B580237FEF7EDF8280001230022CA
:106E20003100FBF7F3F96A4B9D6B28006430FDF7E6
:106E3000DBFC002801D1FEF7BEFC022308AA65484E
:106E400013700AF01DFFC72800D9C7200021634C2A
:106E500008AB4A1C814201D1FE21AFE71100A25CC0
:106E60005A54F6E7AB00E31A0393FAF79DF81F2292
:106E700001005B48534E0DF0BAF859480AF000FF84
:106E800004238008013000010343F362039A554B49
:106E9000136001235B1B9B00E418494B1B78002BFC
:106EA00001D0FEF7A9F80022BB5E019A0099A21A50
:106EB00092100A617F21414A1D120B409B009B5892
:106EC0000237FEF797F8A900611A012D1EDC1C227B
:106ED00000203B4B1A7001235B1B9B00E418384BCE
:106EE00008601B78002B01D0FEF786F80022BB5EFD
:106EF000019A0099A21A92100A617F212F4A1D124D
:106F00000B409B009B580237FEF774F8231F18684C
:106F1000029A019B9342DED22300083B1A68531069
:106F2000012AD8DD029A0C3A126852109342D2DC40
:106F3000043B9B1A029A9B009858CCE70B22AB00AB
:106F4000E31A1A6001235B1B9B00E4181C4B1B789F
:106F5000002B01D0FEF750F80022BB5E019A009989
:106F6000A21A92100A617F21144A1D120B409B0045
:106F70009B580237FEF73EF83B22AB00E31A1A603B
:106F800001235B1B9B00E4180D4B1B78002B01D0E9
:106F9000FEF732F80022BB5E019A0099A21A921005
:106FA0000A617F21054A1D120B409B009B58023746
:106FB000FEF720F870040020FEFFFF7F4448010820
:106FC000A404002070060020F0040020378941004E
:106FD000F0050020E025002000000020DF25002033
:106FE000A00600209C060020AE00A61B3100280051
:106FF000FBF71EFD01235B1B9B00E418EB4B30608D
:107000001B78002B01D0FDF7F7FF0022BB5E019A31
:107010000099A21A92100A617F21E54A1D120B40C5
:107020009B009B580237FDF7E5FFAD00641B200075
:10703000FAF718FADD4B1B78002B01D0FDF7DCFFC7
:107040000022BB5E019A0099A21A92100A617F2168
:10705000D74A1D120B409B009B580237FDF7CAFF11
:10706000AE00A61B31002800FBF75AFD01235B1B75
:107070009B00E418CD4B30601B78002B01D0FDF74E
:10708000BBFF0022BB5E019A0099A21A92100A610E
:107090007F21C74A1D120B409B009B580237FDF70A
:1070A000A9FFAD00641B2000FAF766FABF4B1B78FE
:1070B000002B01D0FDF7A0FF0022BB5E019A0099D2
:1070C000A21A92100A617F21B94A1D120B409B003F
:1070D0009B580237FDF78EFF01212800FAF714FABA
:1070E000B24B1B78002B01D0FDF786FF0022BB5E60
:1070F000019A0099A21A92100A617F21AC4A1D12CE
:107100000B409B009B580237FDF774FF00212800BD
:10711000FAF7FAF9A54B1B78002B01D0FDF76CFFAD
:107120000022BB5E019A0099A21A92100A617F2187
:107130009F4A1D120B409B009B580237FDF75AFFD8
:1071400003211C20F9F79CFF1C2008F0BDF8013832
:107150004342584101235B1B9B00AE00A61BE41871
:10716000924B80001B783060002B01D0FDF744FF6C
:107170000022BB5E019A0099A21A92100A617F2137
:107180008B4A1D120B409B009B580237FDF732FFC4
:10719000AE00A61B3000FAF719F901235B1B9B0018
:1071A000E418824B30601B78002B01D0FDF724FFE0
:1071B0000022BB5E019A0099A21A92100A617F21F7
:1071C0007B4A1D120B409B009B580237FDF712FFB4
:1071D000AD00641B2000FBF763F9744B1B78002B98
:1071E00001D0FDF709FF0022BB5E019A0099A21AA7
:1071F00092100A617F216E4A1D120B409B009B5822
:107200000237FDF7F7FE0123AD00641B26681E421E
:1072100000D1C6E26168194200D1C2E2A2681A42F6
:1072200000D1BEE21E41802E00D9BFE24B10039375
:10723000FF2B00D9BCE253100493FF2B00D9B9E215
:107240005C4D2B6D002B19D001255B4AAE40D577E4
:1072500000225A4B03989E765A8409F043F804980A
:1072600009F040F8280008F05FFB011E0BD05448DD
:10727000F9F798FB0520F9F77AFE04E006F0CAFD5D
:107280002B6D002BE0D1494B1B78002B01D0FDF773
:10729000B3FE0022BB5E019A0099A21A92100A6105
:1072A0007F21434A1D120B409B009B580237FDF77C
:1072B000A1FE0123AE00A61B3068184202D07168FF
:1072C000194222D10D23394A137000233360012360
:1072D0005B1B9B00E418354B1B78002B01D0FDF79E
:1072E0008BFE0022BB5E019A0099A21A92100A61DD
:1072F0007F212F4A1D120B409B009B580237FDF740
:1073000079FE1523DFE71623DDE740108028F8D843
:107310004910FF29F7D806F00FFF0123400003436F
:10732000D4E7AD00641B23680393DB071FD5039BE1
:107330005D10FF2D00D93FE202F0E2F8E8B208F05C
:1073400021FE1A4B1B78002B01D0FDF755FE0022C1
:10735000BB5E019A0099A21A92100A617F21144A19
:107360001D120B409B009B580237FDF743FE03980C
:10737000F9F70EFE032800D023E2039D08CD1E0975
:10738000B6B25B0F0340B600F61A02F0B9F8042358
:10739000039A5B429B1A0393039B5B19B342D0DAB7
:1073A000287808F0EFFD0135F6E7C046A404002078
:1073B00044480108700600205D100020581000208D
:1073C0006A63010802F09CF8002008F0DBFD01234D
:1073D000400018435B1B9B00AE00A61BE418DB4B70
:1073E00030601B78002B01D0FDF706FE0022BB5E4B
:1073F000019A0099A21A92100A617F21D44A1D12A3
:107400000B409B009B580237FDF7F4FD019B261DA6
:10741000F31AD04D0393D82B04DD1A2334352B7087
:10742000FDF7EAFDEB6C3435049303F0C7FB002352
:10743000C94A04990AF0F6FDC84B400018400123E0
:10744000034323602B78002B01D0FDF70FFE0022B1
:10745000BB5E039A009992100A617F21BC4A1D12FB
:107460000B409B0034009B580237FDF7C3FDAE0074
:10747000A61B33685B100393012D26DD7068C307DC
:1074800023D54010039BC01A02D58023DB05C0180A
:107490000123400018435B1B9B00E418AB4B30609A
:1074A0001B78002B01D0FDF7A7FD0022BB5E019ADF
:1074B0000099A21A92100A617F21A54A1D120B4061
:1074C0009B009B580237FDF795FDA24BDB6C0493A4
:1074D00003F074FBFA220023049992000AF0A2FD43
:1074E00080008008CEE7AE00A61B33685B100393D4
:1074F000012D26DD7068C30723D54010039BC01AF9
:1075000002D58023DB05C0180123400018435B1B14
:107510009B00E4188D4B30601B78002B01D0FDF7E9
:107520006BFD0022BB5E019A0099A21A92100A61BB
:107530007F21874A1D120B409B009B580237FDF7A5
:1075400059FD03F03BFB80008008D7E7019B221D1B
:10755000D11AD82904DD1A227C4B1A70FDF74CFD94
:107560007B883D881B042B432360784B381D1B7898
:10757000002B01D0FDF77CFD04203B5E00988910B4
:1075800001617F2072491D1203409B0014005B586B
:107590000637FDF72FFD0023FE5EBB1CB005400D36
:1075A00038180393FAF740FBEDB2AB00E41AB6B219
:1075B000010023002A00B00AF9F704FA634B1B7894
:1075C000002B01D0FDF757FD0222BB5E019A009906
:1075D000A21A92100A617F215D4A1D120B409B0086
:1075E0009B580437FDF706FD0023FE5EBB1CB0056B
:1075F000400D38180493FAF717FBEDB2AB00B6B2A2
:10760000E31A01002A00B00A0393F9F7DBF9039BA0
:10761000186001235B1B9B00E4184C4B1B78002B6C
:1076200001D0FDF72AFD0222BB5E019A0099A21A41
:1076300092100A617F21464A1D120B409B009B5805
:107640000437FDF7D7FC2200002D00DC8AE0012082
:107650004042F9F78CFC231F1E68012D0CD12E42ED
:1076600007D1042E05D90F22336830001340042BB4
:1076700010D001235B4212E0022DFAD12300083B17
:107680001868C307F5D40428F3D90F220368134000
:10769000042BEED1FAF7C8FAF9F7C6F80300AA00EE
:1076A000A21A591C5ED00020022D13D131000130E6
:1076B0000140064223D1042E21D90F2430682040F6
:1076C00009281CD1706808364010C0B284008C4272
:1076D00011D112190199009C511A89102161FF21C1
:1076E0001C008C431E498C4211D11B061B0C14003C
:1076F0000343FDF7EAFF755855500431E7E71400DE
:107700000B22124B1A70002308C4FDF775FC84008D
:10771000141B2100984700220E4B01C41A64343315
:107720001B78934201D0FDF767FC0022BB5E019AF3
:107730000099A21A92100A617F21054A1D120B407E
:107740009B009B580237FDF755FCC046A40400205F
:10775000444801087004002040420F00FEFFFF7FF4
:1077600000FFFFFF0023140008C4174B1B78002BF9
:1077700001D0FDF741FC0022BB5E019A0099A21ADC
:1077800092100A617F21114A1D120B409B009B58E9
:107790000237FDF72FFC0B23FFF774F91323FFF7D4
:1077A00071F90D23084A1370FDF726FC1523F9E73C
:1077B0001623F7E71723F5E71723034A1370FDF79E
:1077C0001BFC0D23F9E7C046A4040020444801082F
:1077D000012370B50200FF25074C41185B428A4225
:1077E00001D3D84370BD10781E0A2B4043409B0044
:1077F0001B5901327340F2E76055010870B5114D15
:10780000114B2A68C118824202DC0020286070BD3A
:107810000C78461CFA3C012C07D8B24210DD4C789B
:10782000002C02D0283C9F2C0AD830000131EAE716
:107830001C5C01311C7001338A42F9DC101AE5E747
:107840000100F9E7F845002060520020038BC08A50
:10785000181A70471B22024B00201A707047C0464E
:10786000A40400201B22024B00201A707047C0465F
:10787000A40400201C23012808DD012208680F3B16
:10788000104203D04968114200D00E33014A002053
:1078900013707047A4040020012070470120704736
:1078A0000120704701207047012070470120704778
:1078B0000120024B5B685B0018437047F8450020CD
:1078C000C30711D404280FD90F2302681340032BD8
:1078D0000AD1194001335B1AC0215B07C9050B406F
:1078E00002490A40134303607047C046FFFFFF9FF1
:1078F0000020704700207047042070470268030092
:10790000916830B5490701D4002030BD91688907DE
:1079100005D490680B49084010210143916004246C
:107920000948056891682142EED00168491B022987
:10793000F8D910220120996D0A439A65DA6D024345
:10794000DA65E2E7E8FFFF7F040500200121036814
:1079500030B59A689C680C4201D1002030BD0224E9
:107960002242FAD105259A682A40012A17D199683E
:107970000F4D29400C4303219C600E4C1960256873
:1079800099681142E9D02168491B0229F8D91023CE
:10799000816D0B438365C36D1343C36506E01023FC
:1079A000826D13438365C36D1943C1650120D5E71B
:1079B000E8FFFF7F04050020036810B599691A6885
:1079C000436B002B00D0984710BD07203822184B7E
:1079D00010B519689C68890801400131144207D12B
:1079E0001B68DB0A03401348D8400AF065F910BD54
:1079F00098681040082812D098681040202810D0AD
:107A00009868104018280FD0986810401038431E0E
:107A10009841094B40421840064BC018E5E707481B
:107A2000E3E780200002E0E7FA20C001DDE7C0467E
:107A300000100240006CDC02009423FD00127A006A
:107A4000836A30B51A0706D50168284C4A68224077
:107A5000846B22434A60DA0706D50168244C4A68E1
:107A60002240C46A22434A609A0706D50168214C25
:107A70004A682240046B22434A605A0706D50168CF
:107A80001D4C4A682240446B22434A60DA0606D500
:107A900001681A4C8A682240C46B22438A609A06A5
:107AA00006D50168164C8A682240046C22438A601D
:107AB0005A0610D50168134D4A68446C2A40224387
:107AC0004A6080225203944205D14A680E4C2240FB
:107AD000846C22434A601B0606D502680B49536832
:107AE0000B40C16C0B43536030BDC046FF7FFFFFAE
:107AF000FFFFFDFFFFFFFEFFFFFFFBFFFFEFFFFFAD
:107B0000FFDFFFFFFFFFEFFFFFFF9FFFFFFFF7FF1D
:107B1000030088331B6870B5212B21D103000100BD
:107B200080246A331B885631002B19D00A88002A1A
:107B300017D1EFF31084013282F310880168114DE0
:107B40008B682B408B6084F31088EFF3108182F3F5
:107B500010884023026810680343136081F3108883
:107B600070BD0568EA69224208D0026D16780132BC
:107B7000AE6202650A88013A92B20A80013B9BB26A
:107B8000D2E7C046FFFF7FFF030088331B6870B554
:107B9000212B21D10300010080246A331B88563138
:107BA000002B19D00A88002A17D1EFF31084013274
:107BB00082F310880168124D8B682B408B6084F330
:107BC0001088EFF3108182F3108840230268106858
:107BD0000343136081F3108870BD0668F269224286
:107BE0000AD0056D2A880235D205D20DB26205652C
:107BF0000A88013A92B20A80013B9BB2D0E7C046A4
:107C0000FFFF7FFF30B5EFF31084012282F310886D
:107C1000802501680B68AB430B6084F31088EFF399
:107C2000108182F3108840230268106803431360B8
:107C300081F3108830BD030088331B6810B5212BF9
:107C400006D1020056321388002B02D1FFF7DAFF6B
:107C500010BD036D01681C7801338C6203651388C5
:107C6000013B9BB21380F3E7030088331B6810B518
:107C7000212B06D1010056310B88002B02D1FFF7D2
:107C8000C1FF10BD026D046813880232DB05DB0DF5
:107C9000A36202650B88013B9BB20B80F1E70300F6
:107CA0004C331A78012A09D0020002214D3211709A
:107CB000006901394161117000221A707047030098
:107CC00010B594331B680438984710BD01008C31FF
:107CD0000A68F8B50368222A55D1040060345B6A4B
:107CE0002488826D234013700200836D5E3201335D
:107CF00083651388013B9BB2138013889CB2002BD1
:107D00003DD1EFF31086013383F310880568204FCF
:107D10002A683A402A6086F31088EFF3108683F3CE
:107D200010880568AA689A43AA6086F31088202202
:107D30000A60026804675268446712020AD5EFF3CA
:107D4000108183F310880268124C1368234013607B
:107D500081F31088C36E012B12D10022C266EFF3AB
:107D6000108483F3108801680F330A689A430A600D
:107D700084F310880268D169194200D01362F8BDFB
:107D8000FFF79DFFFBE7082299690A439A61F6E72E
:107D9000DFFEFFFFFFFFFFFB02008C321168F8B52A
:107DA0000368222954D104006034596A2488836D01
:107DB000214019800100023383655E310B88013B4D
:107DC0009BB20B800B889CB2002B3DD1EFF3108649
:107DD000013383F310880568204F296839402960F2
:107DE00086F31088EFF3108683F310880568A9687E
:107DF0009943A96086F31088202111600268046706
:107E00005268446712020AD5EFF3108183F3108899
:107E10000268134C13682340136081F31088C36E0B
:107E2000012B12D10022C266EFF3108483F3108875
:107E300001680F330A689A430A6084F31088026865
:107E4000D169194200D01362F8BDFFF738FFFBE794
:107E5000082299690A439A61F6E7C046DFFEFFFFF0
:107E6000FFFFFFFB074B1888074B1B88C01A074B07
:107E70007F30184004D5802301385B42184301301D
:107E80007047C046B84E0020B64E00207F000080EC
:107E900013B56B460268D971073354681900012283
:107EA000A04716BD13B5104A104B128801A992B213
:107EB0000A801A006846C4321288063092B20280E4
:107EC0001A00C23214880088844201D30020108036
:107ED0001A00C23210880988884202D01288985C41
:107EE00016BD01204042FBE7304E0020704D0020BF
:107EF000802010B5074A0849404213880C88803317
:107F00001B1B064C234002D5013B03430133002BCE
:107F1000F3DC10BDB64E0020B84E00207F0000807C
:107F2000B5230A00B0219B00C35889009B00C318E9
:107F300070B55D5804000320002D13D004300240BA
:107F4000213042430831615889188322FC31496F3E
:107F50009200A950A918B8329B58C03ADB68A858BB
:107F60009847002070BDB523B0229B00C3589200F3
:107F70009B00C31870B59C580320002C10D004320D
:107F80009B58002B0BD08025AD00605DFF2806D0EC
:107F9000044A9B682100A25C9847FF236355002098
:107FA00070BDC046010200000A23038000487047EC
:107FB0003400002000207047212817D0222825D027
:107FC000202811D14B780A781B0213438A7816486F
:107FD00012041A43CB781B061343C3600B79037456
:107FE0004B7943748B798374002070470E4AD368B1
:107FF000180A0B704870180C1B0E8870CB70137C1D
:108000000B71537C4B71937C8B71EDE74B88012195
:10801000064A19401172117A002901D00021D1605D
:108020009B07DB0F1374DFE734000020F8450020C6
:1080300010B5037842889A420AD904780019E318E7
:1080400044789BB2052CF6D184788C42F3D110BDD4
:108050000020FCE7F7B5134D134B832107002800E0
:108060000193FFF7E5FF012106002800FFF7E0FF7D
:10807000822104002800FFF7DBFF002E01D010232F
:10808000B371002C03D040232371002363710028B7
:1080900003D04023037100234371432301983B80A5
:1080A0001430FEBD4800002034000020F7B5134D09
:1080B000134B8321070028000193FFF7B9FF01212B
:1080C00006002800FFF7B4FF822104002800FFF714
:1080D000AFFF002E01D01023B371002C03D000237A
:1080E000237102336371002803D00023037102332C
:1080F0004371432301983B805830FEBD8C00002023
:1081000034000020F7B5134D134B832107002800DE
:108110000193FFF78DFF012106002800FFF788FF7C
:10812000822104002800FFF783FF002E01D01023D6
:10813000B371002C03D04023237100236371002806
:1081400003D04023037100234371432301983B80F4
:108150001C30FEBDD0000020B400002012230148D6
:108160000B80704714010020042301480B807047E6
:1081700028010020004870477446002070B5002692
:1081800052008A18050FECB223003733092D00D8AE
:10819000073B0B704E70023100018A42F2D170BD74
:1081A0001A2370B50B800C4B0C4C18680C4B1B68D9
:1081B000C01800280CD021000A4B08227A311D6813
:1081C000FFF7DCFF2100042228008A31FFF7D6FFE9
:1081D0002000783070BDC0465075FF1FB4000020ED
:1081E0005875FF1F5475FF1F00207047C28A018B0E
:1081F0000300914204D90169885C0132DA82704738
:1082000001204042FBE7C38A028B9A4202D90269ED
:10821000D05C704701204042FBE713B50400FF2803
:1082200015D00B4BC200D058002810D04168083040
:108230008900FFF7CDFA01900920FCF7A1FD042287
:108240002100172001ABFCF7DFFAFCF799FA13BD08
:10825000E81D0020002310B501001A001A20FCF7C9
:10826000D3FAFCF78DFA10BD10B507F0C1FE10BDB2
:108270000100020010B541310C7800234032602C1F
:1082800004D1403C0C700363137010BD0363137082
:10829000030092331B78002BF7D109F046FBF4E77B
:1082A000806A10B5836B002B01D000229A63C36BE8
:1082B000002B01D000229A63FFF7DAFF10BD70B5E2
:1082C0000600913633780400051F012B05D1AB6EF3
:1082D000002B02D02800EB6E984702233370002356
:1082E0002000AB6609F021FB70BD10B5002804DC4E
:1082F0001C22074B1A70002010BD0B68DB0702D44C
:108300000D22034BF6E70220F8F731FEF3E7C046F3
:10831000A404002070B500282BDD01250B682B423A
:1083200027D02B41144C63610023A84207D04A6830
:108330002A4204D053105A1E022A00D900230F4AA1
:10834000536101232376032813DDC86805001D400F
:1083500018420ED104280CD90F2203681340042BB5
:1083600007D1F9F761FC064909F080FC002800D02C
:108370002576002070BDC04634010020F84500205D
:108380007A63010870B5012804DC1C220C4B1A70BA
:10839000002070BD01230868184202D04D681D42BC
:1083A00002D11122064BF2E74010F9F72DF8040034
:1083B0006810F9F729F80443EAD41B22004BE6E7DA
:1083C000A404002001207047164B37B51B680A250E
:1083D0001B0200241B0A102B14D1033301A9012016
:1083E0000193FAF725FB43100F481049584309F051
:1083F000EDFCC3210E4BC01809F0E8FC430001203E
:1084000018433EBDCF2006F059FE013D2418002D33
:10841000F8D19720FA21074B8900E4186043F53022
:10842000FF30E9E70470FF1FE8800000FF03000051
:1084300060F0FFFF68F7FFFFF8B5164CE069002811
:1084400001DB07F037FE0120002540420021E061FA
:10845000F8F716FE104B2A005C680920611C5D606D
:10846000FAF7CEFCA8420AD00122630013439446D7
:108470002A000500094E43600835A24200DBF8BD22
:108480005300F35E61465B0097000B43EB510132F2
:10849000F3E7C04634010020F84500206051002079
:1084A000044B10B59869002802D0034806F056FA2C
:1084B00010BDC046F8450020FC4F0020054B0A00C7
:1084C0009B6910B5002B04D0034B0100180006F087
:1084D000FBFA10BDF8450020FC4F0020164B70B58C
:1084E0009B69002B05D12522144B00241A70200013
:1084F00070BD01204042F8F73AFDFFF7D1FF104C64
:10850000051EF4D0002802DA1B220C4BEDE7C11C3B
:10851000002203208910FAF773FC041E02D10A22FC
:10852000064BE2E729000430FFF7C8FF29002000CE
:10853000FFF7C6F9DBE7C046F8450020A404002099
:108540005401002070B5002804DC1C221C4B0020C4
:108550001A7070BD01240D68254206D1042D04D97E
:108560000F232E681E40032E02D02422144BEEE768
:10857000144B9B69002B02D12522114BE7E7012008
:108580004042F8F7F4FCFFF78BFF03002000002BBC
:10859000DFD002DA1B220A4BD9E72A681409A4B2F9
:1085A000520FA4003240A41A9C4200DD1C0021009E
:1085B000281DFFF783FF012064002043C9E7C04660
:1085C000A4040020F8450020064B10B5040098696B
:1085D0000A00002804D0044B2100180006F0B6FB66
:1085E00010BDC046F8450020FC4F00200322E120CA
:1085F000054B10B54002DA63013A9A6307F082FF37
:108600000122024BDA6110BDF8500020F84500202D
:10861000144B70B5DB69002B01D1FFF7E7FF124E59
:10862000300006F09BF9114C051E0ADDC11C00222A
:1086300003208910FAF7E4FB041E04D10A220C4B34
:108640001A70200070BD2A00011D300006F03CFAAF
:1086500020002900FFF734F901204042F8F787FC99
:10866000EFE7C046F8450020FC4F002054010020F1
:10867000A404002070B586B0002805DC1C224E4BF7
:108680001A70002006B070BD0D68EB0702D40D22F1
:10869000494BF5E7494E6D10B369002B03D0002319
:1086A000B36106F0BBFF464B464C1A68464B1000C0
:1086B00018401A4275D1F8F7A7FEC3B23C2B44DC30
:1086C000E02242499B00D200024058581043230048
:1086D000FC33D8630120F8F797FEC3B23C2B4ADC89
:1086E000E0223A499B00D200024058581043FC3423
:1086F000A063280007F006FF0123F920FA21344D7A
:10870000B361AB68890001936C680134604309F080
:10871000D3FA0022019B0093AB6801930099019B5F
:10872000994244D20099019BE31A5B18D218019B2D
:1087300000939042F0D8FFF7B3FE0100102800D953
:10874000102102A8FFF7BAFE9BE7C0220240C02A10
:108750000ED1CE2B0CDC3F231E4903409B005B58FF
:10876000E0211A4A9B009B58C90008401843AEE715
:1087700001204042ABE7C0220240C02A0ED1CE2BDE
:108780000CDC3F23134903409B005B58E0210F4A58
:108790009B009B58C90008401843A8E701204042AD
:1087A000A5E723000A22FC330920DA639FE7009B38
:1087B00001995B1ABAE7C046A4040020F8450020DE
:1087C0000470FF1FFC4F0020F0FFFF00444A010827
:1087D00010E000E0C042010810B5044CA369002B72
:1087E00001D006F01BFF0020A06110BDF84500205D
:1087F00003000022903370B51A602A4B04001E68F3
:1088000003681B681B071CD580213200264B890397
:1088100006F0E8FD002814D0EFF31081012383F364
:1088200010888020226813688343136081F31088C6
:108830002300202288331A6003200023843423700D
:1088400070BD250023688C351B685B0721D580210E
:1088500032002000144BC90306F0C4FD002818D0D4
:10886000EFF31080012282F3108821680F4E0B680D
:1088700033400B6080F31088EFF3108082F3108890
:1088800021688B6893438B6080F3108820232B60D2
:10889000D2E723002022002088331A602A60E06695
:1088A0002067CAE704050020FFFFFF01DFFEFFFF8E
:1088B000836810B5002B01D10BF0BEFCC36898474C
:1088C00010BD836D10B51800D4308268002A03D023
:1088D00000225A84FFF7ECFF10BD10B50200007FA4
:1088E0000138072810D809F0D3F904140F100F0F1E
:1088F0000F120123043A10681B016433C018836807
:10890000002B01D0FFF7D4FF10BD0323F2E70423AF
:10891000F0E70223EEE70222036870B5DD681E6906
:10892000040016420AD0154208D0053A1A610432F2
:1089300002779B69FFF7D1FF0023237704231E42B0
:108940000DD01D420BD00522236852421A61073216
:10895000227720009B69FFF7C0FF002323770823BD
:108960001E420DD01D420BD00922236852421A61CB
:108970000D3222772000DB69FFF7AFFF002323775A
:1089800010231E420DD01D420BD0112223685242EB
:108990001A61193222772000DB69FFF79EFF00235E
:1089A000237701231E420DD01D420BD002222368E3
:1089B00052421A61231F1868C36E002B02D0643024
:1089C000FFF776FF82239B011E4204D02B0602D5BF
:1089D00023680E4A1A61F30504D52B0602D52368D5
:1089E0000B4A1A6140231E4205D01D4203D041228A
:1089F000236852421A6120231E4205D01D4203D033
:108A00002122236852421A6170BDC0467FDFFFFFFA
:108A1000FFFEFFFF002310B5012809D11330584392
:108A2000054BC0188368002B01D0FFF741FF10BD34
:108A300001334008DBB2EFE7C04E002070B5084DAF
:108A40000400EB68184202D0E860FFF7E3FF2B69EF
:108A5000234203D020002C61FFF7DCFF70BDC0462D
:108A6000001802408722F8B52E4D0400002128008E
:108A700092000AF05DF9B5239B00E3582600B0335D
:108A80009B001D51AF239B00E550237C4C36002BEF
:108A90003CD1802382219B000222200007F0FEFEB1
:108AA0000121802331809B000222200007F0F6FE86
:108AB000BC2301265B00E652713B03228321200088
:108AC000FF3B07F0EBFE184B0027236681239B003A
:108AD000EF50D033E358B0339B00E3185B681B685A
:108AE000984785239B00EF500433EF50143BEA581E
:108AF0000220BA4209D0237CBB4211D180239B00C3
:108B00002000310008F0FCF90020F8BD402382214C
:108B10000222200007F0C2FE012140233180C3E77A
:108B20004023EDE7544B00200100100070B5040015
:108B3000822107F021FE230000254C330121200073
:108B40001D8007F019FEBC23B5265B00E55283218A
:108B5000200007F011FEB022B600A35925669B0045
:108B6000E31892009A58AA420BD0B12292009B5867
:108B70005B689847A359B0339B001D51AF239B00FE
:108B8000E550002070BDB523B02273B59B00C358DB
:108B900092009B00C3180D009E58694600220400F5
:108BA0004A71CA80964263D029786032080010402A
:108BB000114238D0202858D1EA886878002A2BD072
:108BC00049B2002910DAB12189005B5831009B6855
:108BD0009847EB881A1C072B00D90722310092B264
:108BE000200008F0C4F915E080239B00F054131C0A
:108BF000402A00D9402303211E4A9BB2B35493322A
:108C0000A1502200FC32D3651366002132002000FF
:108C100008F076F9002076BDB12189005B58290063
:108C20009B689847F6E768780B281ED809F0D8F9B2
:108C300006F21D1D1D1D1D1D1D1D0F18A7239B00C8
:108C4000E35C032B11D16B460222991DC8E7A723D1
:108C50009B00E35C032B08D16B460122591DBFE743
:108C6000A7239B00E35C032BD4D0200008F0ECFD8D
:108C70000320D0E701020000B523F7B59B00C358DD
:108C800004009B00C3180193B023019A9B00D7589E
:108C90000E000320002F19D00F2314250B405D4335
:108CA0006519A869002812D02821B2224B439200EE
:108CB000A258D318596A09F085F80A1E07D10B008B
:108CC000A9612000310008F038F90020FEBD85239D
:108CD00000229B00FA50019AB033D3581B69002B35
:108CE000F3D08422822092008000B91838583200D4
:108CF0009847EAE7AF231E489B00C258A83BD358C9
:108D000070B5002B30D11B4C1B4B220082321D88CA
:108D100011888D4229D31B8812889B1A22009BB28E
:108D20008432138022008232128892B2002B1BD030
:108D300012490D681249CD60B52189004158B03102
:108D40008900415800290FD0A2188224A4000A519A
:108D500008340B5104340D59002D05D101350D5146
:108D60008221036408F0E9F870BD80231288D4E7FB
:108D7000C40A0020364E0020B64E00200405002014
:108D8000F8450020F7B5170000910192002F4CD054
:108D9000A72189008C46264A264DD368264E0020FE
:108DA000834202D025480068C01A6146244C645CA6
:108DB000032C3AD1022838D8107A002835D0280060
:108DC000803034880088241A1E487F34044004D53B
:108DD0008021013C49420C430134BC4200D93C0093
:108DE000002CDCD02B00802680331A881888B61A15
:108DF0002818B44210D22200009909F0F4FF7F2213
:108E000080352B883F1B1B1913402B80009B1B199F
:108E10000093FFF76FFFB9E73200009909F0E3FF15
:108E2000009B2800A21B9919E7E7019BD81BFEBDF8
:108E3000F8450020364E0020B84E002004050020E2
:108E4000C40A00207F00008010B50024064B074AAA
:108E50000749DC60138809885B187F210B40138069
:108E6000FFF748FF200010BDF8450020B84E002055
:108E7000BA4E00200022104B10B51A800F4B10493B
:108E80001A80104B0A801900C0310A80C433C032E6
:108E90001A800D4BBF3ADA7707F0CAF8B5230B4AB0
:108EA0009B00D358B0339B009B58002B02D08122EB
:108EB00092009850002010BDB84E0020B64E002001
:108EC000324E0020704D002039010020C40A0020DD
:108ED00010B5114CE37F002B01D0002010BD07F02E
:108EE000A7F8021EF9D0B52301210C489B00C358F6
:108EF000E177B0339B001B58002B09D08124A400DC
:108F00001A51037C002B05D180239B0007F0F8FF4A
:108F10000120E3E74023F9E739010020C40A0020DB
:108F200037B5164B164A1B8801A89BB20380130065
:108F30006946C4331B8806319BB20B801300C233D1
:108F40001D880C88A54201D100241C801300C23367
:108F50001C88008884420ED01C88601C80B2188057
:108F6000145D18880A88904201D300221A80FFF706
:108F7000AFFF20003EBD01246442F8E7304E0020E0
:108F8000704D0020F0B585B06B46060000921C883D
:108F9000294B01911B68C360284B29491B8802AAF1
:108FA0009BB293800B00C4331B889BB2D3800B0011
:108FB000C2331888D288904201D300221A800A0056
:108FC00002ABC23210889B88984232D802AB9B8891
:108FD0001288251C9B1A9BB29C4200D91D1C0F00B5
:108FE000C2373B88ADB22A00C918019809F0FBFED0
:108FF0003B88EB189BB23B8002AB3A88DB889A42F5
:1090000001D300233B80FFF763FF019B641B5B19C7
:10901000A4B20193002C09D0074BF2681B689B1A7D
:10902000B2689342B8D3009B1B1B0093009805B015
:10903000F0BD02ABDB88CBE704050020304E0020FA
:10904000704D0020F0B507001D009CB23C4B87B06E
:109050001B6803910192C3603A4B3B4A1B8804A9E9
:109060009BB28B801300C433198804AB89B2D980BA
:109070001100C2310E88D8880633864201D3002001
:109080000880110004A8C2310E888088864222D848
:1090900004AB9B8809885B1A9BB2211C9C4200D9B7
:1090A000191C8BB21100C231098852189446002154
:1090B0008EB2B34211D825490A889A1892B20A8012
:1090C00004AA063208881288904201D300220A803E
:1090D0001E00002315E01B88DCE76246505C039A03
:1090E00082421DD1194A13880133F3189BB21380B1
:1090F00004AB063311881B88994201D300231380E7
:1091000001230293FFF7E4FE019BA41B9B1901932B
:10911000029BA4B2002B07D02D1B280007B0F0BD86
:10912000019A50540131C3E7002CF6D0044BFA6881
:109130001B689B1ABA68934200D28DE7ECE7C046E1
:1091400004050020304E0020704D0020324E0020DB
:1091500010B5154809680288144B521892B2028063
:109160001A00C43200881188884201D3C0211180BE
:10917000C0331A88BF2A01D900221A8000220C4B62
:10918000DA77FFF7A5FE021E0CD1B52309489B0034
:10919000C358B0339B001B58002B03D01300012190
:1091A00007F0AEFE002010BD304E0020704D0020B4
:1091B00039010020C40A002010B5002804D103485A
:1091C00006F0CCF8024810BD0248F9E77E630108BA
:1091D000744700209B63010810B5024806F0BEF8F2
:1091E000014810BDAF6301087447002010B5024864
:1091F00006F0B4F8014810BDBF63010874470020B1
:1092000010B5024806F0AAF8014810BDD86301085D
:1092100074470020F8B5431DDB7F04000E001500E5
:10922000002B24D08023408CDB008018984235D856
:10923000238C984218D90700202800D22027390013
:10924000E0690AF0AFFE00280DD0E0612784638C4E
:10925000E0692A00C018310009F0C5FD638C5B1974
:109260006384280002E0FEE70028F0D1F8BD97B241
:109270001800202FFAD821002834BC319AB2974226
:1092800004D80B785B19DBB20B70EAE70A78F05C64
:10929000D218A218743210700133EFE70020E5E70E
:1092A00070B5431DDB7F04000E00002B0BD10200C4
:1092B000BC321378C3189C33197013780133DBB2B6
:1092C0001370012070BD8023458CDB0001359D4269
:1092D00015DC038C9D420AD9202D00D220252900BF
:1092E000E0690AF05FFE002808D0E0612584638C05
:1092F000E269D654638C01336384E2E7FEE7002021
:10930000E0E7F0B5846D05002700C437BB68866EC2
:1093100085B0002B28D0E28A238B9A4224D3A38ADB
:109320009E420DD90196202E01D22023019301994E
:1093300020690AF037FE002811D0019B2061A3822A
:10934000290032002069743109F04DFD0023E382C9
:10935000BB6826830396002B02D10AF06DFFFEE75F
:109360003800FB6803A9984705B0F0BD426E031FA3
:1093700010B51F2A02DC9A6E01329A660200913201
:109380001278012A04D1996E7031411807F0FEF865
:1093900010BD70B5FBF7E4F8FF25E82604002D04A6
:1093A0007603002801D1200070BD03682B40B34232
:1093B00000D10400FBF7A0F8F3E7F7B50190FFF741
:1093C000E8FF01250400FF276D42002C01D1280091
:1093D000FEBD266833143B40152B0DD121000198AA
:1093E000083108F043FC002801D135123D4020002F
:1093F000FBF782F80400E8E71D2BF8D101256D4248
:10940000F5E710B50868F8F70FFCFFF7D6FF013055
:10941000431E9841800010BD10B50868F8F704FCA1
:10942000FFF7CBFF030001205A1C02D0014A9B002A
:10943000985810BDBC11002010B508680C00F8F752
:10944000F3FBFFF7BAFF431C03D06268024B8000B6
:10945000C250002010BDC046BC110020F8B5002845
:1094600016DD0D68EB0713D56D10013D0124FBF7E8
:1094700077F80026FF27644200280CD1002E21D067
:10948000300008F0FDFB01003000FAF7FFF9F8BDED
:1094900001256D42EAE703681A143A40152A0BD1F8
:1094A0001B123B409C4200DA1C009D4201D1060089
:1094B0000836FBF721F8DFE71D2AFAD10124002640
:1094C0006442F6E70120013464002043DFE770B511
:1094D000084D2C6806F08CFD8022D200121B8242BF
:1094E00000DD0200044905486118FFF74BFD001933
:1094F000286070BDF84500206052002078060020EA
:1095000073B500210C20F7F7BBFD01210D20F7F703
:10951000B7FD01210B20F7F7B3FD234B1A68234B4E
:109520001A4234D10D20F7F76FFF06F043FB0E20EF
:10953000F7F76AFF06F068FB0F20F7F765FF06F004
:109540008DFB1B4C0021250001221A4B1A487C354B
:109550001970A0672A8006F0ABFB184BA66F5869FC
:109560001A7E174B009059696B46C9B21A7159712E
:10957000B04203D12E889D88AE4207D02500009EC0
:109580007835A6679B88AB8006F092FB73BD0C20F4
:10959000F7F73AFF06F00EFB0D20F7F735FF06F060
:1095A00033FB0E20C9E7C0460470FF1FF0FFFF0029
:1095B0003C1100209911002000093D0034010020D9
:1095C000F84500200378013B1F2B00D9704701307C
:1095D000F8E710B5FFF7F6FF0378002B0BD001304A
:1095E000222B11D10378002B03D0421C222B03D154
:1095F0001000FFF7E7FF10BD5C2B03D14378002B71
:1096000000D0821C1000EDE73A2BF2D02C2BF0D0CA
:109610007B2B0BD1FFF7D6FF0378002BE9D07D2BF6
:1096200001D10130E5E7FFF7D4FFF5E720225B2BFE
:1096300014D1FFF7C7FF0378002BDAD05D2BF0D0F1
:10964000FFF7C7FFF7E7202BD3DD2C2BD3D0190072
:1096500091435D29CFD0222BCDD001300378002B50
:10966000F1D1C6E7020010B5002816D0FFF7AAFF17
:1096700003780422222B10D0023A7B2B0DD0013A22
:109680005B2B0AD0190030390232092905D92D2B5C
:1096900005D14178303909290AD8100010BD0522BA
:1096A000742BFAD00132662BF7D001326E2BF4D036
:1096B0005A1E93415A42F0E770B5FFF783FF0278D4
:1096C000030001202D2A01D11B18023800220A258F
:1096D00002E06A4301338A1819783039CCB2092C78
:1096E000F7D9504370BD70B50C001500FFF76AFF45
:1096F0000378222B02D00023237070BD6A1E210044
:10970000082501300378222B02D100230B70F4E7E7
:10971000002BFAD0441C5C2B0BD14378841C622BA9
:109720000ED0662B0ED06E2B0ED0722B0ED0742B5B
:109730000ED0002AE9DD0B702000013A0131E1E78B
:109740002B00F6E70C23F4E70A23F2E70D23F0E7FA
:109750000923EEE710B5002815D00378002B13D0AD
:10976000FFF730FF2021027803008A4300205D2AA2
:1097700009D01800FFF72DFF03782C3B5A425341C4
:10978000C018FFF71FFF10BD1800FCE770B50C00F4
:109790001500002901D000230B70002820D0037889
:1097A000002B1ED0FFF70EFF037806002C2B03D1F1
:1097B0000130FFF707FF0600337800207D2B0FD024
:1097C000844204D02A0021003000FFF78CFF3000D3
:1097D000FFF7FFFE03783A2B02D10130FFF7F2FECC
:1097E00070BD1800FCE7F0B50D0004009DB02F78A7
:1097F000002F11D02E2128000AF0EBFB061E0ED000
:10980000431B0093303F092F20D82800FFF754FF57
:109810000190002808DC002420001DB0F0BD2800C5
:1098200008F02EFA0090EDE723785B2BF3D1601C53
:10983000FFF7C8FE01270400019BBB421BD020009C
:10984000FFF788FF041EE6D00137F5E723787B2B6E
:10985000E1D1601C642203A9FFF798FF041EDAD04F
:109860002900009A03A809F06BFA002803D0200011
:10987000FFF7AFFEEEE7002ECED0009B0133ED18D0
:10988000B5E710B504780B2C13D801228823825633
:109890009B1A9B008B4208DC0222962382569B0077
:1098A0009B1A9B008B4200DD0B00024AE400121958
:1098B000536010BD70050020002805DB1F231840F1
:1098C0001E3B8340014A13607047C04600E100E040
:1098D000002809DB1F2318401E3B8340034AD3673F
:1098E000BFF34F8FBFF36F8F7047C04604E100E0B6
:1098F00010B5FF2403220B0021000240D20091404A
:109900009B012340C943934000280ADBC0240B4A33
:10991000800880008018A40002590A4013430351B4
:1099200010BD0F2210400838054A800880008018BA
:10993000C26911401943C161F2E7C04600E100E08D
:1099400000ED00E0F8B50123411DCB77841DE27FD7
:10995000022A03D00422C2631800F8BD0E26026852
:109960001568B54315601568466C9D4315603268EF
:10997000114D2A403260026C104E15001C22154019
:10998000AB4077683B437360C26C836C5A60036D75
:10999000002B06D01A68084D2A401A60436D826D6C
:1099A0005A600123E3770023CB77836B002B00D031
:1099B00098470020D1E7C046FFFEFFFF00000240AD
:1099C00003689A69920701D500229A620122996977
:1099D000114202D199690A439A61704730B5039CDC
:1099E00000682343120489051A43890D054B456815
:1099F0000A43640D234352009D4352082A434260A8
:109A000030BDC046FF63FF0310B5426B194C0BB26B
:109A1000A2421ED0184CA2421BD0184CA24218D011
:109A2000B822F224DB171A40CB07DB17234013437D
:109A30008A0702D5F422134306E0102901D19022AF
:109A4000F9E7202900D10B4301680A6813430B6032
:109A500010BDB822F224DB171A40CB07DB172340D6
:109A600013438A07E6D41029E9D02029ECD16022DB
:109A7000E1E7C046E59E00082DA40008ED9F000820
:109A8000002310B5CA0708D5030041331A782823EC
:109A90001A40CA33282A00D1B03B8A0708D50200F1
:109AA0002824413212782240A2420BD1442213438F
:109AB00009B2002901DAB822134301680A689A43FF
:109AC0000A6010BDF422F2E702000023202110B545
:109AD00042321370013A04001078117021280AD123
:109AE0001122636322631F392000FFF7C9FF00239F
:109AF0004034237010BD1222022122636363F3E716
:109B00000100036810B5040000201A684231087093
:109B1000510417D51A6817490A401A6023004133C7
:109B20001A78292A13D1013A1A70212320002363BD
:109B30000121FFF7A5FF220000234032903413706B
:109B4000237010BD1204E9D51A680B49E4E71A78AE
:109B50002A2AF6D1023A1A70222320002363022116
:109B6000FFF78EFF23000022403320001A70FFF71A
:109B7000FDFBE6E7FFBFFFFFFF7FFFFF184B10B5C0
:109B8000C3620023020003630400202041321070EE
:109B9000537004226363114212D02368596A636AC6
:109BA0001970636A01336362238D002B08D0013B77
:109BB0002385638D013B9BB26385636C1A436264AA
:109BC00020000849FFF75CFF102223682000DA61BB
:109BD0002300002240331A70FEF771FB10BDC0460F
:109BE0000000FFFF0380000070B5050000220400A4
:109BF000413542302B7802703948283BE06262855B
:109C0000626C0A436264022B2AD803212000FFF70A
:109C100037FF28232B70334BA06B6363236B002823
:109C20003FD01A001021113A8A433AD123681A68AA
:109C3000520403D51A682C490A401A60831DDB7F41
:109C4000012B2AD0294B00228363230040331A7052
:109C5000FFF778FE002823D0A06B836B98471FE0A6
:109C600020002349FFF70CFF2000FFF7A9FE2B7807
:109C7000602B10D020222A702368996911420AD0E3
:109C80009969103A114204D0DA61616C0C3A0A43C6
:109C900062642022DA610023BEE72000FEF7E8FAC2
:109CA00070BDE06B0028F8D01022123B9343F4D132
:109CB00023681A68120403D51A680E490A401A600C
:109CC000831DDB7F012BE8D0084B00228363230038
:109CD00040331A70FFF736FE0028E1D0E06BBCE796
:109CE0000000FFFF11A30008FFBFFFFFA1820008D3
:109CF00003800000FF7FFFFFF7B520230500066803
:109D00004135F3612B7804000F00212B2BD1012169
:109D1000FFF7B6FE112323637368204A1340736074
:109D2000002363631E4BE36210231F4204D0F361E0
:109D3000626C0C3B134363642B78602B05D17F0767
:109D400003D5736ADBB20193019B2000FFF738FE55
:109D5000636C2A78602A01D0002B0CD02000616C43
:109D6000FFF742FFF7BD2B78222BD5D10221FFF759
:109D700087FE1223CFE72A78212A09D1013A2A70D7
:109D80002200236342324034117813702370E9E7D4
:109D90002A78222AE6D1023AF1E7C04600E800FE1E
:109DA0000000FFFFF0B5070040373B7804000D00CE
:109DB0001600022085B0012B1AD001233B700F330F
:109DC000194217D01A4215D022682000D361626C64
:109DD0000C3B13436364FFF7F3FD20231D4205D0C2
:109DE0001E4203D029002000FFF786FF00203870B4
:109DF00005B0F0BD04231D4211D01E420FD09D437B
:109E000023685A6A636A1A70636A01336362238D36
:109E1000013B2385638D013B9BB26385DDE76B06C8
:109E2000DA0F002B0CDB02231D4209D01E4207D0A3
:109E3000638D002BD1D0636A226819789162E4E7C0
:109E40002B0635D57306C8D5628D2368002A23D02A
:109E5000208D002820D15968638D8905890DFF2B3D
:109E600008D9FF22802322855B0400902000FFF7A1
:109E7000B5FDB2E7628DE36A92B20393184B228577
:109E80009C46039BD2B2634502D0E36A0090EDE7A3
:109E9000802300909B04E9E75B689B0103D42000CA
:109EA000FFF712FE99E740212000FFF79DFE94E79F
:109EB000002A00D191E7730600D48EE7638D002B52
:109EC000F1D123685A68920100D586E7E16A044A15
:109ED0009142E4D180225968D2010A435A607CE75A
:109EE0000000FFFFF7B5070040373B780400022071
:109EF000012B15D001233B700F33194211D01A42A8
:109F00000FD022682000D361626C0C3B13432021E8
:109F10006364FFF779FD2000FFF752FD00203870E1
:109F2000FEBD4023080641D51A423FD0266832685C
:109F30009A433260638D002B2CD07168638D890544
:109F4000890DFF2B17D9FF25802325855B04002071
:109F5000EAB200902000FFF741FD638D5B1B9BB2CE
:109F60006385413423783268222B10D180231B0271
:109F700013433360D2E7658D1B4BE26AADB2258592
:109F80009A4201D0E36AE2E780239B04DFE7802363
:109F9000DB01EDE773689B0103D42000FFF794FD1C
:109FA000BCE740212000FFF71FFEB7E7194212D09F
:109FB0001A4210D0638D002BF3D1226853689B01A5
:109FC000ACD4E16A084B9942E7D180235168DB01A8
:109FD0000B435360A2E7202319429FD01A429DD021
:109FE0002000FFF789FE99E70000FFFFF7B50600A4
:109FF0004036337804000220012B15D00123337042
:10A000000F33194211D01A420FD022682000D361B9
:10A01000626C0C3B134320216364FFF7F5FC2000C6
:10A02000FFF7CEFC00203070FEBD0223194208D09D
:10A030001A4206D02368226D9A6201235B4223658F
:10A04000F0E740250B063ED52A423CD001212000F6
:10A05000FFF716FD10212000FFF7D6FC638D002BC3
:10A060002CD0638DFF2B19D90023BF35E16C2585DA
:10A07000009380232A0089B25B042000FFF7AEFC26
:10A08000638D5B1B9BB26385230041331A78236881
:10A090001968222A0DD1802212020CE00023658D5E
:10A0A000E16CADB2258500938023EAB289B29B04AE
:10A0B000E3E78022D2010A431A60B3E729002000B7
:10A0C000FFF792FDAEE7294230D02A422ED027007A
:10A0D00001212000FFF7D4FC413710212000FFF7B9
:10A0E00093FC3B78223B5A425341164A9B029B18F1
:10A0F000628DFF2A10D9FF25E16C2585009380230E
:10A100002A0089B25B042000FFF768FC638D5B1BAB
:10A110009BB263853A78BAE7658DE16CADB225856F
:10A1200000938023EAB289B29B04ECE72023194212
:10A1300000D177E71A4200D174E72000FFF7DCFD79
:10A1400070E7C04600200080F7B5056806002B6860
:10A1500041360093C36A04000193202330780F0036
:10A160002138EB6109280CD807F092FD05680B0B2C
:10A170000B0B0B6E056820005D49FFF781FC212366
:10A18000236380226B68120213436B606B68594A29
:10A19000200013406B60FFF713FC009B5B0459D554
:10A1A0002B68554A13402B60A36B002B03D01B6810
:10A1B0005B689BB2638504231F420FD06A6A9F438A
:10A1C000636A1A70636A01336362238D002B05D0C2
:10A1D000013B2385638D013B9BB26385638D002B1F
:10A1E00003D00423626C1343636410231F4211D015
:10A1F000009A1A420ED0628D002A49D13378282B5A
:10A2000033D18023019A9B049A422ED13900200039
:10A21000FFF7B4FC2300002242331A70656C6263BE
:10A22000954244D02000616CFFF7DEFC3378282B88
:10A2300003D139002000FFF7A1FCF7BD20002F4912
:10A24000FFF71EFC22239BE720002D49FFF718FC97
:10A25000002395E78022009B12021342ABD02B68AB
:10A26000284A13402B60E36B9FE731781022236864
:10A2700029290BD124490198884207D02000DA61AE
:10A28000FFF79EFB2000FFF73BFCC3E7DA61C1E765
:10A290002268D3610423626C13436364019A1B4BED
:10A2A0001A42B7D12000616CFFF79EFCB2E727008D
:10A2B000E36A154A403793420CD02000FFF720FC98
:10A2C0002023114A2000E262337025633D70FDF7C0
:10A2D000F6FFB2E720233278337025633D70222ADF
:10A2E00003D12000FFF742F8A7E790342570A4E7D8
:10A2F0000180000000E800FEFFBFFFFF02800000B9
:10A3000003800000FF7FFFFF0000FFFFFFFFFFFE55
:10A3100070B5050040352E780400C36A0220012E76
:10A320000BD0013828701F30014207D0024205D0FF
:10A330002000FFF709FF0020287070BD10200142A7
:10A340002FD002422DD0628D002A1CD12200413232
:10A350001078282807D180208004834203D1200070
:10A36000FFF70CFCE7E7102110782268D16129285B
:10A37000E1D12C488342DED02000FFF721FB2000F2
:10A38000FFF7BEFBD7E72268D0610422616C0A4365
:10A390006264254A1342CED12000616CFFF724FC91
:10A3A000C9E70420014219D0024217D0628D002A69
:10A3B0000DD02268516A626A1170626A013262626B
:10A3C000228D013A2285628D013A92B26285628DB8
:10A3D000002AB0D1134A9342ADD0D0E70820014201
:10A3E00005D0024203D0200007F060FAA3E7022064
:10A3F0000142A0D002429ED0628D002A0DD0636A35
:10A4000022681978013391626362638D013B9BB2CC
:10A410006385238D013B23858DE7034A134200D0DA
:10A4200089E7ACE70000FFFFFFFFFFFEF8B505007E
:10A4300040352E780400C36A0220012E0BD001386B
:10A4400028701F30014207D0024205D02000FFF7DC
:10A450007BFE00202870F8BD102631425ED03242CB
:10A460005CD080273F0250043A401700C00F0743DA
:10A4700051D0E66B002E1DD0002A03D032685268FE
:10A48000564272412600A76B4136002F05D00028A6
:10A4900003D038684068002801D0012A1CD13278E6
:10A4A000282A09D180229204934205D12000FFF787
:10A4B00065FBCEE73200E5E7102130782268D161F4
:10A4C0002928C6D11A488342C3D02000FFF778FA62
:10A4D0002000FFF715FBBCE710212268D1610422A0
:10A4E000616C0A4362643078124AC0B21342B0D140
:10A4F0002138092808D807F0CBFB050C0707070708
:10A500000707050C212323632000616CFFF76CFB18
:10A510009FE72223F7E72368DE619AE708231942C1
:10A5200097D01A4200D194E7200007F0BFF990E7D6
:10A530000000FFFFFFFFFFFE10B5FDF746FA1F21E9
:10A54000094C0A4AA3681B051B0F9B009B580B4034
:10A55000D840074B9862A3685B045B0F9B00D2183E
:10A56000136C0B40D84010BD00100240384B01085E
:10A570003401002070B504000568C3698268006971
:10A5800029680243606902434F481A4301400A4365
:10A590002A606A684D49206A0A40E1680A436A6095
:10A5A000A269A96802434A4801400A430F21AA60F0
:10A5B000EA6A8A43616A0A43EA62464A954215D1C9
:10A5C0000321454A526D0A40013A022A6DD8434997
:10A5D000885C80221202934236D1082863D807F0A3
:10A5E00057FB68620B623062626214003C4AA81832
:10A5F000421E90410001ECE7374B3A4819680906C2
:10A60000490F013107F058FB0300616A364A4900DF
:10A61000895A180007F050FB666840007308C0189C
:10A62000310007F049FB0200304B103A9A423AD809
:10A630000F23020000079A4393B2400F0343EB60DD
:10A640003BE0FDF7C2F936E008282CD807F020FBE4
:10A65000052B0A2B252B2B2B2800FFF76DFF00283D
:10A660002BD007E01C4B1F4819680906490F013120
:10A6700007F022FB626A1C4B5200D15A07F01CFB08
:10A6800066687308C018310007F016FB0200174B0C
:10A69000103A9A4207D8E8600FE0FDF796F9DEE736
:10A6A00080200002E6E7012008E0802212029342A7
:10A6B000D3D1FFF741FF031EA7D100200C4BA366A7
:10A6C00000236367A36770BDF369FFCFFFCFFFFF70
:10A6D000FFF4FF110038014000100240984B0108C0
:10A6E00000BCFFBF006CDC029C4B0108EFFF0000C8
:10A6F000010001000023092803D81B011843C0B240
:10A7000070470A380133C0B2F5E730B5EFF3108473
:10A71000012282F310880168134D0B682B400B60F7
:10A7200084F31088EFF3108182F3108802680F4CD5
:10A7300093682340936081F31088C36E012B0AD184
:10A74000EFF3108183F31088102402681368A34389
:10A75000136081F31088030020228C331A600023D9
:10A76000C366436730BDC046DFFEFFFFFEFFFFEF5D
:10A77000F7B5040000250121071D3888002826D0E0
:10A7800023002A017C339B580193002B07D03F4BB9
:10A79000E95C2369CA431A61DA680A43DA6001385E
:10A7A000AE000A2812D807F073FA06060606060657
:10A7B000066A6A6A3200635DDB0604D52000310058
:10A7C000103006F071FE635DDB071AD400210135FD
:10A7D0000237042DD1D1E36E002B07D0022223696A
:10A7E00052421A61D86803320243DA60002907D066
:10A7F00023691B68DB0703D42000103006F042FFFA
:10A80000F7BD20003100103006F0DEFEDEE720004C
:10A810003100103006F088FE1D491026685C0138B2
:10A82000225C13003340324204D0022825D8430072
:10A83000C9188B88D20707D503281ED807F028FA35
:10A840000215171A012213432269116A0B4313627E
:10A85000019B002BBAD0032810D80C4B195CCB43BA
:10A860001361D3680B43D360B0E71022EBE780227B
:10A870005200E8E780225201E5E7FEE7FEE720000C
:10A880003100103006F050FEA0E7C046B44B01087E
:10A89000B84B0108C36E70B504000D006430002B86
:10A8A00002D007F0A1F870BD07F09EF8AB68002B4E
:10A8B000F9D00222236952421A61D96803320A434D
:10A8C000DA60F0E770B5012503690C001B682B42C4
:10A8D00004D1CB682B4202D1FDF7E1F970BDCB6802
:10A8E000AB43CB60FDF7DBF902235B422361E368F6
:10A8F0001D43E560F2E70F4A0300904213D0802227
:10A90000D205904211D00C4A904210D00B4A03203D
:10A91000934209D00A4A0130934205D0094A0130D6
:10A92000934201D0FEE7002070470120FCE702209F
:10A93000FAE7C046002C014000040040002000401F
:10A940000044014000480140074B10B59A681A685E
:10A950009A689B68054B1B680369013300D1FEE7C9
:10A96000FFF7EAFD10BDC046001002400020024083
:10A9700070B505000C00022A0BD1FFF7E5FF21009E
:10A9800007F09AF92B69010C9962013107F094F9EB
:10A99000040023005A1E93412969E41A2800CC625E
:10A9A000EC61FFF78FFF70BDF8B52F492F4A0B7888
:10A9B0002F4D5BB22F4ED77F002B18DA0023736226
:10A9C0002C002C3423782C4801335BB2237023787D
:10A9D0005BB2BB4203DA23785BB20B2B1BDD736ADD
:10A9E000264A0433934235D9FDF759F938E00B78FC
:10A9F0005BB2BB42E4DA0B78214A5BB2DB00D318CE
:10AA00005B78012BDCD10B7800215BB2DB00985C1A
:10AA100004F01EFCD4E72378194D5BB2DB00EB1881
:10AA200059680022FFF7A4FF23785BB2DB00EB1824
:10AA30005A68736A9B18736223785BB2DB00EB1869
:10AA40005978012905D123785BB2DB00585D04F009
:10AA5000FFFBF8BD736A0B490022C91AFFF788FF94
:10AA6000FF232C352B70F4E760010020F94500200E
:10AA700034010020F8450020A40F00201F4E0000E4
:10AA800070050020204E0000044B10B5986A002885
:10AA900002D00430FDF73FFF10BDC046F84500204E
:10AAA00010B5FFF7F1FF10BD044B10B5D86A0028B0
:10AAB00002D00430FDF72FFF10BDC046F84500203E
:10AAC000044B10B5186B002802D00430FDF723FFAB
:10AAD00010BDC046F8450020044B10B5586B002847
:10AAE00002D00430FDF717FF10BDC046F845002026
:10AAF000044B10B5986B002802D00430FDF70BFF13
:10AB000010BDC046F8450020044B10B5D86B002896
:10AB100002D00430FDF7FFFE10BDC046F84500200E
:10AB200010B508F043FB10BD10B508F03FFB10BD99
:10AB30007FB5002304280FD81B4B5A6B07F0A8F8E9
:10AB4000030F18212A0001210A435A635B6B0B4053
:10AB50000193019BA023DB05180007B000BD022173
:10AB60000A435A635B6B0B400293029B0F4BF3E764
:10AB700004210A435A635B6B0B400393039B0C4B0A
:10AB8000EAE708210A435A635B6B0B400493049B7A
:10AB9000084BE1E720210A435A635B6B0B400593A6
:10ABA000059B054BD8E7C04600100240000400504A
:10ABB00000080050000C00500014005037B5FA2473
:10ABC0000B4A0C4B10689968A400019115689A68AB
:10ABD000009259680131854207D00098081A6043F5
:10ABE00007F06AF86C4300193EBD0198F6E7C046CD
:10ABF0000405002010E000E030B5174C0D00E069BE
:10AC000085B0002801DB05F055FA012328685B4276
:10AC10004010E361F6F7F8FB0023984219DB0025AA
:10AC20001900E061F6F72CFA0C4B022200930C4B52
:10AC3000694603930B4BE0690293019506F004FF0C
:10AC4000684606F0C9FE084C6560FFF7B7FF0423AD
:10AC50002064180005B030BD3401002001B60008A2
:10AC60002D03000835030008F845002010B5FFF754
:10AC7000A5FF064A536C834201D900235364C01ACE
:10AC8000034B83428041404210BDC046F84500203E
:10AC9000204E00000020084B10B55C6C844209D0A7
:10ACA000FFF78CFF0300844200D8031B0020034AF7
:10ACB0009A42404110BDC046F84500203F4B4C0031
:10ACC00070B5B2B00400FFF7E5FF002822D06D4652
:10ACD000022320002B7006F0D3FFC72800D9C7201D
:10ACE0000023013C5E1C834216D132331800FAF770
:10ACF00047F82B003200FF211420F9F785FDFFF7FC
:10AD0000C9FF002806D0084B084A1B6812689B1A26
:10AD10009B0505D132B070BDA25D3300AA55E1E7B5
:10AD2000F9F72EFDEBE7C046740600207006002000
:10AD3000F0B5B9B0F9F724FDA64F3C6805F058F915
:10AD40008022D200121B824200DD0200A24DA348E5
:10AD50006119FEF717F904193C60002C0FD0FFF7BA
:10AD60002DFF2B787864FA2B00D032E2022C08DC1D
:10AD7000FFF77CFF002802D00120FCF73FFD39B02F
:10AD8000F0BD6B78AC78981E242800D91CE207F03F
:10AD900031F9250038003F004300480051001B02F4
:10ADA0005C009900A000F800370184019C011B029F
:10ADB0001B021B021B021B021B021B021B021B02AB
:10ADC0001B023B001B021B021B021B0236001B0264
:10ADD0001B021B021B021B021B02A400FF2C0ED035
:10ADE0002000F9F705FF00227D49E3005A50C918F9
:10ADF0000A711300210013200092F9F737FD032098
:10AE0000BBE72000F9F795FD2000FDF723FAF6E7F0
:10AE10002000F9F7EDFEF7E7012CF0D1F9F792FFEA
:10AE2000EDE7F9F70BFF0020F9F72CFF6D48FFF76E
:10AE300047FFE4E763B2002BE1DB6B4BA20021008C
:10AE40001520D258F9F7BEFFD9E7FEF7A2FA041E83
:10AE500003D1FFF7B3FE7864D1E7FF23A822266869
:10AE60001B0433405203934203D02000F9F744FB04
:10AE7000EDE7230008331800029306F001FF0500F8
:10AE80000530F9F77DFFFB20F9F7A0FC1D20F9F74D
:10AE90009DFC3012C0B2F9F799FCE8B2F9F796FCC4
:10AEA0002812C0B2F9F792FC08235B421B1B029EDA
:10AEB0000293029B9B199D42D7DD3078F9F786FCFF
:10AEC0000136F6E7012C9AD1F9F72AFDF6F786FE4E
:10AED00095E72000FDF7A1F991E7012C8FD1200023
:10AEE000FDF7B8F900231A003D4ED1007158013228
:10AEF000481E81415B18FF2AF7D105240A205C43D4
:10AF0000F9F73EFFFB20F9F761FC2720F9F75EFC1B
:10AF10000020F9F75BFCE0B2F9F758FC2012C0B250
:10AF2000F9F754FC314BFA21186806F04FFF002561
:10AF30000290EB00F05800281FD0416808308900CB
:10AF4000FCF746FC04000520F9F71AFFE8B2F9F710
:10AF50003DFCE0B2F9F73AFC2004000EF9F736FCAC
:10AF60002002000EF9F732FC200EF9F72FFC029BAD
:10AF7000002B02D0180004F0E7F90135FF2DD8D1DD
:10AF800067E7012C12D11A4B64211B68194A1B0276
:10AF90001B0A06A808F0B0FF06A806F071FE210003
:10AFA000020006AB1620F9F72FFC28E7F5F7FCFFA7
:10AFB0006421114B114A009006A808F09DFF02235E
:10AFC00004AA137206A806F05BFE0021020006AB7D
:10AFD000E8E7C046F84500206052002078060020CF
:10AFE000E81D0020F4630108BC110020300000209F
:10AFF0000470FF1F06640108566101080D64010812
:10B00000012C00D0FBE62000FDF724F9CC4BFA21FF
:10B01000186806F0DBFE0026CA4F03903C68002C3F
:10B020002DD03B790493636808349D00A81D0293DA
:10B030006B1C0593F9F7A4FEFB20F9F7C7FB202052
:10B04000F9F7C4FBF0B2F9F7C1FB6B46187DF9F7CD
:10B05000BDFB6B1C1812C0B2F9F7B8FB0498F9F7E6
:10B06000B5FB6519A54213D8F9F78AFB0298039B33
:10B070005843002801D004F067F9F9F781FB013645
:10B080000837FF2ECAD1FFF799FDAF4B5864B6E6DB
:10B090002078F9F79BFB0134E4E7012C00D0AEE601
:10B0A0000024F9F7CBFD230022002100DA200094D0
:10B0B000F9F7DCFBFF222100D200A24807F038FE9E
:10B0C000F6F78CFDA14B1C6099E6012C52D10020B3
:10B0D000F9F712FA002504002F00FF260295002C34
:10B0E00027D19B4C2068F9F7DDF99A493B00029A79
:10B0F0000190009506A808F033FF06A8FFF7E0FDD1
:10B10000954B80201A682368C001591E8B419349D2
:10B110009B035B186421D21A5143CB179B049B0CF1
:10B120005B1800908E499B1306A808F019FF06A82B
:10B130007DE6029B20680133029363689C460233DC
:10B14000FF18031233409D4200DA1D000214324002
:10B15000039262463040834901920090039A06A808
:10B1600008F0FEFE06A8FFF7ABFD2000F9F7C4F9D2
:10B170000400B4E7022C18D1F9F742FA764B2120EB
:10B180001A68734B1B68591E8B4174499B035B18EB
:10B19000D31A06938023DB0107930822002106AB14
:10B1A000F9F732FBF9F7ECFA29E6032C06D1002275
:10B1B000664B1A600120F9F765FD20E6C72CF9D12E
:10B1C000F9F7AEFB09F048F8C83B052B00D916E6A5
:10B1D000E8E7FB2B00D0CFE5042C00DCC8E52E7996
:10B1E000EB7836021E43604B9E4200DDC4E5331D02
:10B1F0009C4200DCBCE5EB5CFE2B00D0BCE56B7830
:10B20000AC78771E222B00D9C8E01A2B05D8072B63
:10B210005CD0082B2ED0701DAFE518001B38072816
:10B2200000D9BBE006F03EFD6B00BA007000A8003C
:10B23000BA000800BA00F7FF2000FDF70BF8FF2C5A
:10B2400014D02000F9F7D4FC6D79484A2100B31ED0
:10B2500000920C202A00F9F709FB3A4BE200D0508B
:10B26000411E8841404205409B181D712000FCF79B
:10B27000D4FFD0E763B2002BCDDB6A79022A13D06A
:10B28000032A1BD0012AC6D1EB79A8791B020343FC
:10B29000287A3749000418436B7AA4001B0603433D
:10B2A0005B001A436250B6E7002FB4DD2F48B11E91
:10B2B000F8F7ECFA2E4BA4001851ACE7AB79A400D8
:10B2C0005A1E93412A4A9B00A350A4E7632FA2DC95
:10B2D0003A00284906A807F086FD0821002304AAA1
:10B2E0005218D35506A8FEF768F8431C93D0204B9C
:10B2F0008000C25821001520F9F764FD8BE7390062
:10B300001C48F9F763FB86E7632F00DD6327002302
:10B31000184A06A99F420FDCFB430022DB173B4083
:10B32000CB181A70152000917B1C2100F9F79EFAAA
:10B330002000FCF78FFF6EE7D05CC8540133E9E7CB
:10B3400030000020E81D0020F8450020B80400204F
:10B3500064060020286401086806002000800108B7
:10B360000363010814640108F6030000665200201C
:10B37000BC11002065520020012C00D04BE7002FAB
:10B3800000DC48E76B79002B03D01C00322B00DD7A
:10B39000322464236343054A13603CE7C83B052B12
:10B3A00000D938E7F9F7ECF935E7C046300000205E
:10B3B00070B505000C00802916DD26220C4B1A7092
:10B3C00070BDF9F753FBFFF7B3FC012003F0BCFF9E
:10B3D000FEF77DF821002800FDF7F6F80028F0D0F0
:10B3E0002D18241AFEF773F8002CF1DCE8E7C046AC
:10B3F000A4040020F7B5002804DC1C22254B1A7099
:10B400000020FEBD244B9B69002B02D12522214B3D
:10B41000F5E70C6801210C420BD00C41FF2C02DD3A
:10B4200028221C4BEBE76B46D81D0470FFF7C0FFCA
:10B43000E6E7042CE4D90F2223681A40042A08D135
:10B440002000F6F7F1FB040006F01AFC01002000D2
:10B45000ECE7032A07D1190989B25B0F8900134071
:10B46000C91A201DE2E7092ACAD10D000F0066683B
:10B470007610AE42C4DB0135AB00E3583B42F8D056
:10B480005B10FF2BCCDC6A463900D01D0370FFF740
:10B490008FFFEEE7A4040020F8450020F0B508680F
:10B4A00087B0C30705D40D22514B1A70002007B096
:10B4B000F0BD4010F5F7A8FF04003C28F6D80221A3
:10B4C000F5F7DEFDFFF77AFBFA260500760020008F
:10B4D00003F0FAFE002867D0FA267600200003F079
:10B4E000F3FE002866D1434BA200D3580190059388
:10B4F0000023039307330F2201250293059B0027A6
:10B5000013409D40059B1B091340042B03D83A4A66
:10B510009B00D218D768FFF751FBFA260490B600BB
:10B520003B692B409D424BD0FA26B6003B692B402D
:10B530009D424CD1FFF742FB06003B692B409D42E8
:10B540004CD0FFF73BFB831BB042AFD0282B05DD6F
:10B550000123029A9340039A1A430392029B013BF0
:10B56000C9D2019B254D039A5A5501330193052BEE
:10B57000BED100212000F5F783FD0122062109201C
:10B58000F7F73EFC002800D190E70B2302000100F2
:10B590000124436008321C312B7801355B002343C2
:10B5A00008C28A42F8D182E7FFF708FB401BB0428D
:10B5B0008DD97BE7FFF702FB401BB0428ED975E7C0
:10B5C000FFF7FCFA049BC01AB042A9D96EE7FFF757
:10B5D000F5FA049BC01AB042A8D967E7FFF7EEFA64
:10B5E000049BC01AFA239B009842A6D95EE7C04686
:10B5F000A4040020444A0108B84B0108404600203A
:10B60000F8B50B4E74687F2C11DCFFF7D7FA356C58
:10B61000084B0700451BD86903F056FE012800D1EE
:10B620006D42631C7360044B6400E5523764F8BDDF
:10B63000F84500203401002060510020024A1368C0
:10B64000013313607047C0460405002080210E4B73
:10B650004905DA6B84B00A43DA63DA6B0A400121E8
:10B660000192019A1A6C0A431A641A6C0A408021EA
:10B670000292029A9A6B49010A439A639B6B0B40B0
:10B680000393039B04B070470010024010B50120E3
:10B69000FDF7D4F90220FDF7D1F910BD10B5042053
:10B6A000FDF7CCF90820FDF7C9F910BD70B50C24E1
:10B6B0001025A8B2013CFDF7C1F96D00002CF8D1AE
:10B6C00070BD032349434B43DB43012A04D0022AC4
:10B6D00007D0C268134002E0C26813400B43C36046
:10B6E0007047C26849001340F8E7F7B505000C0041
:10B6F000431C00D1FEE70F22404B02409200C0B233
:10B700009B1809381F6A03280ED806F0C1FA0226D2
:10B710003035C0232A009B011A409A4204D10823E5
:10B72000374A11680B4313602806000FFFF700FA31
:10B73000390082687943944603224A430300D04388
:10B74000019060460726104326409860032E4CD88F
:10B75000300006F09DFA4B4D2B15C0232A009B01AB
:10B760001A409A42E0D1264A10231168DAE70821EC
:10B77000234A13688B43D6E7214A10211368F9E75F
:10B78000032041431A68019D013E2A400A431A6082
:10B79000012E04D822072DD55A683A435A60A206D2
:10B7A00039001800920FFFF78CFFF7BD6204520EAC
:10B7B00094467F2A0CD02D070CD50F253A0A524308
:10B7C00052435543586AA84365466A43104358623A
:10B7D0000220D6E70A000F254A435543186AA843BA
:10B7E00065466A4310431862F2E7FEE70020C8E7A7
:10B7F0000120C6E75A68BA43D0E7C046B84B0108F3
:10B800000000014010B5431C07D110BD984203D180
:10B810008968FFF76AFFF8E70C310B685A1CF5D10D
:10B82000FEE7431C02D1002006E00C310B685A1CD5
:10B83000F9D09842F9D148687047F8B5124F060020
:10B840003900FFF7EEFFFFF756F8104C8000241880
:10B85000A36A002B0DD1B42007F09EFC390005002F
:10B860003000FFF7DEFF0100280005F0D8FBA36AD7
:10B870001D601C68002C05D0200006F0DBF92000BC
:10B8800007F094FCF8BDC046184F0108F8450020A9
:10B890000300421C05D00868421C02D0834201D13B
:10B8A000886870470C31F6E7F0B5A5B00BAF04001F
:10B8B000642202913800002107F03AFA002304AA1A
:10B8C0005380802322005B011A4003921C420CD05B
:10B8D000C34B9C4209D8C34A0B92C34A944200D13D
:10B8E000AAE09C4200D1AAE0FEE7C04D200029005A
:10B8F000FFF797FF29000B902000FFF7C9FF000317
:10B90000C00E162800D996E0B94B80001B181D6E9A
:10B9100003230B9E0193002E00D189E08023029A1D
:10B920001B067B60082A00D18BE00A2A00D18AE03E
:10B93000062A01D11232BA603B6104237B61033BCA
:10B94000FB6180235B013B63019BAA4A7B63BB6372
:10B950000023BB650593BB6D1463002B1AD18021B6
:10B96000A54A4903136C0B431364136C0B400693F5
:10B97000069B536D9B009B085365039B002B03D1D3
:10B9800020009A49FFF73EFF7021002304AA5218B5
:10B99000FB6513708023B2685B051A4255D0B2680C
:10B9A0000023D20007D41023BA6D1343BB650123D3
:10B9B000FA6D1A43FA6510210424B068BA6D20406C
:10B9C0000A4002435DD1B96D8C4C023221400A43DA
:10B9D000BA65B268D2070FD4F26889490A40B968DB
:10B9E0000A43802149010A43F2603169854A1140C6
:10B9F000802212060A4332610721726901988A4344
:10BA0000024370207261726982430198000102430F
:10BA1000726172690A400199914229D10022032181
:10BA2000FA65BA6D8A4302390A43BA65002B2CD0F5
:10BA3000002025B0F0BDFEE7734D072369E7734D85
:10BA4000FBE7102277E7082275E7B26870490A40E1
:10BA50001343B360674B6F49986A06F02DF94000B5
:10BA60000590059B002B9AD0059B013B0593F8E7B9
:10BA70001223BA6D9A4310231343BB65FA6D012359
:10BA800029E1BB6D0B43BB65D2E77022079304AB82
:10BA90009B181970B3685B0700D59EE0B26A6B0211
:10BAA0005B0A1343B36273692A0293437361002DE7
:10BAB0001DDAC020584B54491A68000410408D42CA
:10BAC0004FD1802109040A4211D11A68534D2A40EE
:10BAD000024311431960474B4E49986A06F0ECF84F
:10BAE0000C23434301330793079B002B36D10023DC
:10BAF00070220125089304AB9B1838001D70FBF7DA
:10BB000025FFB26813002B402A4238D10222B96DBA
:10BB100021400A43BA65F168414A08241140019165
:10BB2000F26840490A40F2608022120694463E497B
:10BB30006546B2680A402A43B260B268002A77DAE2
:10BB4000AE25089AAD0201320892089AAA42F4D3AF
:10BB50001223BA6D9A43023B134394E7079B013BC0
:10BB6000C1E72A498D42C2D18021C9030A42BED110
:10BB70001A682A4D2A40024311431960B7E710237F
:10BB8000BA6D1343BB65002800D051E7B3685B076B
:10BB900000D54DE77021012304AA52180A901370B2
:10BBA000B2681A4200D199E0BA6D204B70211A4058
:10BBB00080235B001343BB651C220023FB653260BE
:10BBC00004AA52181370B368174A1340042213438F
:10BBD000B360F368DB0700D4B5E02023BA6DBBE7A0
:10BBE0000210000000240140011000006853010809
:10BBF000B84B01083401002000100240FDFEFFFF99
:10BC00000102DEFF02FCFF1F000200A4000400A8E6
:10BC1000E8FFFF6F400D030008270140FFFF3FFFD3
:10BC200003800000FC7FFFFFE8FFFF7FFEF0FFFFC7
:10BC300032007F25B4321268013C2A4001329B1841
:10BC4000002C00D074E7B26801340A402243B2608D
:10BC5000802235690433DB08D205954219D33400BC
:10BC60007F25B4342268AA431A4302232260B268B3
:10BC70000A40134301228E49B3600C68B368134233
:10BC80001DD1F36801991943F1600321BB6D8B430A
:10BC900077E7884A1568F02292032A40E0256D0371
:10BCA000AA42DCD3920C033A94400994099A5208B0
:10BCB0000992099A002AD2D0099A013AF8E70B684A
:10BCC0001B1B022BDAD9B3681342D7D01023B96DEE
:10BCD0000B43BB65FB6D1343FB65A9E6B168764A70
:10BCE000114205D01022B96D0A43BA65FA6DF2E728
:10BCF000B268724C22401343B3606E4B1B681B0248
:10BD000013D401226A4908683368134200D04BE714
:10BD1000B368134203D1B36823401343B3600B6885
:10BD20001B1A022BF0D9BA6DA5E6654B6549986AD6
:10BD300005F0C2FF01300A900A9B002BE1D00A9B5C
:10BD4000013B0A93F8E75A4908683368134200D167
:10BD50009BE08023B96D9B000B43BB65C023F1685A
:10BD60001B01194211D133681B070ED5B36813426A
:10BD700000D093E00C22736893437360BA6D524B0A
:10BD80001A400433FF331343BB650C233360219BFC
:10BD90009B0503D5336C04AA9BB253807022012407
:10BDA00004AB9B1838001C70FBF7A8FD002800D0DE
:10BDB0003EE63800FBF7CAFD002800D038E6BB6D30
:10BDC000414A134023437332BB65FF3204AB9B18D7
:10BDD00018700223BA6D38001343BB65FBF78EFD64
:10BDE000002809D13800FBF7B1FD002800D1BC655F
:10BDF000B368364A1340B3607368354A2D4913401F
:10BE00007360344B344A3360F368344C1340072278
:10BE1000F36033699B009B083361736993437361DB
:10BE2000336A2F4A13403362736A13407362F36AB2
:10BE300013400022F362B36AB2620B68234080248D
:10BE40000B60284B64031D6B25431D631E6B264D41
:10BE50002E401E631E6B34431C631C6B2C401C6302
:10BE60001C6C2C401C64702404AB1B19FA653A66E8
:10BE7000BA651A70904200D0DAE50B681B4A13408D
:10BE80000B6004AB588880B2D3E50B681B1A0A2BF1
:10BE900000D85AE7219B13432193C9E52023BA6DAB
:10BEA0001343BB650123FA6D1343FB656DE7C04681
:10BEB000040500200827014017000080E8FFFF7FED
:10BEC00034010020400D0300FEFEFFFFE8FFFF6F7E
:10BED00060F4FFFF9F0B000000021E83FFFF03FFC3
:10BEE00000F000F000100240FFFFEFFFFFFF3FFFF8
:10BEF000030008008B4205D0002B03D04242504182
:10BF00004042184070478022014B12059A607047EA
:10BF100000ED00E003682A4A86B0934217D18020E2
:10BF2000284A0001116C01431164126C0240009216
:10BF3000009A254A934217D18021224BC9021A6CDC
:10BF40000A431A641B6C0B400593059B0CE080228E
:10BF5000D20593420AD101211A4BDA6B0A43DA6304
:10BF6000DB6B0B400193019B06B07047174A93426D
:10BF700009D10221134BDA6B0A43DA63DB6B0B4006
:10BF80000293029BF0E7124A93420AD180210D4BA3
:10BF900009021A6C0A431A641B6C0B400393039B3F
:10BFA000E2E70C4A9342C4D18021064B89021A6C05
:10BFB0000A431A641B6C0B400493049BD4E7C046ED
:10BFC000002C0140001002400048014000040040E5
:10BFD00000200040004401400368184A93420BD1FE
:10BFE000174918480A6C02400A64174A93420CD158
:10BFF000134A1649136C16E08022D205934205D1EC
:10C0000001210F4AD36B8B43D3637047104A93428D
:10C0100003D10B4A0221D36BF5E70E4A934205D1B7
:10C02000074A0D49136C0B401364EEE70B4A934229
:10C03000DBD1034A0A49136CF5E7C046002C0140E6
:10C0400000100240FFF7FFFF00480140FFFFFBFF29
:10C050000004004000200040FF7FFFFF004401403B
:10C06000FFFFFDFF0300421C17D0114A904217D07A
:10C070000BD8104A904215D00F4A904214D080221B
:10C080000F20D205934207D0FEE70C4A90420DD014
:10C090000B4A16209342F7D170470E204042FBE72F
:10C0A0000D20F9E71020F7E71320F5E71520F3E757
:10C0B000002C0140000400400020004000440140EA
:10C0C000004801400300421C17D0114A904217D08B
:10C0D0000BD8104A904215D00F4A904214D08022BB
:10C0E0000F20D205934207D0FEE70C4A90420DD0B4
:10C0F0000B4A16209342F7D170470E204042FBE7CF
:10C100000E20F9E71020F7E71320F5E71520F3E7F5
:10C11000002C014000040040002000400044014089
:10C1200000480140F0B595B00D931AAB0C9204CBCA
:10C1300004001B780B910F931CAB1B780E9210938D
:10C140001DAB1B781193002802D1002015B0F0BD63
:10C150000300A0331B68AB4D180029000293FFF7C2
:10C1600060FB2300A4331E68A74F079039003000FE
:10C17000FFF757FB2300A8331B68A449039018005E
:10C180000493FFF74EFB2300AC331B68A0490890D3
:10C1900018000593FFF745FB390009900298FFF757
:10C1A00040FB290007003000FFF73BFB079B019095
:10C1B000002B01D1002FC8D0731C05D0039B002B8E
:10C1C00002D1019B002BC0D0049B013302D0089BFD
:10C1D000002BBAD0059B013302D0099B002BB4D0B1
:10C1E00003990798FFF784FE002803D138000199CE
:10C1F000FFF77EFE0899FFF77BFE0999FFF778FEAF
:10C20000051E2060A1D0834B984200D0B2E080226E
:10C21000814BD201196B814811431963196B01409D
:10C220001963196C114319641B6C13401293129B10
:10C23000002306931B330A932300069AB1331A7026
:10C240000A9A013B1A70079B002B00D1A9E06D49A7
:10C250000298FFF7D7FA039B002B03D030006A49FE
:10C26000FFF7D0FA002300270293089BBB4205D0BA
:10C2700066490498FFF7C6FA0137FF37099B002B80
:10C2800006D0802362499B0005981F43FFF7BAFA46
:10C29000069A634B92009B18261D1E650B9B6560DA
:10C2A000A3600C9BE761E3600E9B23610D9B6361C0
:10C2B0000C23A361002323620833E362029BE36340
:10C2C0000F9B002B04D00A23E36280235B0263638D
:10C2D000109B002B06D00123E26A1343E362802304
:10C2E0009B022363119B002B06D00423E26A1343B5
:10C2F000E3628023DB02A3630023012163620A98C7
:10C30000FDF7F6FA2300039A8C33002A5AD1019ADA
:10C31000002A57D11A68002A03D1220001998832D5
:10C32000117024221A602B68233A93432B60E36A2E
:10C33000002B02D03000FBF783FB3000FEF71AF928
:10C34000012800D101E76B68364A134022226B6056
:10C35000AB689343AB600823AA681343AB60012327
:10C360002A68300013432B60FCF742FA43425841DD
:10C37000C0B2EBE62C4B984200D0E6E68022264B7A
:10C380009202D96A29481143D962D96A0140D96217
:10C39000D96B1143D963DB6B13401393139B0123B8
:10C3A00047E7002F00D15DE717490298FFF72AFA07
:10C3B000019B002B03D030001249FFF723FA8023A2
:10C3C0001B0250E71A68002A02D1210088310A7046
:10C3D00024221A602B68233A93432B60E36A002BD4
:10C3E00002D03000FBF72CFB3000FEF7C3F8012829
:10C3F00000D1AAE66B680B4A13402A226B60AB6837
:10C400009343ABE7904E0108F44D0108744C0108CA
:10C41000E04C01080038014000100240FFBFFFFF60
:10C42000F8450020FFB7FFFF00440040FFFFFDFF7D
:10C43000B1300278084B92009B181B6D1A008C33A8
:10C44000883210681B681843222318402238434260
:10C450005841C0B27047C046F84500200122036829
:10C4600010B5D96904000438114201D01A620BE0FA
:10C470000222D9691142F9D10422D9691142F5D1B8
:10C480000822D9691142F1D1FFF7D2FF002804D167
:10C4900021002000AE3103F053FF10BDF7B5026854
:10C4A000C14DD3690400116890682B4210D120253A
:10C4B0002B4200D19BE0802676050D400640354397
:10C4C00000D194E0636F002B00D18BE0200084E06A
:10C4D000B64D05400095B64D009E0D40354300D148
:10C4E00085E0250001269035334205D0CF0503D5E0
:10C4F00016622F683E432E60022633420CD0C707D7
:10C500000AD52700166290373E680197B446042684
:10C5100067463E43019F3E60042633420CD0C70766
:10C520000AD52700166290373E680197B446022666
:10C5300067463E43019F3E600826B446334209D019
:10C540002027009E0F40374304D0664616622F68AE
:10C550003E432E6080263601334206D04F0104D57B
:10C56000166220222E6832432A602A68002A39D0B7
:10C57000202213420AD080235B050A4003401A435D
:10C5800004D0636F002B01D02000984722682B68ED
:10C590004027966828223E40134020001E4322D0A8
:10C5A000FEF7B3F823689B683B4218D0EFF3108185
:10C5B000012383F31088250004CD9368BB43936067
:10C5C00081F31088E86F002809D07A4B8363FDF768
:10C5D000B9F9002806D0E86F836B984702E0200085
:10C5E000FFF73CFFF7BDFFF739FF2E60FAE7E56E76
:10C5F000012D00D0CBE01026334200D1C7E03142FC
:10C6000000D1C4E01662936822005C324021178892
:10C610001A000A400B4200D187E0201DC36F1A6840
:10C6200053689BB2002B76D0BB4274D227005E3792
:10C630003B801268202317001F4000971A423DD10B
:10C64000EFF3108C85F3108827685B4B3A681A402B
:10C650003A608CF31088EFF3108C85F3108827680C
:10C66000BA68AA43BA608CF31088EFF3108C85F394
:10C6700010882768BA688A43BA608CF31088220051
:10C6800022338C32FF331360009BE366EFF310819B
:10C6900085F3108822681368B343136081F3108810
:10C6A000C36F002B0AD0981DC27F591D0191022A29
:10C6B00009D00422DA630A00009BD37702232367A0
:10C6C0005E3423888EE70E271A683B491668BE43FE
:10C6D0005F6C16603E680E403E6016681E31AE43C9
:10C6E00016601A6CFF310A409540344E9A6C776898
:10C6F0003D437560DD6C55601A6D002A06D01568E3
:10C700002D490D4015605A6D9B6D53600123019AB0
:10C71000C3770023D1E7BB4200D063E713689B06D1
:10C7200000D45FE7022323675CE721005E310B88BA
:10C7300009889BB2002900D154E7BB4200D151E7E0
:10C74000EFF3108085F3108821681D4F0B683B4084
:10C750000B6080F31088EFF3108085F31088216858
:10C76000184F8B683B408B6080F31088230020219A
:10C770008C331960E2666267EFF3108185F31088ED
:10C7800022681368B343136081F31088CAE78025D9
:10C790006D032B4218D0460216D5210020001562E9
:10C7A000AE3103F0CDFD1DE70F08000001000010C1
:10C7B0002001000419C80008FFFEFFFF000002402E
:10C7C000DFFEFFFFFEFFFFEF8022134207D0802530
:10C7D0002D040A402840024301D0A36F73E6402293
:10C7E000134200D1FEE6114200D1FBE6EFF31080C8
:10C7F000012383F3108821680B6893430B6080F357
:10C8000010882300203A88331A600023201FA36772
:10C81000983423689847E5E6806A0022030010B543
:10C820005E331A80FFF71AFE10BDF0B506000368EC
:10C8300085B0DD691A688C3603929A68040001920B
:10C840003268222A00D0C0E0030068331B88002B26
:10C8500000D190E0030060331B88029320231D4227
:10C8600000D188E0236802995B6AA26D0B401370C7
:10C870002200A36D5E320133A3651388013B9BB296
:10C88000138007232268D5691D422FD0063B1D4225
:10C8900008D00399C90505D52100136290310868B5
:10C8A00003430B6002231D4209D00199C90706D535
:10C8B0002100136290310868DB1803430B600423E6
:10C8C0001D4209D00199C90706D513622200903292
:10C8D0001168023B0B431360270090373B68002B25
:10C8E00004D02000FFF7BAFD00233B6023005E3335
:10C8F0001B8899B2002BB1D1EFF31085013383F37C
:10C9000010882068334F02683A40026085F310882F
:10C91000EFF3108583F3108820682F4F82683A4028
:10C92000826085F310882022326022682167526875
:10C93000616712020AD5EFF3108183F31088226831
:10C94000264813680340136081F31088E36E012BBF
:10C9500037D10022E266EFF3108083F3108821685C
:10C960000F330A689A430A6080F310882268D169FD
:10C97000194200D0136223005E331B889AB2002B49
:10C980001DD0230068331B88934218D9EFF3108021
:10C99000012282F310882168114D8B682B408B6037
:10C9A00080F310880F4B6367EFF3108182F31088D8
:10C9B0002023226810680343136081F3108805B0B8
:10C9C000F0BD2000FBF77BF9D5E7082299690A43FF
:10C9D0009A61F4E7FFFEFFFFFEFFFFEFFFFFFFFBA3
:10C9E000FFFFFFEFCD7C0008F0B50600036885B0BF
:10C9F000DD691A688C3603929A68040001923268E5
:10CA0000222A00D0BEE0030068331B88002B00D12F
:10CA10008EE0030060331B88029320231D4200D167
:10CA200086E023680298596AA26D014011802100B6
:10CA30000232A2655E310A88013A92B20A80072268
:10CA4000DD6915422FD0063A154208D00399C90571
:10CA500005D521001A629031086802430A6002225B
:10CA6000154209D00199C90706D521001A629031F3
:10CA70000868921802430A600422154209D00199FD
:10CA8000C90706D51A6222000223903211680B43AF
:10CA90001360270090373B68002B04D02000FFF77D
:10CAA000DDFC00233B6023005E331B8899B2002B22
:10CAB000B3D1EFF31085013383F310882068344F2E
:10CAC00002683A40026085F31088EFF3108583F323
:10CAD000108820682F4F82683A40826085F3108862
:10CAE00020223260226821675268616712020AD5EB
:10CAF000EFF3108183F310882268274813680340FE
:10CB0000136081F31088E36E012B37D10022E266B7
:10CB1000EFF3108083F3108821680F330A689A437B
:10CB20000A6080F310882268D169194200D013622C
:10CB300023005E331B889AB2002B1DD0230068337C
:10CB40001B88934218D9EFF31080012282F31088DA
:10CB50002168124D8B682B408B6080F31088104B3E
:10CB60006367EFF3108182F3108820232268106836
:10CB70000343136081F3108805B0F0BD2000FBF77C
:10CB80009EF8D5E7082299690A439A61F4E7C046FE
:10CB9000FFFEFFFFFEFFFFEFFFFFFFFBFFFFFFEFCB
:10CBA000997D0008C023802110B5044A5B00090567
:10CBB000D150034B186DFFF771FC10BD00E100E090
:10CBC000F8450020C0238021054A5B00490510B5C7
:10CBD000D150044B586D002801D0FFF75FFC10BD09
:10CBE00000E100E0F845002003000A4910B5486B59
:10CBF000C318EFF30882934205D90C220120064B9B
:10CC000040421A6010BD054A054C121B9342F4D2F3
:10CC10004B63F7E734010020D45700200060002068
:10CC20000004000001204042704780239B01002047
:10CC30004B6070470120704700207047002070470C
:10CC4000FEE716220120024B40421A607047C046A0
:10CC5000D457002001207047F0B5834B85B01E7873
:10CC60000093002E00D0D9E0AE23AD227F4C9B0074
:10CC7000E6500C33E6500C33E6507D4B92000193A6
:10CC80007C4B7D4FA350A72301229B00E2542670CA
:10CC9000BB6D7A4A0A201340BB6502F055FB802326
:10CCA000BA6D1B021343BB650423754D2B71023B08
:10CCB000EB71FF33FF33AB60DC33EC50143BE550DA
:10CCC000704B2F60AE81EB5CDAB2002B20D1A52334
:10CCD0006D4F9B00EA543868431C00D0A0E08021CF
:10CCE0006A4B8901DA6B09300A43DA63DB6B0B406C
:10CCF00003930121039BFCF7FBFD0820FCF7DCFDFF
:10CD0000EB7A012B04D1624A0F3311680B43136095
:10CD100003235C4A5F49AB542B6801261A6CB44666
:10CD20000A4000211A6408002A002F79B94200D075
:10CD30007BE000210800584A8F4200D080E00121AA
:10CD400019641A6C00208A431A641A6C8A40CA401B
:10CD50001A644C4A58646874A9542A7B8A420BD1DD
:10CD6000B52189006A5008396854596D0A435A65DB
:10CD70000222596D0A435A6500202825474A802718
:10CD80001368566899B28C46916889B23B4261D06B
:10CD90006346793F3B406B439C46414B6344B7B28B
:10CDA00000295CD11973DF8001300C320528E6D1EF
:10CDB000002302AA5380AE23019A9B005832E2500E
:10CDC000019B0833DB6F002B05D002AA901C98470B
:10CDD000B4239B00E050B6229200A358A520013353
:10CDE000A350B5239B00E3582E4AB0339B00E318B1
:10CDF0005A60B2239B00E2588000135C012B0AD0DA
:10CE00000024136828495C64196480219D6D09021F
:10CE10002943996514540123009A137005B0F0BD9D
:10CE2000B968FEF762FC0C3755E7664611750131AB
:10CE30005675D07550629062D062C9B2283275E7DB
:10CE4000117001315070D070106150619061C9B2A1
:10CE5000283271E79BB26B439C460F4B9EE7012142
:10CE60009E601973A0E7C0466C060020C40A00202B
:10CE7000340100206C010020005C0040FF7FFFFFB8
:10CE80007448002095020000404D01080010024047
:10CE9000901802407F40FFFFC8490020644D010800
:10CEA00088480020C401002080BF0000802180222B
:10CEB000F0B5B74D09022C681202636C89B01940B5
:10CEC000134201D100F0A9FE8022B14D12022E685A
:10CED000736C134201D109B0F0BD0F270F22736CA0
:10CEE0001F40134200D04EE318000132104013429D
:10CEF00020D13368A74A13408022120213433360C3
:10CF00002B7DA54ADB009B181B68AA6A9B019B0D21
:10CF10002B63D318AB6204F02EFC6B7C002BD3D0B8
:10CF2000EA6A002AD0D180206B7C29680343CB6455
:10CF30006A74C9E7336880221C001201144013424E
:10CF400000D1E8E2AA235B00E85C04F09BFC2B0024
:10CF5000FC335867AD235B00E95A02008F4803F0A9
:10CF600000FE29688E4B0A68A5201A4080231343CF
:10CF70000B60B7239B00EF588A4B8B4AFE180E3B81
:10CF8000E95C884BAA5AF954884B8000EB5CF2802C
:10CF900073709C46864BEC5A0233EB5A0125748021
:10CFA000B3803D5004303A501F200840A84200D1C1
:10CFB0007FE1022800D1A4E1002800D0A3E2603084
:10CFC00001400D006030203D054205D000290ED003
:10CFD000380004F039FC77E7B5239B00FB58AE33EB
:10CFE0009B00DB599B683100380098476CE761462D
:10CFF0000929EDD8604604F055FE29014D01EBFFEB
:10D000003F01EBFF76000A00EBFF10019F0006AB2B
:10D010009D1D0023200A01382B800628D8D804F053
:10D02000DFFF041C2AD7D74C5600AD239B00FB58CA
:10D03000387C1B68290098475A4BFB18D98800296F
:10D0400000D1C9E02A88002AC2D00B1C914200D925
:10D05000131C9AB22B800100F4E0AE233A7C9B00B3
:10D06000FB58002A05D19B6A280098470223437089
:10D07000E2E7DB6AF8E7AD23E1B29B00FB58052944
:10D0800014D8080004F004FE03080A0C0E105B68B4
:10D09000002B9DD0387CCDE79B68F9E7DB68F7E78C
:10D0A0001B69F5E75B69F3E79B69F1E7DB69002B37
:10D0B0008ED02A00387C9847BEE73B7C002B87D176
:10D0C000AE239B00FB5828005B6B9847B4E73B7C82
:10D0D000002B00D07CE7AE239B00FB5828001B6B85
:10D0E00098470723C3E71A4300D071E77F2C00D984
:10D0F0006EE7A7239B00FB5C032B00D168E7A5220A
:10D100002B4BE4B2FC542A33FB589200995C012962
:10D1100007D05C74002C02D180201968C8640021FB
:10D120009954380003F030FFA72302229B00002C03
:10D1300000D10122FA54C7E61E4EE4B23470012C2D
:10D1400000D945E7A725AD007B5DDAB20192022B3D
:10D1500009D0032A37D0380004F076FB21003800CC
:10D1600003F0F8FCB0E6002C36D0AE2301219B0082
:10D17000FB587960002B1FD038001B6898470028A7
:10D180001AD0380004F060FB019B7B559CE6C0463A
:10D19000744800200F8FFF0700980040104B0020BC
:10D1A0008F0FFF07AA020000A20200009D020000EC
:10D1B0009E02000050460020380003F0E5FEA72341
:10D1C00003229B00B6E7002C0AD1022321007B55E5
:10D1D00038007C6003F0BEFC380003F0D5FE73E637
:10D1E00079680129F8D0C9B2380003F0B3FCAE2346
:10D1F0009B003178FB587960002BEDD038001B681C
:10D2000098470028E8D0380004F01EFB7968380001
:10D21000C9B203F09FFC0223B7E7012A00D0D7E68A
:10D22000A7239B00F95CCBB2022907D8002B00D1C1
:10D23000CEE600233900BB60083103E0391D032B23
:10D2400000D0C5E6380003F092FE3DE6A7239B0020
:10D25000FB5C013B022B00D9BAE6022A00D0B7E6FC
:10D26000A9239B00FA580123002A00D00233390079
:10D27000FB600C310222E5E7012C03D1A9239B00BE
:10D28000FC50A9E7022C00D0A2E6A8221B0A9200BB
:10D29000BB54A1E7A7239B00FB5C013B022B00D9F9
:10D2A00096E6012C00D00FE6A92300229B00FA503D
:10D2B00092E760220A40490602D5402A00D087E65C
:10D2C000A7229200BA5C013A022A00D980E6DBB2BA
:10D2D000022B00D97CE6AE239B00FB5803209B6801
:10D2E000002B06D0B52200219200B9503800310041
:10D2F0009847F388002B00D0E6E5002800D0E3E54E
:10D300006AE7602001400D00203D019129000018CE
:10D310000140054234D00199002900D058E660460A
:10D32000D9B2012849D0032834D0002800D04FE6D4
:10D33000A7229200BA5CD0B2022A00D1BCE0032836
:10D3400000D045E60F2214200A404243BA181B06BB
:10D3500000D4BEE0938C002B00D139E67F230B4034
:10D360005A1C50433818802900D1BEE02821B2222F
:10D370004B439200BA58D3189B7D5A1E9341B5E097
:10D38000B5239B00F9501C3BFB589B68002B00D039
:10D3900029E699E5A7239B00FB5CD8B2022B64D059
:10D3A000032800D014E64B0600D115E7224300D035
:10D3B00012E7380004F0D8F90EE7A7229200BA5C11
:10D3C000D0B2022A51D0032800D001E6002C00D0B0
:10D3D0007AE54A063BD0B2229200B8580F2205796E
:10D3E0000A40954233D30722114021324A4385181F
:10D3F0001B0645D50123143282186B7500239370E8
:10D40000A52311709B00C45C012C20D00124C454BE
:10D4100053780468002B3AD0D37812789200A11880
:10D420000A68520605D50C68D94A1440D94A2243E5
:10D430000A60012B07D00B68D74A134020225A40BC
:10D44000D64B13430B60A52300229B00C254380027
:10D4500003F09AFDB52300229B00FA501C3BFB58B9
:10D460009B68934200D0BEE52EE538004B0600D104
:10D47000AFE504F079F98021380004F075F923E56F
:10D4800055325635FF32FF3582182C70B6E78900C9
:10D49000641823685B0405D52268BD4B1A40C04B55
:10D4A000134323602368BF4A1340C02292015A40AD
:10D4B000BA4B13432360C6E7490600D088E539001C
:10D4C0005531FF311B0601D54139FF3900230B606F
:10D4D000D0E66532FF321388002B00D178E548434F
:10D4E0005530FF303818002903D100230222036091
:10D4F000B1E52822B2234A439B00FB589B185733BF
:10D50000FF331B7839E77F239943B2239B00F858F8
:10D5100004F0E0F8D8E41B0400D4D5E43268A24B50
:10D520001A40802313433360AA235B002E00E85C7B
:10D5300004F0A8F9FC36021E706711D0F06E0028C6
:10D540000ED0AD235B00E95A03F00BFBF26E736F54
:10D550002100D218B7239B00E858F26603F01FFDA4
:10D5600029680A68130500D5AEE4C0239B011A4060
:10D570009A4200D1A8E40A688A4802405340874A88
:10D5800013430B60A0E4BB000193F3181A680392E5
:10D590006A4692890292039A120400D486E02824F3
:10D5A0001968814A7C43114080222C190A431A6071
:10D5B000230022006133FF3355321B78FF32157888
:10D5C000002B0DD1280004F05DF9019000284AD00D
:10D5D00023005B33FF33FC3402001988E06E40E027
:10D5E00023005833FF331B78022B00D0E4E0802364
:10D5F000029ADB011A400492029A2800FC341A4273
:10D6000000D198E004F02AF9236F020001908342D0
:10D610000DD200232367AB00F3181968614801405D
:10D620008020800148405D490143196002E01B1AD7
:10D630002367F0D0029B5B0607D5AD0075192968FA
:10D64000534B1940534B0B432B60002A0BD028211E
:10D650007943564B5B1819005D31FF31FC33098863
:10D66000D86E03F07EFA2823190079434F48019DB4
:10D670004218FC32546F64195467D46E6419D4662E
:10D68000146F002C03D0926E954200D3B4E01A00C0
:10D690007A4382185532FF3211784B43C318FC335A
:10D6A000DA6EB7239B00C05803F079FC039B1B067E
:10D6B00001D4FFF709FC3D4D3D492B682824019317
:10D6C000019ABB00944663441A680A40802109020B
:10D6D0000A43210079431A606B18DA7D04927A1CA0
:10D6E0000592049A012A00D0B5E07A1C5443002226
:10D6F0002C1962605A1CD27F002A14D0039A520659
:10D7000000D48BE05A7D002A00D07CE01B7D294AA2
:10D71000DB009B181A68920192091A60802219682E
:10D7200012060A431A6028237B43EB18187D04F085
:10D7300022F8FFF7C9FB04F0A5F8236F020001905F
:10D7400083420DD2049B2367AB00F3181968154878
:10D75000014080208001484010490143196002E0E7
:10D760001B1A2367F0D0029B5B0607D4AD00751926
:10D770002968074B1940074B0B432B60002A00D147
:10D7800071E728217943094B5B1819005F3164E781
:10D790008F8FFF07C0800000BF8FFF0780800000D1
:10D7A00080C000008FBFFF078F0FFF077448002065
:10D7B0000F8FFF0700980040AD0075192968D94BFD
:10D7C0001940D94B0B432B6010788300F3181B686A
:10D7D0005B0408D504F042F80190002800D142E72C
:10D7E00023005D33F6E604F04DF80190002800D1E7
:10D7F00039E723005F33EDE65531FF310918006842
:10D8000003F012FA52E7012A8DD11B7DC74ADB00D3
:10D810009B181A6892B21A601A6883E75A7D002A28
:10D820000DD11B7DC14ADB009B185A6892019209F9
:10D830005A608022596812060A435A6073E7012A27
:10D8400000D070E71B7DB94ADB009B185A6892B282
:10D850005A605A68F1E780220398520010408446CB
:10D8600003981E7D10421ED1B048F2001218059890
:10D87000126844432C1967689201920D974203D8AD
:10D8800063463000636052E7986A143180189862EA
:10D89000A368BE1A9B18019849196660A36003F03B
:10D8A000C3F9FFF711FB4023029A30001A4003929C
:10D8B000029A1A4200D1DFE003F0D0FF7B1C5C43E8
:10D8C0002C196368010000208B4200D9581A2823C4
:10D8D00080257A1C5A43964CED01A2185060029A9A
:10D8E0002A40150000284AD17B43E3185B7D002BBA
:10D8F00036D180218D4AF3009B181A6809069201DF
:10D9000092091A601A680A431A605A6892019209C9
:10D910005A605A680A435A60049B022B0AD1019A42
:10D92000B300D3181A6883490A4020215140824A23
:10D930000A431A60300003F01EFF002D01D1FFF7EB
:10D94000C3FA28237B43E3181A7D236892009B18AF
:10D950001968744A1140794A0A431A60FFF7B4FA09
:10D96000012BD9D1714AF3009B181A6892B21A6040
:10D970001A681A605A6892B25A605A68CBE7002A4D
:10D9800008D0019AB300D3181868664A10406B4A51
:10D9900002431A6028237B43E3181D00383528789A
:10D9A00001284FD1986A4218282002929A627A1C64
:10D9B0004243A2189468641894605C6B5A6A94425B
:10D9C00016D3A41A5C6328237B43594CE3185B7D70
:10D9D000002B46D15549F3005B1819688901890964
:10D9E0001960002A0ED180211D680906294312E022
:10D9F000002C02D10A002C70E5E700222A705A633D
:10DA00002200E0E73E2A08D80125510815401E688B
:10DA100049198906314319600CE01F2515406E42F3
:10DA200075415109491B1D688906294380252D062A
:10DA30000D431D6028237B43E418A18B92B202980A
:10DA400003F0BEF828227A43394B3A499B181B7DD4
:10DA5000019A9B00D3181A680A4030215140364A77
:10DA60007AE7012BE6D13149F3005B18196889B2D6
:10DA700019601D681104B9E703F004FF7B1C6343C0
:10DA8000ED186B68010003988B4200D3581A2823C5
:10DA900080257A1C5A43264CED01A2185060029A48
:10DAA0002A40150000284BD17B43E3185B7D002BF7
:10DAB00028D180211D4AF3009B181A68090692019B
:10DAC00092091A601A680A431A605A689201920908
:10DAD0005A605A680A435A60049B022B0AD1019A81
:10DAE000B300D3181A6813490A4020215140124A42
:10DAF0000A431A60300003F03EFE002D01D0FFF70C
:10DB0000E3F91EE7012BE7D1084AF3009B181A68D6
:10DB100092B21A601A681A605A6892B25A605A68C9
:10DB2000D9E7C0468F8FFF07C080000000980040F3
:10DB300074480020BF8FFF078080000080C0000075
:10DB4000002A08D1019AB300D31818689E4A1040E1
:10DB50009E4A02431A6028237B43E3181D00383590
:10DB60002878012800D06DE7986A42182820029290
:10DB70009A627A1C4243A2189468641894605C6BA1
:10DB80005A6A944216D3A41A5C6328237B43904CB0
:10DB9000E3185B7D002B35D18E49F3005B18596883
:10DBA000890189095960002A0ED180215D68090622
:10DBB000294312E0002C02D10A002C70E5E7002274
:10DBC0005A632A702200E0E73E2A08D8012551084E
:10DBD00015405E6849198906314359600CE01F25DC
:10DBE00015406E4275415109491B5D6889062943FC
:10DBF00080252D060D435D6028237B43E418E18BCF
:10DC000092B21CE7012BF7D17249F3005B185968F7
:10DC100089B259605D681104CAE75A0542D5636C40
:10DC20006D4A13406364B72301229B00EC58403BCC
:10DC3000E254083BE15010336160E150043BE15491
:10DC40001833E358002B04D05B68002B01D0200070
:10DC50009847002240231100200002F01FFEB2234B
:10DC600001265B00E65223004027FC3300225F665A
:10DC700080213B00200002F011FEB7239B00EB58EF
:10DC8000A68427621E74A5239B00EA5CB24201D1E0
:10DC9000FFF721F90022802029686A74C864EA54D9
:10DCA000FFF719F95A0405D5636C4C4A13406364B5
:10DCB000FFF711F980211A0089010A400B4202D0B6
:10DCC000636C474AF2E7D90428D50421236C8B43BF
:10DCD0002364236C49188B432364B3239B00E95CC2
:10DCE000012900D1EA54EB7A002B08D0FDF7AEFCF5
:10DCF00001F078F906213B4A13698B431361B7237E
:10DD0000A7219B00EB5889005A5C042A03D1364AAC
:10DD10009A5CD2B25A54636C344AC7E71A050FD5DD
:10DD20000823226C13432364636C314A13406364F9
:10DD30000423226C1343236401F034FBFFF7CBF878
:10DD40001A061BD5636C2B4A1340B32263649200FE
:10DD5000AB5C002BF0D1216C04330B43236408230C
:10DD6000216C0B4323640123AB543C22636D9B085D
:10DD70001340B4229200AB50FFF7ADF89A051BD5C3
:10DD8000636C1D4A13406364B7239B00E858403B13
:10DD9000C35C032B01D0FFF79EF8AE239B00C35852
:10DDA000002B01D1FFF797F8DB69002B01D1FFF7BA
:10DDB00092F89847FFF78FF8DB0501D4FFF78BF84F
:10DDC000636C0E4A72E7C0468F8FFF0780C0000069
:10DDD0007448002000980040FFFB0000FFBF0000D7
:10DDE000FFDF000000ED00E09D020000FFEF0000FB
:10DDF000FFF700007FFF0000FFFD0000FFFE0000B6
:10DE00000300C06910B5002803D000211A8C04F06B
:10DE10008FFF10BD1722F0B5B34BB44C8BB0DA674F
:10DE20002300002120698833013A1A60E1822183AE
:10DE3000884202D0A28A04F07BFF0026200066847C
:10DE4000A676FFF7DDFF231DA948DC6702F026F95F
:10DE500080239B00A38423000125BE3327001D805F
:10DE600023000837C033F86F1E7001F00DF9310040
:10DE700001F090F90F21FB6F1A090A40042A00D91A
:10DE80002DE19C4E92000B40B218D2689B00F31813
:10DE9000196A1369984A0B401068994264D001F0DE
:10DEA000F3F8290001F076F9142301930F21924B26
:10DEB0001B681A090A40042A00D912E10B40092004
:10DEC000FA2192009B00B218F318D7681B6A8B4D99
:10DED000BB620393AB68890006936B6801335843B8
:10DEE000029303F0E9FE0022069B0793AB680693BA
:10DEF0000799069B994200D3A7E0079B02999C468D
:10DF0000069BCB1A6344D218069B07939042EDD828
:10DF10000920FA21039B8900BB61AB6804936F68F9
:10DF20000137784303F0C8FE0022049B0593AB68D9
:10DF300004930599049B994200D38AE00599049BB8
:10DF4000FB1A5B18D218049B05939042EFD8019BF3
:10DF5000013B0193002BA9D123008833186801F0FD
:10DF600093F8019901F016F923000833DB6F019350
:10DF7000634B019819000293FDF753FC230088338B
:10DF80001E68604F050039003000FDF74AFC0100B3
:10DF9000002D00D184E0002800D181E0A31DDB7FAB
:10DFA00028000393FDF7A4FF051EA06278D0564B0E
:10DFB000984252D18022554B9203D96B1143D963B9
:10DFC000D96B114009910999D96A0A43DA62DA6A70
:10DFD0004F490A40DA62230017228C331A704D4BE6
:10DFE0004D4ADA6539003000FDF70CFC02990198C2
:10DFF000FDF708FC4948E56201F010FC039B002294
:10E0000063630123A363230020632264E263BF33BD
:10E010001B788C25591E8B41DB04A3642300C0337D
:10E020001B78591E8B415B04E36423006D331A7027
:10E03000655702212800FBF75BFC2800FBF73CFC3E
:10E0400001F014FC002824D0FEE7079B06995B1A18
:10E0500059E7059B04995B1A74E7314B9842C1D18B
:10E0600080222A4BD203D96B1143D963D96B11405B
:10E0700008910899D96A0A43DA62DA6A29490A409A
:10E08000DA62230018228C331A70224B224A1A6655
:10E09000A8E723009033186023000222BD331A70D2
:10E0A0002300BE331B78002B0DD123001A4D1E4ACE
:10E0B000983328001A6003F038FC1C4B9434280075
:10E0C000236003F032FC1A4803F040FC0122194B94
:10E0D000002152201A6000F02FF80BB0F0BD336918
:10E0E000FFDE00239B62FBE7601000205810002039
:10E0F0002C110020B84B0108E010002010E000E0D7
:10E10000DC5401085854010800540040001002403B
:10E11000FFFFDFFFF845002084100020A0860100EB
:10E1200000580040FFFFBFFFC388000803930008AA
:10E13000801A0600C0060020F7B5184C05002368B9
:10E140000191002B14D001260027154B154C019886
:10E15000DE776B00A376678402F0C4F8380001F024
:10E16000E3FB071E0BD00520F2F701FF7F4212E010
:10E17000FFF750FE2368002BE5D16427F6E7310056
:10E18000280001F0FBFF228BE38A9A4203D0200093
:10E19000FAF72CF807003800FEBDC046C006002084
:10E1A0005D1000205810002070B500281ADD0C68A2
:10E1B000E30717D50C4D2B68002B0ED0012004412E
:10E1C0000A4A8440D0770022094B9C765A8401F099
:10E1D000ABFB002806D1043070BDFFF71BFE2B6897
:10E1E000002BEBD10020F7E7C00600205D100020D7
:10E1F00058100020F7B5012801DC0120FEBD0B6896
:10E2000001930123019A1A42F7D04D682E001E4057
:10E210001D423BD1042D39D90F222B681A40092AFF
:10E2200029D16C6800966410002CE6DD214F3B6814
:10E23000002B30D0202C00DD202401204042F2F7BA
:10E2400096FE019B2100581001F098FFFF271A4805
:10E250003B00018BC28A914202D0F9F7C7FFC3B2DB
:10E26000009A002A1DD093550136B442EFD1012007
:10E2700064002043C2E7032A08D11C09A4B25B0F43
:10E280001340A400E41A2B1D0093CDE724220B4B6E
:10E2900000201A70B2E7FFF7BDFD3B68002BACD041
:10E2A000C8E7290001205B000831B20003438B500E
:10E2B000DAE7C046C006002058100020A404002061
:10E2C000F7B5012203001000934245DD0D682A4294
:10E2D00042D04C680092022B05D08B68043B5A4216
:10E2E0005341DBB200933A4E3368002B2ED001200D
:10E2F00001274042F2F73BFE364B374EDF776B107B
:10E30000BB402500B37600233D4073843C4224D1BA
:10E31000042C2BD90F2223681A40092A32D1172640
:10E3200063685B100193019B9D421FDA2300AA00E2
:10E3300008339858384222D04010FF2801D9274B83
:10E340001E70C0B201F0CEFF0135ECE7FFF762FDB1
:10E350003368002BCBD10020FEBD6410FF2C02D906
:10E3600017221E4B1A70E0B201F0BCFF009801F0BA
:10E37000DBFA0028EFD00520F2F7F9FDEBE7174BA9
:10E380001E70E1E7032A12D1190989B25B0F13400D
:10E390008900CF1A04235B42251D1C1B63199F4271
:10E3A000E4DD29783000FAF77BFF0135F6E7042A2F
:10E3B000DCD12000F3F738FC070003F061FC040017
:10E3C000A542D3DA795D3000FAF76AFF0135F7E745
:10E3D000C00600205D10002058100020A40400207A
:10E3E00070B500280CDD0B68DA0709D55D10032B2A
:10E3F00006DD074C2368002B04D0280003F0A6FAA2
:10E40000002070BDFFF706FD2368002BF8D0F4E76D
:10E41000C0060020002110B50400C18201830069FC
:10E42000884202D0A28A04F083FC00232000638487
:10E43000FFF7E6FC10BD204A030010B5904234D12E
:10E440001E4CC022616D92010B001340114204D199
:10E45000FCF772F800280AD010BD802252019342C6
:10E4600002D1F9F7B2FAF5E7226852050ED4C022BC
:10E47000636D9201134080225201934212D0802298
:10E480009201934206D0002B13D0FEE78022920126
:10E490009342ECD121680A480906490F013103F083
:10E4A0000BFCD9E7074B986AD6E7074A002093424E
:10E4B000D2D1FCF741F8CFE70054004000100240F1
:10E4C000006CDC023401002000580040F0B58C4A9A
:10E4D000A1B01091C90003005018446E9C4203D1B2
:10E4E000806E002800D009E1864F521858081900A4
:10E4F0005366C01903F0E0FB1C23109A824D5A4367
:10E50000AC18A16E06004808C0190A9203F0D4FBAB
:10E510000A9B6835ED18EA8A2B8B0B92A97E2A8A12
:10E5200011900B9812931218CB1C734312981792E8
:10E53000AA8971431218323AD21A0192D243019831
:10E54000D21710400190EA890B98F318121A053A75
:10E55000FF3AD31A0293DB43029ADB171A400C915D
:10E560003800E16E029203F0A7FB216F189038008B
:10E5700003F0A2FB0C9A73009B1832331593F51825
:10E58000119B002419901393012010230D941493D0
:10E59000404222071E920022E3B21693159B099275
:10E5A000EB1A0F93179A0F998A4200D992E0099AB1
:10E5B0001E990A431D92002208920792019A079918
:10E5C0008A4279D8029A8A4276D3169A149991424D
:10E5D00072D00D9A01320D92072A00D98EE00A9965
:10E5E0004A4A5218528A0B991A92129A5218521980
:10E5F0000E920C9A0899AA1A05921D9A0A431C9227
:10E600000022069205990C9A52181A99914245D205
:10E61000059A323A9208964240D20E9A06995219B9
:10E6200000921C9A0395114300220492374A1B91D1
:10E630001F92199A00998A4221D8189A8A421ED3A9
:10E640001F9A0A995118898A039A8A4217D39642C7
:10E6500015D2119A0099891ACF17CA1913997A40BD
:10E6600017008A420BD21B9A049825491043109A2E
:10E670001397D2009446169A614488661492009AC1
:10E680000499D2180092039A0131FF31D2180491F3
:10E6900003920A00802149028A42CAD1069A0132B5
:10E6A00006920E9A0699D2180E92059AD2180592E1
:10E6B000802252009142A5D1079A0899D218079258
:10E6C000802252028A1808928022089952039142AD
:10E6D00000D073E7802149038C460F9AD2180F921D
:10E6E000099A62440992802209995204914200D009
:10E6F00058E70134AD19102C00D04AE721B0F0BD25
:10E70000F845002000CA9A3B384D0108A04D010889
:10E7100070B58025174B6D00DC6D2000F9F74CF9C2
:10E72000236899691A68294206D0100604D5012089
:10E73000666C30436064DD618025ED00294206D0BF
:10E74000100604D50820666C30436064DD618020CB
:10E750008000014206D0120604D50222616C0A43F1
:10E760006264D8610B23616C194202D02000FBF770
:10E770003BFA70BDF845002010B5024B186EF9F752
:10E780001BF910BDF845002070B5002815DD0E6896
:10E790003000F2F7FDFB03280FD1350008CD1C092E
:10E7A000A4B25B0F0340A400E41AFAF7A9FE042305
:10E7B0005B429E1B73199C4201DC002070BD2878CF
:10E7C00001F0E0FB28700135F4E7F0B5354BA3B05C
:10E7D0009B69002B05D12522334B1A70002023B0F2
:10E7E000F0BD012802DC1C222F4BF6E74B685C10C1
:10E7F0000193671E02D512222B4BEEE70D6828000D
:10E80000F2F7C6FBC31E0600012B04D9092802D06B
:10E810002422254BE1E70122019B134202D1224B26
:10E820001032DAE7FAF753FE092E26D16A68521041
:10E8300097421ADA002102A8A2420CDB0126013419
:10E84000A300EB58334214D03341FF2B13D80B54A1
:10E8500089198029F0D102A8F9F7B6FE0400FAF769
:10E8600036FE012064002043B9E712230E4A1370DC
:10E87000B4E71123FAE72823F8E7042E0AD1280089
:10E88000F3F7D2F903F0FCF98742B4DA0334C11B81
:10E890002819E1E72B68180980B25B0080009B0F04
:10E8A000C01AF1E7F8450020A4040020284BF7B572
:10E8B000DB6904000D00002B01D1F9F797FE012C54
:10E8C00005DC1C22234B00261A703000FEBD6F6849
:10E8D000FB0702D411221F4BF5E72D682800F2F741
:10E8E00057FBC31E012B02D924221A4BEBE77F10E2
:10E8F0007C1E02D51222174BE5E704281FD1280001
:10E90000F3F792F903F0BCF9A042F3DD124B041BBC
:10E910001800019300F03BF8844200DD040001265A
:10E92000002CD2D0F91C22006918019800F00EFAD0
:10E930000120B4404042F2F71AFB2643C5E72B689A
:10E94000180980B25B0080009B0FC01ADCE7C0464C
:10E95000F8450020A4040020FC4F0020AA23A82191
:10E960005B00C35A4900405A4033181A3F231840ED
:10E970007047AA235B00C25A043BC35A9A4203D091
:10E98000FC30C26CD05C704701204042FBE7A923F9
:10E99000AB225B005200C35C805AC0B2834202D3F8
:10E9A000C01A3F307047C01A0138FBE7037C002BC8
:10E9B00009D0054BAB211B68A9235B00C25A490053
:10E9C000435A9A42FCD170470405002013B56B46A8
:10E9D0000268D9710733546819000122A04716BD97
:10E9E0000300FC33DB6BF7B5040001333BD1036854
:10E9F000DB6898475E23FF33E55C002D33D10122AD
:10EA0000E25423003933FF331B6801332BD14634E2
:10EA1000FF342178144B8900CB58190084310878D1
:10EA2000904220D01C00242088340A702060EFF32C
:10EA30001080019082F310881E68306807000C2057
:10EA400087433760019880F31088EFF3108082F3DA
:10EA500010881A68042316683343136080F3108803
:10EA6000202323600D70F7BD4846002010B5040038
:10EA7000FFF7B6FFAA23A8225B005200E15AA35A6F
:10EA8000994208D02100FC31C96CC85C3F21013398
:10EA90000B40A35210BD01204042FBE770B50400BB
:10EAA000084D2B68C360236820005B6998470028E5
:10EAB00007DAE2682B689B1AA2689342F3D301201D
:10EAC000404270BD04050020F8B506000F00150097
:10EAD0000024AC4201D12000F8BD3000FFF7DEFF7A
:10EAE000431CF8D038550134F3E7F7B50F00160092
:10EAF0001D001C1E01900BD000240198FFF7CEFFD3
:10EB0000431C05D0B84203D030550134A542F4D19E
:10EB10002000FEBD30B50F250F4803681A092A40B2
:10EB2000042A15D80D4992005158002910D00C4CD8
:10EB30002B4042689B001B59002A0AD001DD013A94
:10EB400042601A00486902401204834313438B61F8
:10EB500030BD8B62FCE7C04608000020C44B0108B2
:10EB6000D84B0108FA21104B10B51868890003F042
:10EB7000A3F88022431E52040120934212D2C021E6
:10EB80000A4C0B4A6360136A09061B021B0A0B43FB
:10EB9000136200200723A0602360136A1B021B0A74
:10EBA0001943116210BDC0465C01002010E000E076
:10EBB00000ED00E0202370B5FA260C4A0C4CD16819
:10EBC000B6009943D1602568D16808001840194201
:10EBD00001D0002009E02168491BB142F4D9D26874
:10EBE0001A4202D10320034BD87770BD00280040A1
:10EBF000040500200E05002070B504000D0000285B
:10EC000055D0030006000020334A9C331A60B0360A
:10EC10003056FAF75DFE2200B13212782F4B920087
:10EC2000D35822001800C23288301188026889B295
:10EC3000202A38D1B83422685218002A33D0ADB215
:10EC4000002D30D0802499686401A14204D11C6950
:10EC5000002C01D1D40726D41A651A00002454329E
:10EC600015805580D4633C322122026080228020AE
:10EC70005C6E9205400194421AD1194A814204D136
:10EC80001969184A002900D0154A9A67EFF31081D4
:10EC9000012282F310881A68802390681B040343C2
:10ECA000936081F3108800203056FAF705FE70BD9E
:10ECB0000D4A814204D119690C4A002900D00A4A40
:10ECC0009A67EFF31081012282F310881A6880237B
:10ECD000106803431360E4E7F1EC000848460020A5
:10ECE000117B0008897B0008377C0008697C0008DC
:10ECF0000300020070B5C233C432198814680919C0
:10ED00003F24214019800100BE3109881D8800245C
:10ED1000A94216D01D8840311C880B4B491BA4B258
:10ED2000194004D5402301395B4219430131402386
:10ED30001B1B994200D9190001241160FFF75CFFE9
:10ED40006442200070BDC0463F000080F0B50368FB
:10ED500085B09B680292009104009847A9235B004C
:10ED6000E65A23004022FC33DB6B961B3F3A070038
:10ED70002274013334D15E23FF33E15C00292FD0AC
:10ED8000200000214630E154FF300178454B8900D6
:10ED9000CB581800843001900178914220D0242172
:10EDA0000270043003900160EFF3108C82F310883E
:10EDB0000C201D682968814329608CF31088EFF3CB
:10EDC000108182F310881A68082315682B4313609A
:10EDD00081F3108820230021039A1360019B19708E
:10EDE000236820009B6898470028F9D0029DB5420F
:10EDF00032D8BD4230D8A92327005B00E35AFC3744
:10EE0000386D5A19C018402A3FD82A00009903F0DB
:10EE1000EAFF2E00A9223F215200A35A20005B19CD
:10EE20000B40A35222004632FF3212781D4B920053
:10EE3000D258943013008C3288331B681268134305
:10EE400021221340934204D0FC343100E665FFF7E1
:10EE5000D3FE029805B0F0BDBE4200D93E00236843
:10EE600032005B68009920009847009B20009B19A6
:10EE700000932368AD1B9B689847A9235B00E65A63
:10EE8000133BFF3B07009E1BB1E74026F61A3200FA
:10EE9000009903F0A8FF009B386DAA1B991903F095
:10EEA000A2FFB7E7484600202023F0B5474D85B0C4
:10EEB000EC6A0190A1690A001A40194201D00020B1
:10EEC0003FE0A76910203E001100064007420CD029
:10EED0009446E0613E4F0198A16919425AD16146BA
:10EEE000002930D00426012116438020A269400069
:10EEF000024202D00121E0610E438020C0000242A4
:10EF000003D00821E0610E430739802080000242CF
:10EF100045D00223E0611E432E48FAF751FD636895
:10EF20002D4A134063602B6F202233432B672B0045
:10EF30006D331A7000236E352B7000220120274B91
:10EF40001A7005B0F0BD3968091A6429C4D961681E
:10EF5000029123490E78F1B280260391A16936020D
:10EF600031420BD08021029EC9010E4206D1039E80
:10EF7000202E03D06068014361603868144EA16997
:10EF80001942A9D13168091A1929F8D901211A00A1
:10EF90008C46A1E761460029A4D1E361A2E70029DC
:10EFA000BAD10B4A01981268121A642A00D881E774
:10EFB000A2691A4200D07DE72A6F1A432A672A0005
:10EFC0006E356D3213702970B7E7C04658100020B7
:10EFD000040500208410002000E800FEC41000207A
:10EFE000C61000200723204910B50A689A43063B43
:10EFF000134380220B601D4B520019680A431A60AC
:10F000008022D20019681142FCD080221968D203F4
:10F010000A431A608022120419681142FCD0596810
:10F02000134A11408022D2010A435A601A681149DA
:10F030000A401A609A6810490A4007219A609A6843
:10F040008A439A60382299681142FCD19A680B4928
:10F050000A409A600A4B0B4A1A60FFF783FD0028AA
:10F0600000D0FEE710BDC046002002400010024064
:10F07000FF80FFFFFFC7FFFFFFF0FFFFFF8FFFFFD6
:10F080005C010020006CDC020206030010B53D208C
:10F09000120F042A0AD80020074AD9B28400145952
:10F0A0008C4204D1E022D2001340184310BD01303D
:10F0B0003D28F3D1FAE7C046444A0108F7B5FF22DC
:10F0C0000400010014400E2C10D82F4BA000C35890
:10F0D0001A403C2A29D9C0201840C02801D1CE2A84
:10F0E00034D90020CF292CD1284827E0C02505405D
:10F0F000C02DF6D1CE2CF4D803003F2633409B0020
:10F10000E02001930B00C00003409C461E4F019B72
:10F11000DB5967463B431A403C2A13D91D40C02D9A
:10F12000DFD1CE2ADDD8334012E0194892001258C0
:10F13000E020C00018401043431CD2D00A21FCF745
:10F14000B3FBFEBD124C92001259F3E73F2213406D
:10F150000D4D9B005B590E4A9B009858E022D2004F
:10F160000E2C04D8A400635913401843E4E7C024CC
:10F1700013000C40C02CF8D10B00813C0C40A400C3
:10F18000645913402343EFE7C04201080110000017
:10F19000444A0108F7B5C3B2040001913C2B14D8CE
:10F1A000E02227499B005C58D20002401443631CB4
:10F1B00036D00F2625093540224FAD00EB592640A9
:10F1C000F340DB071FD5204B15E0C0220240C02AC8
:10F1D00026D1CE2B24D83F231C4903409B005B58EB
:10F1E000E021174A9B009B58C9000C401C43DEE7F6
:10F1F000944221D00C331A68511CF9D10122B2403B
:10F200007B5993437B51019B052B14D8180002F0C6
:10F210003FFD030E080A0C1000212000FCF765FAE0
:10F22000F7BD1021F9E72021F7E70321F5E70121D8
:10F23000F3E70921F1E7FEE72000FCF7FEFADDE73E
:10F24000444A010860560020184F0108C0420108D6
:10F25000C3B210B53C2B19D8E022174C9B00D2004A
:10F26000024018591043431C0FD0030600221B0F05
:10F27000042B02D8114A9B009A580F24104B2040AF
:10F280008000C358002914D0936110BDC0220240F1
:10F29000C02AFAD1CE2BF8D83F230A4C03409B005A
:10F2A0001B59E024044A9B009B58E400204018436B
:10F2B000D9E79362E9E7C046444A0108C44B010814
:10F2C000D84B0108C0420108C2B2030010B53C2A65
:10F2D0001BD8E02118489200C900194013580B436D
:10F2E00000205A1C10D00F241A092240042A20D8CA
:10F2F0001249920051582340114A9B009B580869BB
:10F300001840C01A4342584110BDC021014000209E
:10F31000C029F9D1CE2AF7D83F220A481A409200D4
:10F320001258E020044992005258C0000340134391
:10F33000D6E70369FFDEC046444A0108C44B010812
:10F34000D84B0108C0420108034A116813685B1AD0
:10F350008342FBD37047C0460405002070B50D0002
:10F36000040002F08DFC8021C3B2013349000A0081
:10F370005B008B4200D89AB20323002008492A8000
:10F380004B700A70013B2278002A00D170BDCA542C
:10F390005A1CD2B28A18023301341070DBB2F2E781
:10F3A00074470020B723A72210B50B489B00C35811
:10F3B0009200995C042903D0995C084CC9B2195594
:10F3C00004219954C37A002B04D00623044A1169FE
:10F3D0000B43136110BDC046744800209D0200001D
:10F3E00000ED00E0F7B50F0040250400403F006845
:10F3F0000193AF4304239C461A4EC5690D40A942B0
:10F4000001D100201BE03568019BAD1AAB4226D329
:10F41000634605681D42F0D0002FEDD0C369082572
:10F420001E002E402B420BD005622000FBF76DF929
:10F43000230090331D600023012084342370FEBD1F
:10F440008025C3692D012B42D4D005622000FBF733
:10F450005CF923002022903384341A602670032044
:10F46000EDE7C04604050020F0B589B00F00049216
:10F47000002800D199E0431E012B00D9BEE0624B69
:10F48000624E05931B68624C07933378012B4ED86C
:10F49000B13422785F4B9200D458FA252200AD3265
:10F4A000127821269200D258AD0010008C3288309C
:10F4B000036811680B433340212B00D178E0200012
:10F4C00088300368202B70D1002F6ED06B461B8ACA
:10F4D000002B6AD08022A1685201914204D1226996
:10F4E000002A01D1FA0760D422000025903215606D
:10F4F00021220260059A26001268563605922200E3
:10F5000054321380338080235B01994204D12369F4
:10F51000AB4201D13D001F003388002B50D1FA23AC
:10F5200040212000059A9B00FFF75CFF51E03A4B19
:10F53000022019000693FCF774F9002835D0002347
:10F540003370344E35689D4206D002200699FCF790
:10F5500068F92B6883429BD0230001227668B1337F
:10F560001A70002E06D002200699FCF75AF933686B
:10F5700083428DD0022523002800B13326491D7017
:10F58000FCF74FF9002810D0230000229621A03369
:10F590001D602000130003920292019200928901E3
:10F5A000FCF7C0FD002800D072E7049809B0F0BD58
:10F5B000059B07991B685B1AAB4200D278E7F4E71A
:10F5C000FA2380212000059A9B00FFF70BFF0028FB
:10F5D00003D0202388342360E7E72268002F09D175
:10F5E0002B880235DB05DB0D93623388013B9BB230
:10F5F000338091E73B7801379362F6E70368049A1A
:10F600005B689847D1E7C04604050020AD020020A2
:10F61000FC01002048460020904E0108AE22002147
:10F6200070B5354B520099541A7C8A4213D0A922E6
:10F63000FA2632485200573105689C5AFF31B6000D
:10F640005A5A944207D00268521BB242F8D3A922F8
:10F65000595A520099521A0094321268002A28D03E
:10F660004622FF329C5C002C29D0012C35D0244A44
:10F67000A1008A58002A16D01500242101261068FE
:10F68000883529600168B143016000210160416053
:10F690008160100090300160043829600160D166FB
:10F6A000116784321170174A1178A14201D10221E9
:10F6B0001170A8225200995A0432995270BD8021CB
:10F6C000114AC901106B01431163116B0F480140CE
:10F6D0001163116C01401164C9E780210A4A890253
:10F6E000D06A0143D162D16A09480140D162D16B2D
:10F6F0000140D163BBE7C046FC4F00200405002059
:10F7000048460020AD02002000100240FFBFFFFF6E
:10F71000FFFFFDFF124B4022D968F0B508001040F2
:10F72000114201D00020F0BD8021FA26DC68B6002D
:10F7300021430C4CD9602568D9680F00174011424D
:10F74000F1D10328EFD021683800491BB142F3D929
:10F75000D9681142E6D103200349C877ECE7C046D7
:10F7600000280040040500200E050020802210B56E
:10F770000F4CE3689343E360A369603A134207D1F7
:10F78000FFF718FA002802D003200A4BD87710BDE3
:10F79000A3699343A361FFF70DFA002802D0032069
:10F7A000044BD8772023A2691343A361EFE7C04637
:10F7B000002800400E050020FA2130B58024134AAD
:10F7C0008900136864025B1811490869204204D05B
:10F7D00010688342F9D8032007E00B690D48034005
:10F7E0000B6103D001200C4A536030BDFA20802405
:10F7F000136880001B18E4020D6928002040254290
:10F80000F3D010688342F7D8E5E7C046040500202E
:10F8100000200240FAC300004C0600200F4A0300FB
:10F8200010B5904207D80E4B986AFEF704FE0021EF
:10F83000FEF74CFE10BD0B4A904209D90A4A00203F
:10F840009342F7D8064B986AFEF7F5FD0221EFE7E1
:10F85000034B986AFEF7EFFD0121E9E7A08601005E
:10F8600058100020801A060040420F0030B5284B87
:10F87000284A1B78D9B2002B02D113006C331970BF
:10F880001300242101206D331970D36A946B196819
:10F89000556B814319602048116B014019619968CB
:10F8A0001E4801409960012C07D18021090229439B
:10F8B000996059681A4C214009E0842109022943C2
:10F8C0009960022CF5D180215C68090121435960BF
:10F8D0005C68144921435960D9680140D960106CB3
:10F8E000D16B0143506C00020143D960D06C916C24
:10F8F00001431960012118680143196013000020B9
:10F9000020216D3310671970D0656E32107030BDD4
:10F91000C510002058100020FFFFFFF0FF7FFFFF01
:10F92000FFF7FFFF00800002F0B5AA23984C87B0D4
:10F93000002850D1A3652300BE331978042501297E
:10F940006AD1E369934FA57E0293628C3B6803936F
:10F95000002A00D077E0230005926D331A78202A20
:10F960004CD1E26A906980220600120216401042D1
:10F9700044D122006C32107801283FD0117024222B
:10F980001A702667A36B012B27D1834BE16A2B43A7
:10F990004B6038688B698A699B06D206DB0FD20FF1
:10F9A00013431CD08A69102316001E401A4241D10D
:10F9B000FFF77AFA002832D0236F042B03D12022DC
:10F9C000E36ADA612667059B01330593059B059B76
:10F9D000002BD7D007E01B02ACE7704BD6E73B68A3
:10F9E0001B1A642BD6D9220020236D321370226F8C
:10F9F00013432367230000226C331A706D3423787D
:10FA00000225202B14D00425614C2000FEF7F8F9C4
:10FA1000002363840534E377E8B207B0F0BD202308
:10FA2000E26AD36122006C346D32137020700025BD
:10FA30006DB2E9E7CB61FFF737FA0028C3D1202286
:10FA4000E36ADA61BFE70026A36D6C342178504881
:10FA50008C4653490C78202C00D090E06446012C51
:10FA600000D18CE0040001276C34277021240C7035
:10FA70000100113C6E310C70040000210700563467
:10FA8000016722800299474A0165836502662288E0
:10FA900045495437FF2A19D98020FF224004844663
:10FAA0003A801940002919D13948029FC46A3F7829
:10FAB000A7620700029C5637013404653C88543025
:10FAC000013CA4B23C80541E048008E02288806D72
:10FAD00092B284463A801940002AE3D100222C4C8D
:10FAE000E06D112806D1AA2B04D0AA2700203F02DE
:10FAF000BB420CD1A36DAA2B39D10023A3652300EF
:10FB000056331B88FF2B01D8A36D9C462748284FEE
:10FB1000D2B2002902D0230054331A786346290058
:10FB200000903800F9F75AFF230000226C330121BE
:10FB300038001A70F9F768FF2100164B6D311A680A
:10FB40000878202806D0632E04D81E68206FB61AC5
:10FB50000028F5D0236F632E00D954E79A0600D50C
:10FB600051E75A0712D4002B00D160E74BE7AA23D4
:10FB7000A06D1B029842C2D180239B04BEE73E6861
:10FB8000039C361B642E00D864E73CE703254FE74F
:10FB90005810002004050020002000020028000268
:10FBA000C5100020A59D0008FFFFFFFD002000807C
:10FBB00084100020C3B23C2B09D8E0220F499B00DF
:10FBC000D2000240585810430D4B18677047C022AE
:10FBD0000240C02A0ED1CE2B0CD83F230949034046
:10FBE0009B005B58E021054A9B009B58C9000840D8
:10FBF0001843E9E701204042E6E7C046444A0108CD
:10FC00003C110020C0420108C3B23C2B09D8E022BD
:10FC10000F499B00D2000240585810430D4B986684
:10FC20007047C0220240C02A0ED1CE2B0CD83F23F1
:10FC3000094903409B005B58E021054A9B009B5803
:10FC4000C90008401843E9E701204042E6E7C04602
:10FC5000444A01083C110020C0420108C3B23C2BB9
:10FC600009D8E0220F499B00D200024058581043A7
:10FC70000D4BD8667047C0220240C02A0ED1CE2B51
:10FC80000CD83F23094903409B005B58E021054AFB
:10FC90009B009B58C90008401843E9E701204042F7
:10FCA000E6E7C046444A01083C110020C042010872
:10FCB000F0B5A64BA64C89B005000E00E06E190009
:10FCC00005920393FBF7ADFDA2490700A06EFBF779
:10FCD000A8FDA1490090206FFBF7A3FD636F019081
:10FCE0009E4918000293FBF79CFD0490002F00D161
:10FCF0000CE1009B002B00D108E1019B002B00D1FF
:10FD000004E100993800FCF7F3F804990700019822
:10FD1000FCF7EEF8010000903800FCF7E9F86066A7
:10FD2000002F00D1F2E0009B002B00D1EEE0002874
:10FD300000D1EBE0029B206001335A425341884AD4
:10FD40005B4213408022D2029B18A36182235B0096
:10FD50006360FAF7F1FB00234208AA4218D982082F
:10FD60000833954214D2C2080833954210D20209D2
:10FD7000083395420CD242090833954208D28209D1
:10FD80000833954204D2C0090833854200D20833B3
:10FD9000E3613500331E07D00023022E04D0731E0A
:10FDA0005A1E93415D00012363610723E362E02350
:10FDB000DB00E360059B00265A425341DB012362CE
:10FDC00025616B425D410399E06EA660A6626662A2
:10FDD0006663FBF717FD5F49A06EFBF713FD276F06
:10FDE0005D493800FBF70EFD3B0630006A1C1B0F17
:10FDF000042B02D85B499B0058580F215A4B0F40E7
:10FE0000BF00F958FBF75DFC5449606FFBF7FAFC43
:10FE10002268564B9A4200D07AE08021544B490127
:10FE2000186C08431864186C084007900798186B02
:10FE300001431963196B4F4801401963666A616891
:10FE4000002E00D07AE082235B00994200D0E66168
:10FE50000023A36223005D331B78D8B2002B02D1AC
:10FE600023005C331870230002205D331870136880
:10FE70003E3083431360E023E568DB009D4261D997
:10FE8000F02300271B019D4201D00023A3628420A0
:10FE9000A36900020093A368034082204000014050
:10FEA0000B4303382169FF3801400B436169013876
:10FEB00001400B43802100988900014038200B430A
:10FEC000E16901400B43216A483001400B4308219E
:10FED0001360636B0B4049180E401E43F0231B0157
:10FEE0001D40009B3543180C042318402843384319
:10FEF0005060D369204901200B40D3610023236661
:10FF000040235D34207011680B43136009B0F0BDCD
:10FF10001A4B9A4200D091E78021154BC901D86B4A
:10FF20000843D863D86B084006900698D86A014306
:10FF3000D962D96A12480140D9627FE70023236160
:10FF4000636185E780277F019DE7C046705D0108FA
:10FF50003C110020C85C0108445C0108B45B010846
:10FF60000002FCFFC44B0108D84B010800300140DF
:10FF700000100240FFEFFFFFFFF7FFFF00380040D7
:10FF8000FFBFFFFF0A4A10B511680221094B1B6829
:10FF90009C680C42FCD00121187398680842FCD080
:10FFA000187B12688022C0B299681142FCD110BD42
:10FFB000040500203C11002070B505003235040016
:10FFC0002800F4F711FC002806D1FAF763FE002898
:10FFD0000BD02800F4F7D4FE1B2022000021034B95
:10FFE000F4F712FC0120F0F7C2FF70BDE0250020FD
:10FFF00013B50D4A0D4B118801AA89B21180190061
:020000040801F1
:100000006846C4310988063089B20180C2331C8831
:1000100011888C4203D810881B88C01A16BD00882E
:1000200012881B888018F8E7304E0020704D0020A1
:1000300013B56946174A184B1288063192B20A80E6
:100040001A00C0321488088884421AD310887F2886
:1000500005D91288802A07D10A88002A04D01A00FC
:10006000C0321088181813E00A880020402A0FD9DF
:100070001A001C00C0321188C43489B2218010805B
:10008000EFE710880C88010040310020A142E8D33E
:1000900016BDC046324E0020704D0020836810B55A
:1000A0000400002B05D00322010098470023A36021
:1000B000E36010BDC3B270B53C2B39D8E0222949AA
:1000C0009B00D2000240585810430F2103090B40F7
:1000D000042B2CD8244A9B009B58002B27D00123AB
:1000E0000840834000249BB2012B37D1142666437D
:1000F0001E4D301D4019FFF7D1FF2B000022715714
:1001000000201856884202D1D86800280FD1013249
:100110001433102AF4D11649164AA000CB6F825826
:100120009343CB6714236343E856F9F7D1FB70BDC3
:10013000C0220240C02A0ED1CE2B0CD83F230E493C
:1001400003409B005B58E021064A9B009B58C90076
:1001500008401843B9E701204042B6E701345B0884
:10016000E4B2C1E7444A0108C44B0108BC4E002078
:100170000418024060590108C0420108F0B5524B12
:1001800005001B780E00514C87B0012B00D082E097
:10019000A38A994209D92021206903F003FF00288E
:1001A00000D17AE020232061A382AA2369000025E0
:1001B0001B02A365CBB202932369454A0393B3B2F2
:1001C00004931368A06D05936C3427783F4B414C22
:1001D0002178202900D06EE0012F00D16BE01A00B9
:1001E00001276C321770222222701A0010246E32FE
:1001F000147000221A67039A374C1A651A001C669D
:100200001C00049956321180986517885434FF2FCA
:1002100044D9FF22802322805B042C4CE76D122FEF
:1002200006D1AA2804D0AA210027090288420BD1AE
:10023000A06DAA2837D10020A06520005630008884
:10024000FF2800D8A36D254F25480299D2B2009708
:100250000700F9F7C3FB230000226C3302213800AA
:100260001A70F9F7D1FB2100194B6D311A68087823
:10027000202806D0632D04D81D68206FAD1A0028F1
:10028000F5D0236F632D1CD8F6B2002B19D10022B4
:100290000E4BDA821E8307B0F0BDFEE712889B6D1D
:1002A00092B22280B9E7AA20A76D00028742C4D18A
:1002B00080208004C0E7156805996D1A642D00D868
:1002C00086E70026E3E7C0461611002058100020FC
:1002D00004050020C5100020A59D00080024008012
:1002E0008410002010B5C1B20148F8F7D9FF10BD45
:1002F00058100020F7B5104C0193237806000092A7
:10030000012B18D00127002327706360FFF754FAF0
:1003100000280ED1094D6B693B436B61009B336034
:10032000BFF36F8F019B7360FFF746FA6B69BB43A6
:100330006B6100232370F7BD4C06002000200240B3
:1003400070B504008C342368202B63D1802382682D
:100350005B019A4204D10369002B01D1CB0759D428
:100360000023C36603685B681B020CD5EFF310859E
:10037000012383F3108880230268DB04166833436B
:10038000136085F31088030001225C3381651A80B5
:100390005A80802100238268436749018A423AD10A
:1003A00003695A4253411B02FF330200603213803B
:1003B0000300002290331A6022232360EFF31081A0
:1003C000213B83F31088026894682343936081F390
:1003D000108880248022456E81680369A40552013B
:1003E000A5423ED1040068342488012C39D89142BA
:1003F00032D1002B21D12C4B4367EFF31081012325
:1004000083F31088802302685B0590680343936040
:1004100081F3108870BD002A05D10269FF23002AEC
:10042000C3D0803BC1E7802149058A42BDD1026922
:100430007F23002AB9D0403BB7E71C4B4367EFF35B
:100440001081012383F310880268FF33146823436B
:10045000136081F31088D0E7144A4267002BCCD098
:10046000EDE791421AD1002B0AD1114B4367EFF30C
:100470001081012383F3108802681F3310680AE09B
:100480000C4B4367EFF31081012383F3108802685C
:1004900020331068FF3303431360B9E7054A42670E
:1004A000002BE4D0EEE7C046E9C900082BC80008DD
:1004B000997D0008CD7C000870B5041E1ED0FBF7A6
:1004C000B7FF00281AD122002100B13212780C4B5C
:1004D0009200D058B2310D78FFF732FF22003F2151
:1004E000C032138801330B402100BC3109888B4294
:1004F00004D0B434118820684554138070BDC046C0
:10050000484600207FB5AF2306221A4C5B00E25418
:100510000022194D194E6866E37C01000393A37C09
:1005200030000293637C009201931300FBF7FAFD05
:10053000AE235B00E05400281AD02000FEF750FAEA
:100540003000FBF775FF002812D10D4B2B63A2255D
:100550006D006057F9F7BCF94622FF32A25C094BE7
:100560009200D0580849FFF7EBFE6057F9F7A4F95D
:100570007FBDC046FC4F0020F85000209050002066
:10058000B90401084846002042510020F8B5070090
:10059000282241373B7804000D001340934204D1D8
:1005A000002903D180239B004364F8BD2600254920
:1005B0004036F9F765FA3378012BF6D00121317016
:1005C0003B78292B16D12000F9F75AFA23681A68CC
:1005D00052040FD51A681C49A06B0A401A60002803
:1005E00008D01A4B8363F9F7ADF9002802D0A06B4D
:1005F000836B98472A233B702300202242331A70D2
:1006000000236364236812495A680A4001215A6032
:100610006185628D6562228580225204E2620D4A04
:10062000986962639A69120C0A4203D10822104247
:1006300000D0DA610023200002493370F9F7E4F9B1
:10064000B3E7C04602800000FFBFFFFFA1820008A1
:10065000FF7FFFFF11A30008F7B50600913633783E
:1006600004000F00051F012B09D1AB6E002B06D033
:10067000EB6E28009847022333700023AB660023FB
:10068000012F66D1337026002A6F90369A4202D02D
:10069000280033709047337826002822DBB201937C
:1006A000413633781340934205D1019B002B03D18F
:1006B00080239B006364F7BD250020002A49403554
:1006C000F9F7DEF92B78012BF5D001232B70337865
:1006D000264F2A2B16D102212000F9F7D1F92368E1
:1006E0001A6812040ED51A68E06B3A401A600028A6
:1006F00008D01F4B8363F9F725F9002802D0E06B7F
:10070000836B9847292333702300202242331A70C9
:100710000023636423685A683A405A6022007032AA
:100720006262019A6285628D228580229204E26271
:10073000104A996962639A69D20303D5082211426B
:1007400000D0DA610023200007492B70F9F75CF92B
:10075000B1E7AB6601233370AB6E20007433E91848
:10076000FFF714FFA7E7C04601800000FF7FFFFFEF
:10077000A182000811A30008B2239B00C0580723E0
:1007800028220B405A4349B2F0B58418002923DAD5
:1007900001211432821861751370A5239B00C15C7E
:1007A000012953D00121C15411780368157B8900B8
:1007B00054785B18334A002D21D11968002C13D0CE
:1007C000490605D51C6830490C4030492143196061
:1007D00019682F4C214033E0002155325634FF3246
:1007E000FF3482182170D7E7490405D526491C68D3
:1007F0000C402849214319601968274CEAE78025F5
:100800002149234EED01002C21D11C682C4204D03B
:100810001F68204C0F403C431C601C681B4F640643
:1008200003D51C680C403C431C601C6821400F43EE
:100830001F601968184C2140114319601968314034
:100840000A431A60A52300229B00C254F0BD1C6815
:10085000104F2C4203D01C680C403C431C601C68A9
:10086000640606D51C680C40A4466546074C2C431C
:100870001C601C6821400F431F6019683140114300
:10088000B9E7C046808000008F8FFF07C08000005E
:10089000BF8FFF0780C000008FBFFF07F7B5072598
:1008A0002826B2240D406E43A400005949B2844664
:1008B0008019002952DA01211436664441753570D9
:1008C0003361F270022A01D100233371A5236146FE
:1008D0009B00C95C012940D060460121C1540368D6
:1008E000A9005B18196891480140022A04D0032A24
:1008F0003CD08020800001438D488E4C014319601C
:1009000019688D4F2140294301431960E900C91935
:10091000377B002F00D06AE07278002A29D00A685D
:10092000120C12040A60F2880D68920892002A43A1
:100930000A601A68520604D51968804A21400A43A1
:100940001A607F4A1968114020224A4002431A6007
:10095000A523002261469B00CA54F7BD00215536ED
:100960005630FF36FF3066440170A8E7C020C00053
:10097000C1E74A68120C12044A60F2884F68920874
:1009800092003A434A604A68920192094A60326989
:10099000002A05D14E688022120632434A600BE0DD
:1009A0003E2A1AD801274E68174001965608F619B4
:1009B000019AB60616434E601A68520404D51968A7
:1009C000604A21400A431A605F4A19681140C022F8
:1009D000002D00D080229201B7E71F2756093A4028
:1009E00057427A41B61A4A68B6061643D3E7022A36
:1009F0003AD11D68554A25402A431A600A68120CEC
:100A000012040A6032890D68920892002A430A6033
:100A10004A68120C12044A6072894D68920892006A
:100A20002A434A6080227778454DD201002F61D158
:100A30001F68174204D01F68424A27403A431A6091
:100A40001A68520604D51A6814403C4A22431A60B8
:100A50000A68920192090A603269002A09D1802449
:100A60000E68240634430DE01A68394D2A400243CB
:100A7000C3E73E2A13D80126540816400F68A4196C
:100A8000A4063C430C604C68A401A4094C60002AF5
:100A900011D14C688022120622434A6015E01F26BD
:100AA000164077427E415409A41B0E68A4063443C5
:100AB00080263606D6E73E2A12D80126540816406C
:100AC0004F68A419A4063C434C6019681E4A1140A3
:100AD000C02292014A4002431A601A682A4035E750
:100AE0001F265409324056427241A41A4A68A4068D
:100AF0001443CFE71968114204D01968114A214004
:100B00000A431A601A68520604D519680B4A214034
:100B10000A431A602022196829404A4002431A6099
:100B20001A6809490A401043186011E78F89FF07C6
:100B3000808000008F8FFF0700980040C080000079
:100B4000BF8FFF0780C000008FBFFF0780810000BC
:100B50008F8EFF07AE2310B59B00C3585B68984784
:100B600010BDF7B50324D31C2240144C9BB20919C5
:100B70001400651EAC419B081B1B04009B000191E7
:100B8000C718BC420ED1002A0BD0C918C0180023C8
:100B90000C682500D900CD401D54013399B28A421A
:100BA000F7D1F7BD019E20CE01962E0A2570667002
:100BB0002E0C2D0EA670E5700434E2E7009800407C
:100BC000F7B50324D31C22401400651EAC419B08DA
:100BD0001B1B144C9B00091904000191C718BC424F
:100BE0000FD1002A0CD000242500C018265CE70095
:100BF000BE4001343543A6B2B242F7D1C9180D60E8
:100C0000F7BD2578AC46664665782D023543A67853
:100C100036042E43E57804342D063543019E20C664
:100C20000196DCE700980040F0B585B001904A7865
:100C30000C000B7B012A00D006E10F698D69BD42D3
:100C400000D93D006069002B1CD1AAB2E188FFF7F2
:100C5000B7FF2378A24ADB009B181A682D0492B2D2
:100C60001A601A6815431D602378019A9B00D318F7
:100C700019689C4A114030224A409B490A431A6035
:100C800005B0F0BD2178964ECB009B19E67889001F
:100C9000B446019E226A71186646022E00D0BDE05D
:100CA000974200D3AAE00F68904A2E041740904A5A
:100CB00003963A430A60226A4719521B22620A6865
:100CC0004021944666460A400292AAB20E424BD098
:100CD00059682E0489B25960596831435960618955
:100CE000FFF76EFF226A2169002367618A4201D9FA
:100CF000531B2A0023626378002B29D1237878497B
:100D0000DB005B181968890189091960002A0AD17A
:100D100080211868090601431960218992B23800C0
:100D2000FFF74EFFA0E73E2A06D8012551081540DF
:100D3000491918688906EEE71F20104045426841AE
:100D40005109091A18688906014380200006E2E764
:100D5000012BE2D123786249DB005B18196889B264
:100D6000196018681104D6E719682E0489B2196051
:100D70001968314319602189FFF722FF226A23692C
:100D800067619A4202D9531B2A000293029B236295
:100D90006378002B26D123785149DB005B18596812
:100DA000890189095960002A07D1802158680906FC
:100DB00001435960618992B2B1E73E2A06D8012504
:100DC00051081540491958688906F1E71F2010405D
:100DD000454268415109091A586889060143802033
:100DE0000006E5E7012BE5D123783D49DB005B18E0
:100DF000596889B2596058681104D9E70D683D4FA8
:100E0000394E3D4035430D60196889B219601D683F
:100E100011042943196092B2218981E7521B226291
:100E20000968AAB22F04490607D5596889B25960E2
:100E3000596839435960618972E7196889B2196044
:100E40001D683D431D60E7E7002B28D10B788A69B8
:100E500001999B00CB18002A1CD1E278002A19D1F5
:100E6000224A19681140224A0A431A60A36922697A
:100E7000934232D99B1AA3612378019A9B00D6181A
:100E800033681D4A1340C02292015A40164B134347
:100E90003360F5E6174A19681140134AE4E7CB7846
:100EA000022B17D1CB69002BE6D00B78019A9B005F
:100EB000D318402219680A40490408D5002ADBD01B
:100EC00019680A4A11400D4A0A431A60D4E7002AF9
:100ED000D2D1F5E7012B00D0D2E60023CBE7C04604
:100EE00000980040BF8FFF07808000008F8FFF07B2
:100EF000808100008F8EFF078FBFFF07C08000003A
:100F000070B5B224A40005590720014021304843A0
:100F10002C182600FC36F266220033670023563276
:100F20005534FF32FF3455307367FF301370217032
:100F300029182868FFF778FE70BD70B5B224A400A8
:100F4000055907200140213048432C182600A26291
:100F500001223836E3623270636300232175236314
:100F60006275143029182868FFF75EFE70BD130003
:100F7000A52210B50224920084500A00836100214A
:100F8000C361FFF7DAFF10BDA52304229B0010B553
:100F9000C25000231A001900FFF7CFFF10BD70B533
:100FA0000400002929D1A5239B00C358032B0FD18E
:100FB00005005535FF35A868EB68984209D9C01A75
:100FC000A860834200D9030000212000FFF798FFAA
:100FD00070BDA7239B00E35C032B0AD1AE239B00CB
:100FE000E3581B69002B04D0B52292002000A150C9
:100FF00098472000FFF7C8FFEAE7A7239B00C35CE0
:10100000032BE5D1AE239B00C3589B69002BDFD097
:10101000B52200209200A05020009847D8E7030096
:10102000F7B504000F00002564330093009E503391
:10103000019330000C22002101F07AFE019BF56043
:101040001036B342F5D13800F9F755FC2200504B69
:1010500080000C322761C2502700230026002C3369
:101060004C374D361D7025636563A563E5632564C4
:101070006564A5643D703570256625000323103531
:101080002800E460E365FAF745FF0098FFF706F8EB
:10109000009B019A103300939342F6D100233D4AFE
:1010A00023606360A3606361A36123626362803332
:1010B000E261A3623378DAB2002B1ED13A702800C5
:1010C000FAF728FF2069FAF7CDFF0500E16DF8F780
:1010D0000FFC2800F8F7F0FB27693800FAF7F2FF59
:1010E00005003800FAF7BEFF854206D02800E16D02
:1010F000F8F7FEFB2800F8F7DFFB022333702369C3
:1011000025481A68834206D08021C9058B4202D047
:1011100022498B4208D170218A43A1690A432049A0
:101120001140226A0A4308E01E498B42F7D01E494B
:101130008B42F4D01D498B42F1D08021A56A8A43AD
:101140001543E269DA6262699A62834205D0164AFF
:10115000934202D0154A934201D1626A1A63042273
:10116000186802431A6001225A611D602300583337
:101170001A7057340A3B1A705A709A70DA701A71E2
:101180005A719A71DA711A7222703270F7BDC046C4
:1011900020460020FFFF0000002C0140000400401A
:1011A000FFFCFFFF002000400044014000480140D8
:1011B000F0B5AA4E89B00691310007920190FAF776
:1011C00030FBF9F798FBA64F8500EC59002C0ED1A7
:1011D000B42001F0E1FF310002900198FAF721FB01
:1011E00001000298FFF71BFFEC59029B23603100BE
:1011F0000198FAF74DFB0003C00E431E0493032B26
:1012000016D824684300E3189C465B880593830046
:101210000393043B0293059B042B00D1EBE0039A5C
:101220002369042A05D0039A082A50D1996B01E05A
:10123000FEE7596B22004C32107801282FD001268E
:101240001670029A8748082A75D000D99CE0002AB7
:1012500049D11A6A1D6AB5431D625E68824D9F6955
:101260003D4060273D43834238D08048834235D09B
:101270007F48834232D0022082435E609D61596381
:101280001A62082299690A4304219A619A698A4379
:101290009A619A699A61230000224C331A700423E0
:1012A00062465380019B013300D1A4E06B4D01984D
:1012B0002900FAF7EDFA0003C00E431E032B00D9F4
:1012C00087E0039B8000834200D183E0FEE7039A1E
:1012D0000C2A01D1D96BADE7196CABE70E20824324
:1012E00064480640C9E710261A6A1D6AB5431D62A4
:1012F0005E68614D9F693D40C027FF013D438342C9
:1013000004D1E02082435D48064007E0202082436C
:1013100056488342F7D056488342F4D05E609D61C0
:1013200099631A628022996912010A439A619A6943
:1013300053490A40ACE71E6A524D1A6A2A401A62A3
:101340005D68494ADF693A4060273A43834204D1E5
:101350004D4830404D4E354007E04D483040434EFB
:10136000B342F7D0424EB342F4D05D60DA61082256
:10137000D9631862D9690A430421DA61DA698A43B8
:10138000DA61DA69DA6186E71E6A424D1A6A2A4032
:101390001A625D68384ADF693A40C027FF013A4364
:1013A0003D4F3740834205D03048834202D0304819
:1013B000834201D1394805405D60DA6180221964B9
:1013C0001F62D96912010A43DA61DA692C490A40BD
:1013D000D6E7FEE729000198FAF714FA29000198E8
:1013E000FAF756FA0122C00200D50F32049BE35CE3
:1013F0001343049AA354022220000699F9F7B8FA7D
:1014000025690798AB6AEB6A25490133584300F018
:1014100053FCEB6A234A934203D10132904200D13C
:101420001800029B002B0CD1686329002000F9F7FB
:1014300049FA059B042B02D02000F9F799F909B06D
:10144000F0BD029B042B01D1A863EEE7029B082BA1
:1014500001D1E863E9E72864E7E7C046184F0108CF
:1014600020460020002C01408CFFFEFF004401407C
:1014700000480140FFFCFFFFFF8CFFFEFFF3FFFF72
:10148000FFFBFFFFFFFEFFFFFFF1FFFFFFCFFFFFAF
:10149000FFFDFFFFFFEFFFFFFFDFFFFFFFBFFFFFCE
:1014A000FF030000FFFF00000300002904D14433C4
:1014B0001A78012A0AD07047042901D14533F7E789
:1014C000082901D14633F3E74733F1E702221A70C6
:1014D00004228A400368196A91431962196A0A430F
:1014E0001A628022596C12020A435A640B4A9342D0
:1014F00006D08022D205934202D0094A934207D1F6
:101500009A6808490A40062AD5D007398A42D2D0BB
:10151000012219680A431A60CDE7C046002C014039
:101520000004004007000100030008293AD03BD81E
:10153000002935D13E331A7806331B78D2B2DBB29C
:10154000012A2CD1012B2AD10200013308292FD0E6
:1015500030D800292AD13E321370937101220368DA
:10156000100088400100186A88431862186A014315
:10157000196212498B4206D08021C9058B4202D0E4
:101580000F498B4218D19A680E490A40062A06D0A4
:1015900007398A4203D0012219680A431A6070474A
:1015A0003F33C8E74033C6E74133C4E73F32D3E7B0
:1015B0004032D1E74132CFE71968EEE7002C014015
:1015C0000004004007000100030008290DD00ED8D8
:1015D000002908D13E331B78013B5A1E9341DBB2F0
:1015E000002B06D070473F33F5E74033F3E7413334
:1015F000F1E702230200082929D02AD8002924D1A2
:101600003E32137001228A400368196A91431962BD
:10161000196A0A4316491A628B4205D0154A934249
:1016200002D0154A934216D18022586C120202430E
:101630005A648B4216D19A6810490A40062AD1D0C2
:10164000802149028A420DD1CCE73F32D9E74032AE
:10165000D7E74132D5E78022D2059342EBD0084A42
:101660009342E8D0012219680A431A60BAE7C046DB
:10167000002C0140004401400048014007000100E7
:101680000004004003003D331978CAB2012918D183
:101690000131197003680C498B4206D08021C905BD
:1016A0008B4202D009498B420CD19A6808490A4002
:1016B000062A06D007398A4203D0012219680A4354
:1016C0001A6070471968FAE7002C014000040040D6
:1016D0000700010007220B000A40017910B5914272
:1016E00026D35CB22821002C23DA51430B000124BD
:1016F00014334118C3184C751A700121A522997032
:101700009200845C8C4213D081541A7801685C7812
:1017100092008B181149002C16D01C68104A1440F6
:10172000102262400A431A60A52300229B00C25483
:1017300010BD59430B000024411855335631FF3377
:10174000FF31C3180C70D7E71C68064A144080228A
:101750005201624011431960E6E7C04680800000F4
:10176000BF8FFF078FBFFF07B22310B59B00C05884
:10177000FFF7B0FF10BDB723324A9B0070B5051EBE
:10178000D4584BD1483BE358022B10D1E369216A6E
:101790008B4214D95B1A926A0100E3612000FFF7C3
:1017A000CCFB2B002A0029002000FFF7A9FBA8236F
:1017B0009B00E25C002A01D00022E25470BD8B4203
:1017C0000FD1A26993420CD8A626B600A3599A421B
:1017D00007D20300020001002000FFF7AEFBA55175
:1017E000DFE7A7239B00E35C032B0BD1AE239B0019
:1017F000E358DB68002B05D0B522002192002000C1
:10180000A150984780212000FFF7AEFFA5230522B5
:101810009B00E25000231A001900C5E7A7239B0094
:10182000E35C032BCAD1AE239B00E3585B69002B1A
:10183000C4D0B52200219200A15001002000984799
:10184000BCE7C0467448002010B504008021FFF7B3
:101850008BFF00212000FFF787FF10BD0A2382B015
:101860000193019B002B07D1054BC000C0180068F5
:101870008001800D02B07047019B013BF0E7C0463C
:10188000009800400A2382B00193019B002B07D1EE
:10189000054BC000C01840688001800D02B0704741
:1018A000019B013BF0E7C04600980040030028215F
:1018B00070B541331B78040002680B408B422ED177
:1018C000956993699168D068E068ED03ED0F02288F
:1018D0001BD1FC301B0C89050340490F4B401900FC
:1018E000F8380140034210D1A36C0133A364A36C08
:1018F000022B09D10633A164D36123004033197050
:1019000029002000FEF7A8FE70BD802120000902FA
:10191000F8F7B6F82300002240331A70F0E70823E6
:10192000D361002340342370EEE7030010B5413348
:101930001A78202A07D1802108321A70024B090236
:101940004363F8F761F810BD11A3000870B50126D4
:10195000FDF764FF0F4CE56A2B68B3432B602063EF
:10196000FDF784FF2B681E4323002E60BE331B78D7
:10197000002B0DD12300084D084A983328001A6027
:10198000FFF7D3FF064B943428002360FFF7CDFF09
:1019900070BDC0465810002084100020C388000885
:1019A000039300088022034B120659690A435A61C7
:1019B0005B69704700200240044B5A69002A04DA30
:1019C000034A9A60034A9A605B69704700200240AC
:1019D00023016745AB89EFCD836810B5002B02D09A
:1019E00003220100984710BDF0B589B00E0004AD88
:1019F00004000C220021280001F09AF90023B768A6
:101A0000EB6001979F4206D0022231002800B847C0
:101A1000F368B768019302AE29000822300001F094
:101A2000E2F92B00220003CA03C3230006CE06C33B
:101A3000A36828000693E368A7600793019BE3600F
:101A4000FFF7CAFF09B0F0BDF0B5C3B20E008BB00E
:101A50003C2B48D8E0216A4C9B001C59C90001402E
:101A60000C43022A55D0033A53425A41654B15059F
:101A7000ED1806AF0C220021380001F059F90023BF
:101A80000993B368002B07D0022231003800984731
:101A9000F3680993B36808930F2601232640B340E7
:101AA00001936B4600229B880292012B33D12006C2
:101AB000000FF9F73DF8041E32D11424029B524D59
:101AC0005C43201D401906A9FFF78EFF64570321D0
:101AD0002000F7F70DFF2000F7F7EEFE06A8FFF74E
:101AE0007BFF0BB0F0BDC0210140C0290ED1CE2B31
:101AF0000CD83F23454C03409B001B59E024404930
:101B00009B005B58E40004401C43AAE701246442A4
:101B1000A7E73F4DADE7029A5B080132D2B2C3E7B7
:101B20003C4BB600F158032349434B43C06818406F
:101B300000F0C2F880235B032B4004938023002134
:101B40009B031D4003900595019BCB40B5D0012719
:101B50003B008B40019A01981A4018424ED0032650
:101B60003500480085402368AB432360E368AB43FE
:101B7000039D854028001843E060274B88088000BB
:101B8000C018A023DB059C46056E0023644511D0D8
:101B9000224B9C463B0064450CD0214FDB18BC42D5
:101BA00008D0204F3300BC4204D01F4BE3185E1E08
:101BB000B341053303260F270E40F600B740B3406C
:101BC000BD431A4E2B430366F06F134B1043F0676F
:101BD000174E049FF06FD5439043F06710001E68C6
:101BE0003043002F01D13000284018605868059E0E
:101BF0000243002E01D102002A405A600131A3E7BE
